:020000040800F2
:1000000000000220813A0108A9990008AB99000874
:10001000AD990008AF990008B199000800000000F0
:10002000000000000000000000000000B39900087C
:10003000B599000800000000B7990008B9990008B8
:10004000C53A0108C53A0108C53A0108C53A010890
:10005000C53A0108C53A0108C53A0108C53A010880
:10006000C53A0108C53A0108C53A0108617C000893
:10007000C53A0108C53A0108C53A0108C53A010860
:10008000C53A0108C53A0108C53A0108C53A010850
:10009000C53A0108C53A0108C53A0108F59B0008B0
:1000A000C53A0108C53A0108C53A0108C53A010830
:1000B000B59B0008C53A0108C53A0108C53A0108D0
:1000C000C53A0108C53A0108C53A0108C53A010810
:1000D000C53A0108C53A0108099D0008C53A01085A
:1000E000C53A0108C53A0108BD990008C53A01089A
:1000F000C53A0108C53A0108C53A0108C53A0108E0
:10010000C53A0108C53A0108C53A0108C53A0108CF
:10011000C53A0108C53A0108C53A0108C53A0108BF
:10012000C53A0108C53A0108C53A0108C53A0108AF
:10013000C53A0108C53A0108C53A0108C53A01089F
:10014000C53A0108C53A0108C53A0108ED99000809
:10015000C53A0108C53A0108C53A0108C53A01087F
:10016000C53A0108C53A0108C53A0108C53A01086F
:10017000C53A0108C53A0108C53A0108C53A01085F
:08018000C53A0108C53A010867
:1001880034BF050800000020300C0020300C00208F
:10019800843D002008B5074B186809F08BFB0EF06A
:1001A800F3FA054B054806221A70BDE8084001F02D
:1001B800C4BD00BFE4260020712600204C1000209A
:1001C80008B5034801F0B9FD024B00221A7008BDBA
:1001D800A01800207126002008B5054B0122002038
:1001E8001A7005F0FDFF0348BDE8084001F0A5BD01
:1001F800FC2C0020101600202DE9F041144C20465C
:1002080004F071F900201349134A03F023FF13493E
:10021800134A0746002003F01DFF1249124A0646FA
:10022800002003F017FFD22105463A462346F62060
:1002380004F028F8D22132462346A62004F022F8FA
:100248005620D2212A462346BDE8F04104F01AB8C8
:100258002414002016AB0508C90100081FAB0508C7
:10026800E101000828AB05089D01000808B502F067
:10027800B3FC034801F061FD024B00221A7008BD6F
:10028800A018002071260020034B0D224FF4864051
:100298001A700FF09BBA00BF71260020034B0D2285
:1002A8004FF402401A700FF091BA00BF7126002077
:1002B8000F4B0D2270B51A7000240BE0A8B2002273
:1002C8003146013505F0FCF8B5F5A07FF6D10134CB
:1002D800CE2C02D00025A6B2F0E70D2000F09EFC3F
:1002E8004FF441400FF0E6FABDE8704004F034BB2B
:1002F800FC2C00202DE9F347234D0024284604F068
:10030800F2F8234622464FF6FF71204800940194E4
:1003180003F0A8F91E491F4A8146204603F09AFEB9
:100328001D491E4A0746204603F094FE1C491D4AF3
:100338008046204603F08EFE1B491C4A064620468E
:1003480003F088FE214682464A462B46204603F0A3
:1003580099FF64213A462B460A2003F093FF8C212B
:1003680032462B460A2003F08DFFB42142462B4625
:100378000A2003F087FFF620D22152462B4602B00E
:10038800BDE8F04703F07EBFA80F002031AB050899
:100398003DAB0508A50200084CAB0508B9020008EA
:1003A8005BAB05089102000816AB0508750200084A
:1003B80008B5054B012200201A7005F011FF03480B
:1003C800BDE8084001F0B9BCFC2C00201016002044
:1003D80008B5034801F0B1FC024B00221A7008BDB1
:1003E800A01800207126002008B5054B07221A70B6
:1003F8000EF0CAF90348BDE8084001F09EBC00BFF2
:1004080071260020241400202DE9F041144C2046C8
:1004180004F069F800201349134A03F01BFE13493E
:10042800134A0746002003F015FE1249124A0646F1
:10043800002003F00FFED22105463A462346F62057
:1004480003F020FFD22132462346562003F01AFF3C
:10045800A620D2212A462346BDE8F04103F012BF68
:100468004C10002016AB0508D90300086AAB050834
:10047800F10300081FAB0508B9030008014801F0A3
:100488005CBC00BF3812002010B5094C204604F0AF
:100498002AF800200749084A03F0DCFDD221024669
:1004A80023464FF48270BDE8104003F0EBBE00BF56
:1004B8005817002073AB05088504000870B50C4C6C
:1004C8000C4D20684FF6E076314603F007F92068B6
:1004D800294603F0B1F86068314603F0FFF8606818
:1004E800294603F0A9F8BDE8704004F035BA00BF0A
:1004F800300C002074B1050838B52B4CFFF7DEFF2F
:10050800002005F06DFE237A23B90A203221274AFC
:1005180005F074FF637A23B90A206421244A05F0A0
:100528006DFF214CA37A23B90A209621214A05F0B0
:1005380065FFA37A1C4DFBB16B7AEBB12B7ADBB16B
:1005480000232B726B72AB721B4B286801221A7046
:100558004FF6E07103F0C2F82868184903F06CF808
:100568006868174903F068F80BF0E1FC04F0F4F947
:10057800144804F035FA0DE00B4C4FF4784120682C
:1005880003F0ACF82068104903F056F860680F498A
:1005980003F052F8FFF792FF00200BF08BFC0C4899
:1005A800BDE8384001F0C9BB300C00207AAB050823
:1005B80088AB050897AB050871260020A5AB050890
:1005C80075B1050880969800B9AB050877B105089C
:1005D800A018002008B500200BF06CFC0248BDE80C
:1005E800084001F0AABB00BFA018002038B5FFF7EB
:1005F80065FF0EF0E1F83C213F220023DF2005F0E3
:10060800DFFE4FF480600EF01BFE124C3E223C21B0
:10061800DF20002305F0D4FE012323720E4B4FF692
:10062800E075186809F046F92068294603F056F87D
:1006380020680A4903F000F86068294603F04EF87C
:100648006068074902F0F8FF04F086F9054B0022BC
:100658001A7038BD300C0020E4260020CBAB05080A
:10066800DEAB05087126002038B5FFF727FF0EF02E
:10067800A3F86E213F220023DF2005F0A1FE4FF4EE
:1006880086400EF0DDFD124C3E226E21DF20002355
:1006980005F096FE012363720E4B4FF6E07518685D
:1006A80009F008F92068294603F018F820680A4973
:1006B80002F0C2FF6068294603F010F86068074935
:1006C80002F0BAFF04F048F9054B00221A7038BD51
:1006D800300C0020E4260020F1AB050802AC050828
:1006E8007126002010B5FFF7E9FE0EF065F8A0218D
:1006F8003F220023DF2005F063FE4FF402400EF096
:100708009FFD114C3E22A021DF20002305F058FE5A
:100718000123A3720D4B186809F0CCF820684FF636
:10072800E07102F0DBFF2068094902F085FF60688C
:10073800084902F081FF04F00FF964200BF07AFAFF
:10074800054B00221A7010BD300C0020E426002052
:1007580013AC050875B10508712600202DE9F74F7F
:100768003A4D3B4E0024284603F0BDFE2246234660
:100778004FF6FF7137480094019402F073FF4FF66B
:10078800E0780427F0604146224623463248009725
:10079800019402F067FF23463060414622462F4805
:1007A8000097019402F05EFF2D4970602D4A2046A3
:1007B80003F050FC2C492D4A0746204603F04AFC1A
:1007C8002B492C4A8046204603F044FC2A492B4AF0
:1007D8008146204603F03EFC29492A4A83462046A2
:1007E80003F038FC21468246F2682B46204603F087
:1007F80049FD5A2132682B460A2003F043FD6E2139
:1008080072682B460A2003F03DFD9B213A462B4691
:10081800FA2003F037FD692142462B46FA2003F0FF
:1008280031FD37214A462B46FA2003F02BFDC8211B
:1008380052462B46AA2003F025FDF020C8215A462F
:100848002B4603B0BDE8F04F03F01CBDC8140020D0
:10085800300C002027AC05082FAC050842AC050871
:1008680051AC0508ED06000859AC050871060008EA
:1008780049AC0508F505000861AC0508DD05000868
:1008880068AC05080105000838B50C4C4FF6E07552
:100898002068294602F022FF2068094902F0CCFEB0
:1008A8006068294602F01AFF6068064902F0C4FE33
:1008B80004F052F8BDE8384004F04EB8300C00207F
:1008C8002FAC05086FAC050870B52DED028B9FEDB8
:1008D800248A88B00A26F0EE488A03E0B0EE608ADF
:1008E800F0EE418A0CF02DFE8DED000ACDED010AE7
:1008F8009DE8030004AB83E80300F0EE680AB0EE5D
:10090800480A9DED041ADDED051A8DED028ACDED3C
:10091800038A0CF0B7FBCDED010A8DED000A9DE8C6
:10092800030002AD85E80300013E6C46DDED020AD6
:100938009DED031AD2D19FED0B0A0CF0F9FD8DED58
:10094800000ACDED010A9DE8030085E80300DDED0E
:10095800030A9DED020A08B0BDEC028B70BD00BF12
:1009680000000000CDCCCC3D2DE9F74F564D574C3B
:10097800DFF86491DFF864814FF6E07005F004FC5D
:10098800286811F081FF064668680F4611F07CFF61
:100998003246CDE900013B464946204616F03AFE6C
:1009A800224600230520372105F028FD2869484FF5
:1009B800484E11F069FF824668698B4611F064FF62
:1009C8005246CDE900015B463946204616F022FE24
:1009D800224600230520692105F010FD286B11F03F
:1009E80053FF8246686B8B4611F04EFF5246CDE9A5
:1009F80000015B464146204616F00CFE0023052008
:100A08009B21224605F0FAFC31462A6C204616F056
:100A180001FE224600239B21A22005F0EFFC4FF4A3
:100A2800FC6005F0B1FBA86811F02EFF8246E8686B
:100A38008B4611F029FF5246CDE900015B46494635
:100A4800204616F0E7FD224605205021002305F038
:100A5800D5FCA86911F018FF8246E8698B4611F0A9
:100A680013FF5246CDE900015B463946204616F091
:100A7800D1FD224600230520822105F0BFFCA86B8A
:100A880011F002FF8246E86B8B4611F0FDFE5246DC
:100A9800CDE900015B464146204616F0BBFD002328
:100AA8000520B421224605F0A9FC31466A6C20468F
:100AB80016F0B0FDA220B4212246002303B0BDE801
:100AC800F04F05F09BBC00BF103B0020400C0020FD
:100AD80094AC0508B7AC050882AC0508A6AC0508B7
:100AE80008B5002005F07CFB0A4B1B780B2B0BD8B4
:100AF800DFE803F00A0A0A0A0A0A08060A0A0A0AC2
:100B0800054802E0054800E00548BDE8084001F056
:100B180014B900BF71260020241400204C100020B6
:100B2800A01800202DE9F14F2D4C204603F0DBFCE6
:100B380000202C492C4A03F08DFA2C492C4A814676
:100B4800002003F087FA2B492B4A0746002003F0C0
:100B580081FA2A492A4A0646002003F07BFA2949E5
:100B6800294A0546002003F075FA2849284A804694
:100B7800002003F06FFA2749274A8246002003F035
:100B880069FAD22183464A462346E62003F07AFBD7
:100B980028203A462346014603F074FB4621324694
:100BA8002346282003F06EFB64212A46234628208A
:100BB80003F068FB822142462346282003F062FBAB
:100BC800524623462820A02103F05CFB28205A46E1
:100BD800BE21234601B0BDE8F04F03F053BB00BF70
:100BE8001016002016AB0508E90A0008BCAC050879
:100BF80019160008C7AC0508F5150008D1AC05089A
:100C0800D1150008DCAC0508AD150008E7AC0508EF
:100C180089150008F1AC050865150008023810B5FB
:100C28000B2800F26E84DFE810F04F005300140127
:100C3800AF016702FD01120363036C04D3032704A9
:100C48000C0000204FF6E0710BF034FB19204FF434
:100C5800FC610BF02FFB4B204FF6E0710BF02AFBE9
:100C68007D204FF6E0710BF025FBAF204FF6E071C9
:100C78000BF020FB4FF6FF7005F086FAC821002321
:100C88005020A94A05F0BAFB4EF29C7005F07CFA98
:100C9800052001210023A54A05F0B0FB05201A21F3
:100CA8000023A34A05F0AAFB05204C210023A14AF2
:100CB80005F0A4FB05207E219F4A002305F09EFB3A
:100CC80005209E4AB02160E0BDE810400BF09CB9B9
:100CD80000204FF6E0710BF0EDFA64204FF6E0715A
:100CE8000BF0E8FAC8204FF6E0710BF0E3FA4FF684
:100CF800FF7005F049FA00237D20DC21904A05F0B9
:100D08007DFB4EF29C7005F03FFA8E4B1C78022C4E
:100D180040D0052C6CD0012C40F0F383B4204FF464
:100D2800F0610BF0C7FA05202146874A002305F039
:100D380065FB05205221854A002305F05FFBB6219B
:100D48007B4A0023052005F059FB4FF4F06005F0BD
:100D58001BFA40F2131021467B4A002305F04EFB94
:100D680040F213105221724A002305F047FB784ADB
:100D780040F21310B621002305F040FB4EF29C70A0
:100D880005F002FA0520A221724A0023BDE81040AE
:100D980005F034BBA0204FF4F0610BF08BFA05206E
:100DA80001216A4A002305F029FB052052216A4ADD
:100DB800002305F023FBB6215D4A0023052005F03A
:100DC8001DFB4FF4F06005F0DFF940F2131001212C
:100DD8005E4A002305F012FB40F213105221544AD8
:100DE800002305F00BFB40F21310B6215B4AC2E763
:100DF80064204FF4F0610BF05DFA20460121584A57
:100E0800002305F0FBFAB621494A0023204605F0E5
:100E1800F5FA4FF4F06005F0B7F940F2131001212C
:100E28004F4A002305F0EAFA40F213105221404AD3
:100E3800002305F0E3FAB62140F21310494A0023D3
:100E480005F0DCFA4EF29C7005F09EF9204652211E
:100E58009AE700204FF6E0710BF02CFA31204FF69C
:100E6800E0710BF027FA63204FF6E0710BF022FADD
:100E780095204FF6E0710BF01DFAC7204FF6E07190
:100E88000BF018FA4EF29C7005F07EF9052001214E
:100E98000023354A05F0B2FA052020210023334A01
:100EA80005F0ACFA052052210023314A05F0A6FAD4
:100EB8000520842100232F4A05F0A0FAB621052039
:100EC8001B4A002305F09AFA4FF4F06005F05CF92C
:100ED800012140F213100023234A05F08FFA40F253
:100EE80013102021244A002305F088FA40F2131039
:100EF80052210F4A002305F081FA40F21310842191
:100F08001E4A002305F07AFAB6211D4A40F2131052
:100F1800002305F073FA4FF6FF7005F035F97D20D0
:100F2800DC21184A31E700BFF6AC05080BAD05080F
:100F3800EDB205080FAD050813AD050817AD050896
:100F4800C7AC05081C0300201CAD050825AD050825
:100F58001BAD05084FAD050820AD050824AD0508F3
:100F68002AAD050829AD050843AD05082EAD0508CD
:100F78003EAD050833AD050838AD05083DAD05089B
:100F880042AD0508D1AC050800204FF6E0710BF022
:100F980091F927204FF6E0710BF08CF94F204FF6AE
:100FA800E0710BF087F977204FF6E0710BF082F9CA
:100FB8009F204FF6E0710BF07DF9C7204FF6E071E6
:100FC8000BF078F94EF29C7005F0DEF8052001214F
:100FD8000023AC4A05F012FA052016210023AA4A7C
:100FE80005F00CFA05203E210023A84A05F006FA70
:100FF800052066210023A64A05F000FA8E21002369
:101008000520A44A05F0FAF90520A34AB6210023D1
:1010180005F0F4F94FF6FF7005F0B6F87D20DC21F5
:101028009E4AB2E600204FF6E0710BF043F93120FA
:101038004FF6E0710BF03EF963204FF6E0710BF0CC
:1010480039F995204FF6E0710BF034F9C7204FF6C7
:10105800E0710BF02FF94EF29C7005F095F8052021
:10106800012100238E4A05F0C9F90520202100231B
:101078008C4A05F0C3F90520522100238A4A05F05D
:10108800BDF9052084210023884A05F0B7F9B62167
:1010980005207C4A002305F0B1F94FF4F06005F013
:1010A80073F8012140F213100023814A05F0A6F9D4
:1010B80040F2131020217F4A002305F09FF940F2E7
:1010C800131052216F4A002305F098F940F21310CB
:1010D8008421794A002305F091F9B621774A40F234
:1010E8001310002305F08AF94FF6FF7005F04CF84D
:1010F8007D20DC21724A48E6724B1C78022C32D0E3
:10110800052C5DD0012C40F08B8000204FF6E0715B
:101118000BF0D0F834204FF6E0710BF0CBF86420D8
:101128004FF6E0710BF0C6F84FF6E07198200BF01F
:10113800C1F84EF29C7005F027F805202146624A56
:10114800002305F05BF905202021604A002305F003
:1011580055F9052050215E4A002305F04FF9052076
:1011680084215C4A59E000204FF6E0710BF0A2F8A8
:1011780052204FF6E0710BF09DF890204FF6E07189
:101188000BF098F84FF6E071B4200BF093F84EF29C
:101198009C7004F0F9FF052001214F4A002305F057
:1011A8002DF905203E214A4A002305F027F905209C
:1011B8007C21484A002305F021F90520A0212BE0D5
:1011C80000204FF6E0710BF075F82E204FF6E07115
:1011D8000BF070F87F204FF6E0710BF06BF84FF6CC
:1011E800E071AD200BF066F84EF29C7004F0CCFF75
:1011F80020460121394A002305F000F92046322112
:10120800334A002305F0FAF820466B21314A0023BF
:1012180005F0F4F820469921314A002305F0EEF84C
:101228004FF4F06004F0B0FF2E4A00230520B621E9
:1012380005F0E4F84FF4FC61C8200BF03BF84FF6DA
:10124800FF7004F0A1FF8720DC21274A9DE50020DC
:101258004FF6E0710BF02EF863204FF4FC610BF0B1
:1012680029F84FF6E071C7200BF024F84FF6FF700D
:1012780004F08AFF002005F089F8A520D7211B4A31
:1012880083E500BFEDB2050846AD05080FAD0508BA
:101298004AAD050813AD05084EAD050852AD050861
:1012A8005EAD050862AD05087FAD050866AD0508A9
:1012B8006FAD05086BAD05086AAD05086EAD05088C
:1012C80073AD05081C0300202AAD05084BAD0508C1
:1012D8000CAD05088EAD05084FAD050810AD050825
:1012E8007EAD050804B40508F1AC05088DB1050804
:1012F800042005F04BF800204FF6E0710AF0DAFF01
:1013080031204FF6E0710AF0D5FF63204FF6E07107
:101318000AF0D0FF95204FF6E0710AF0CBFFC72006
:101328004FF6E0710AF0C6FF4EF29C7004F02CFFF5
:10133800052001210023734A05F060F805202021CB
:101348000023714A05F05AF80520522100236F4AFC
:1013580005F054F80520842100236D4A05F04EF865
:101368000520B6216B4A002305F048F84FF6E070D7
:1013780004F00AFF40F20B100121674A002305F030
:101388003DF840F22B102021644A002305F036F87E
:1013980040F223105221624A002305F02FF840F250
:1013A8001B1084215F4A002305F028F8B6215E4A05
:1013B800002340F2131005F021F84FF6FF7004F0F7
:1013C800E3FE002004F0E2FF6E20D221574A90E0AD
:1013D800042004F0DBFF00204FF6E0710AF06AFFFA
:1013E80027204FF6E0710AF065FF4F204FF6E071B5
:1013F8000AF060FF77204FF6E0710AF05BFF9F204C
:101408004FF6E0710AF056FFC7204FF6E0710AF078
:1014180051FF4EF29C7004F0B7FE05200121002315
:10142800434A04F0EBFF052016210023414A04F04B
:10143800E5FF05203E2100233F4A04F0DFFF052099
:1014480066213E4A002304F0D9FF05208E213C4A3C
:10145800002304F0D3FFB6213A4A0023052004F004
:10146800CDFF4FF6FF7004F08FFE002004F08EFFD2
:101478006420D221344A3CE0042004F087FF002095
:101488004FF6E0710AF016FF43204FF6E0710AF0BC
:1014980011FF85204FF6E0710AF00CFF4FF6E0715E
:1014A800C7200AF007FF4EF29C7004F06DFE05207D
:1014B8000121264A002304F0A1FF05204521244AE2
:1014C800002304F09BFF052087211E4A002304F017
:1014D80095FFB6211F4A0023052004F08FFF4FF621
:1014E800FF7004F051FE002004F050FF1A4A7D20DE
:1014F800D221002304F082FF0420BDE8104004F04C
:1015080045BF10BD82AD05088EAD05088DAD050837
:1015180090AD050894AD050899AD050843AD0508DB
:10152800A0AD0508A4AD0508A9AD0508AFAD05082F
:10153800B5AD05086BAD050870AD0508BAAD050871
:1015480018AD05084FAD0508BDAD0508C6AD0508C1
:101558002AAD0508EDB2050861B2050810B5064CBC
:1015680006480623237000F0E8FB2078FFF756FBB7
:10157800BDE810400DF038BEFC2C0020FC17002000
:1015880010B5064C06480723237000F0D6FB2078D8
:10159800FFF744FBBDE810400DF026BEFC2C0020F0
:1015A800FC17002010B5064C06480523237000F0F0
:1015B800C4FB2078FFF732FBBDE810400DF014BEE5
:1015C800FC2C0020FC17002010B5064C064804230C
:1015D800237000F0B2FB2078FFF720FBBDE8104035
:1015E8000DF002BEFC2C0020FC17002010B5064CA4
:1015F80006480323237000F0A0FB2078FFF70EFBBA
:10160800BDE810400DF0F0BDFC2C0020FC170020B8
:1016180010B5064C06480223237000F08EFB207894
:10162800FFF7FCFABDE810400DF0DEBDFC2C0020F1
:10163800FC17002038B5094C05464FF6E0712068C4
:1016480002F04CF820680DB1054900E0054901F0A9
:10165800F3FFBDE8384003F07FB900BF5C0C002001
:10166800CAAD0508DDAD0508194B10B51C78012C6D
:1016780005D006D3022C0CBF3024002402E000243D
:1016880000E0102404F1C80006F03CFB11490246B2
:10169800114815F0BFFF04F1CC0006F033FB0D49EB
:1016A80002460E4815F0B6FF04F1D00006F02AFBFA
:1016B800084902460A4815F0ADFF04F1D40006F0C7
:1016C80021FB044902460748BDE8104015F0A2BFB7
:1016D8001C0E0020B7AC0508B4260020D826002030
:1016E800EE2C0020A026002010B5E82006F00AFB0A
:1016F8000F4C024621460F4815F08CFFEC2006F0EF
:1017080001FB214602460C4815F084FFF02006F044
:10171800F9FA21460246094815F07CFFF42006F044
:10172800F1FA024606482146BDE8104015F072BF9E
:10173800B7AC0508B4260020D8260020EE2C0020DF
:10174800A02600200E4A012310B513700D4A00246C
:1017580014700D4A204613700AF0ACFB204604F0C2
:101768003FFD0A4B03221A700AF002FF0BF083FCBC
:10177800074B08481C70BDE8104000F0DEBA00BFF7
:10178800FC2C0020770D0020750D0020712600200C
:10179800E4380020DC12002038B50D4B0D4D002434
:1017A8001C700D4B28681C700C4B4FF6E0711C70B8
:1017B80001F094FF28680A4901F03EFF03F0CCF8D5
:1017C800204604F00DFD0748BDE8384000F0B5BAE2
:1017D800D40D00205C0C0020770D0020712600201D
:1017E80079B10508A018002007B50E4B0E481A78E5
:1017F800D2F1010238BF00221A700C4B05221A7070
:1018080000F09BFA022201238DE80C00B020602131
:10181800102232230DF086FE03B05DF804EB03F0CE
:101828009BB800BFD40D0020941100207126002021
:101838002E4A002310B513702D4A13700DF0CCFA00
:101848000446002842D02B4C4FF6E071206801F086
:1018580045FF2068284901F0EFFE60684FF6E07107
:1018680001F03CFF6068254901F0E6FEA0684FF6EC
:10187800E07101F033FFA068214901F0DDFE03F0BB
:101888006BF84FF47A600AF0D5F920684FF6E071EA
:1018980001F024FF20681B4901F0CEFE60684FF676
:1018A800E07101F01BFF6068164901F0C5FEA068F1
:1018B8004FF6E07101F012FFA068124901F0BCFE7A
:1018C80003F04AF8BDE8104003F046B80CF05CFF9E
:1018D800204604F085FC0C4B0C4804221A7000F0DA
:1018E8002CFABDE81040FEF7CFBF00BFD40D002092
:1018F800770D00205C0C0020F0AD050804AE05084B
:1019080014AE050878B1050871260020C814002017
:101918002DE9F04F6A4DDFF8F4916A4E85B0002446
:101928004FF6FF78284602F0DEFD41462246234660
:1019380065480094019401F095FE04270390414600
:101948002246234648460097019401F08BFE414603
:1019580030602246234648460097019401F082FEF3
:10196800414670602246234648460097019401F09C
:1019780079FEA8F50048B060414622462346534800
:101988000097019401F06EFE4146F060224623461E
:101998004F480097019401F065FE414630612246A8
:1019A80023464C480097019401F05CFE2346706181
:1019B8004146224648480097019401F053FE4749A2
:1019C800B061474A204602F045FB4649464A8046F0
:1019D800204602F03FFB4549454A8246204602F030
:1019E80039FB4449444A0746204602F033FB434941
:1019F800434A8146204602F02DFB4249424A83462B
:101A0800204602F027FB21468446039ACDF808C0F9
:101A18002B46204602F036FC052132682B46A020D2
:101A280002F030FC692172682B46782002F02AFC0B
:101A38007D21B2682B46782002F024FC2821F26828
:101A48002B46052002F01EFC4B2132692B4605204F
:101A580002F018FC052072696E212B4602F012FC78
:101A68009121B2692B46052002F00CFCD2213A469E
:101A78002B46052002F006FCD22142462B46562072
:101A880002F000FCD2214A462B46A62002F0FAFBBF
:101A9800D22152462B46F62002F0F4FBB4215A46D6
:101AA8002B46052002F0EEFBDDF808C05620B421D5
:101AB80062462B4605B0BDE8F04F02F0E3BB00BF1D
:101AC8006C1500205C0C002024AE05082EAE05081D
:101AD80035AE05083BAE050841AE050847AE05081A
:101AE8003918000816AB0508A117000850AE0508FC
:101AF800F117000859AE05084D17000862AE050831
:101B0800F11600086BAE05087116000875B10508D6
:101B1800654A00232DE9F04713700125634ADFF871
:101B2800BC811370A842014688F8005003D00228EF
:101B380040F0B3803EE04FF4747006F0CAF80AF043
:101B48003DFC5B4B5B4A1B68934209DD5A4A5B4983
:101B580012688A4207DD5A498A4204DC022210E0F0
:101B6800B3F5FA5F1ADB544A564912688A4201DC17
:101B7800002206E054498B4210DD544B9A420DDC9A
:101B88000122534B01201A7005F078FA0120FFF763
:101B980051FD4F4B1978012901D107E0FEE702D327
:101BA80002297AD102E04020002100E0402007F01D
:101BB8008FFA72E0C82006F0A5F80446CC2006F09B
:101BC800A1F80746D02006F09DF80646D42006F076
:101BD80099F881460AF0F2FB354B37491A68A24258
:101BE800184602DB0B68BB4213DD3A4B04601E60EB
:101BF800394B0F60C3F800900AF01CF9374B0122EB
:101C08001A70374A0520B4210023BDE8F04704F0D4
:101C1800F5BB944218D19F4216D12E4B1B689E42A9
:101C280012D12D4B1B6899450ED14FF4747029467B
:101C380088F8005006F04DF82A4B00221A602A4B0B
:101C48004FF07E521A6028E0244B02251D70294669
:101C58004FF4747006F03DF8154B1B6806EE906A59
:101C68001C1BF8EEE67A06EE904AB8EEE67A1D4BB3
:101C780087EE277A284683ED007A164B1B6806EE16
:101C8800903AB8EEE67A184BC7EE277AC3ED007A99
:101C980005F0F4F90020FFF7CDFC0AF02AFBBDE8B7
:101CA800F04702F059BE00BFD40D0020770D002088
:101CB800F02600205FE31600082D002080D1F008F0
:101CC8007F74D21A4FDA11001FA107007FD1F008E4
:101CD8001C0E0020E42C00209C260020C9010020B6
:101CE80074AE05086C260020AC26002008B500F06C
:101CF80055FFFEF781FA00F051F800F071F8FEF791
:101D08002DFDFEF781FBFEF70DFF01F077FBFFF7D6
:101D1800FFFDFEF7EFFA01F037F9FEF7B5FB01F02A
:101D280069FA00F073FB00F087FD00F091FE00F007
:101D380065FABDE8084000F033BB10B5044628B981
:101D48000F48104A104B552103F02EF80F4B186816
:101D5800844213D010B1C36900219847002004F0D1
:101D68003FFA002004F026FA4FF6FF7004F00CFA50
:101D7800E369204601219847044B1C6010BD00BF51
:101D880088AE0508042C0408A4AE0508780C0020C9
:101D98000048D2E7A01800200CF0DEBF10B5084CB0
:101DA800204602F0A0FB00200649074A02F052F93B
:101DB800D22102462346FA20BDE8104002F062BA5A
:101DC800600E0020C2AE0508A11D0008024B0348A2
:101DD80001221A70FFF7B1BF712600206C15002090
:101DE8002DE9F743374D384F384E0024284602F086
:101DF8007AFB2246234647F6FF7135480094019442
:101E080001F030FC4FF6FF788146414622462346D2
:101E180038460094019401F025FC41463060224682
:101E2800234638460094019401F01CFC414670603A
:101E38002246234638460094019401F013FC2346B9
:101E4800B0604146224638460094019401F00AFCED
:101E58002049F060204A204602F0FCF81F49204A39
:101E68000746204602F0F6F8214680464A462B46A9
:101E7800204602F007FA3C2132682B46192002F06E
:101E880001FA5A2172682B46192002F0FBF97821D1
:101E9800B2682B46192002F0F5F99621F2682B4614
:101EA800192002F0EFF9D2213A462B46EC2002F035
:101EB800E9F99C20D22142462B4603B0BDE8F04305
:101EC80002F0E0B9DC12002075B105087C0C002096
:101ED800B4AE0508C1AE0508D51D0008CAAE050890
:101EE800B120000870B5474E474C327847492DED70
:101EF800028B142592B005FB02420C320FA815F094
:101F080089FB33780E2B05FB03F504EB050332D868
:101F1800D3ED016A9B6807EE103A6359B8EEE68A7A
:101F280006EE903ADFED3A7AF8EEC78AB8EEE67A2E
:101F380088EE278AC8EEA78AC7EE277A17EE900A96
:101F480010F0A2FC02460B466846324915F062FBC7
:101F580018EE100A10F098FC02460B4605A82E4908
:101F680015F058FB18EE900A10F08EFC02460B464E
:101F78000AA82A4929E093ED017A9B6807EE903A6E
:101F8800635906EE903AF8EEE78AF8EEE67AB8EE8C
:101F9800C78A17EE900A10F077FC02460B4668468F
:101FA8001F4915F037FB18EE100A10F06DFC0246B9
:101FB8000B4605A81B4915F02DFB18EE900A10F0EA
:101FC80063FC0B46184902460AA8184C15F022FB78
:101FD8002068174901F030FB20680FA901F02CFB9D
:101FE8006068694601F028FBA06805A901F024FB98
:101FF800E0680AA901F020FB02F0AEFC12B0BDECCB
:10200800028B70BDEA26002000000020D3AE050830
:1020180000007A44DEAE0508EFAE050800AF0508FB
:1020280011AF050822AF050833AF05087C0C002066
:102038007EB1050808B5144B144A1B780D2B01D83E
:10204800012104E00E2B01D1022100E000211170D2
:10205800142253430E49C858CA184FF47A730D49CD
:1020680058430860516892684B430B490B600B4B0F
:102078001A6009F0DFFE0A4B0A4801221A70BDE80F
:102088000840FFF75ABE00BFEA2600201C0E0020B9
:1020980000000020F0260020082D0020E42C00205D
:1020A800712600206C150020C4E700BF4FF6FF70B2
:1020B80070474FF6FF7070471FB5002947D04FF2A1
:1020C800DE7004F08DF8002004F060F90F2004F0B1
:1020D8005BF81F4C1F4A412101230A2004F08EF9A6
:1020E800042004F053F9236828209621042B24DCCB
:1020F8000123194A04F082F903A90DF10E022068A0
:1021080004F002FC0F2004F03FF8BDF80C00BDF805
:102118000E1014380F242822002380B2009404F0F3
:1021280063F8BDF80E10BDF80C000094143989B29C
:102138002822012304F058F809E0084A012304F092
:102148005DF91E20A521064A012304F057F91FBD99
:102158008C0C002044AF050857AF050873AF05087D
:1021680089AF050837B51E4C2368042B05462BDCC0
:1021780001A80DF1060104F0C5FBBDF80630BDF855
:102188000420184904200DF033FC2368002B04DADE
:102198001548164A164B592105E0042B05DD12484F
:1021A800124A144B5A2102F0FFFD04EB8302BDF8DA
:1021B800041001339180BDF806102360052BD180EF
:1021C80008D1201D04F020FC00230B482360FFF7F2
:1021D800B4FD03E028460121FFF76EFF3EBD00BFB6
:1021E8008C0C0020A0AF0508E5AF0508162C0408E4
:1021F80007B005081EB00508B416002037B50B4C0B
:10220800204602F070F90A4B0A4900930025012084
:10221800094A0A4B019502F00EF829460246234660
:10222800284603B0BDE8304002F02CB880130020E7
:10223800C1200008B5200008BB2000086D21000857
:102248004FF6FF7070474FF6FF70704730B54FF686
:10225800E07087B003F0C4FF002004F097F80F2067
:1022680003F092FF00212C4A2C4C01230A2004F091
:10227800C5F8002003F088FF042004F087F80A203E
:102288001921274A012304F0B9F82521254A0123F9
:102298000A2004F0B3F81F2003F076FF01230A2078
:1022A8003721214A04F0AAF82378002B31D00123E2
:1022B8001E2096211D4A04F0A1F862881C4902A834
:1022C80015F0A8F901231E20A22102AA04F096F80D
:1022D800A288184902A815F09DF9AE2102AA012387
:1022E8001E2004F08BF80F2003F04EFF6088A188B1
:1022F800143880B20F2528220023009503F074FFBC
:10230800A18860880095143989B22822012303F036
:102318006BFF07B030BD00BF4CB00508A40C00200F
:102328005EB005087EB005089EB00508C1B0050876
:10233800D3B00508E0B0050801B187E7704713B5C9
:102348000DF1060101A804F091FA144B01221A704C
:102358005988BDF80420891A0E311C2919460AD853
:102368009C88BDF80600201A0E301C2803D89968EE
:102378000131996001E000238B60084B99680129BD
:1023880005DD00229A601A70FFF702FD05E05A8009
:10239800BDF806209A80FFF759FF1CBDA40C002049
:1023A80037B50B4C204602F09EF80A4B0A490093B9
:1023B80000250120094A0A4B019501F03CFF2946F6
:1023C80002462346284603B0BDE8304001F05ABF14
:1023D800B416002041230008492200084F220008B3
:1023E8004723000808B5064B00221A70054B1868E9
:1023F80014F0A6FD0448BDE80840FFF79EBC00BFE6
:1024080071260020D0360020A01800202DE9F04FBA
:10241800514D524E85B00024284602F064F82246F9
:10242800234647F6FF714E480094019401F01AF9CB
:102438004FF6FF77039039462246234649480094D1
:10244800019401F00FF93946306022462346464888
:102458000094019401F006F94FF0010870602246DB
:1024680023464FF6E0714148CDF80080019401F011
:10247800F9F82346B060394622463D48CDF8008039
:10248800019401F0EFF83B49F0603B4A204601F027
:10249800E1FD3A493A4A0746204601F0DBFD394951
:1024A800394A8046204601F0D5FD3849384A8146E8
:1024B800204601F0CFFD3749374A8246204601F0D1
:1024C800C9FD3649364A8346204601F0C3FD2146F8
:1024D8008446039ACDF808C02B46204601F0D2FE68
:1024E8003C2132682B46142001F0CCFE3C21726856
:1024F8002B46EC2001F0C6FEB421B2682B460F2013
:1025080001F0C0FED2213A462B46E62001F0BAFE81
:10251800642142462B46052001F0B4FE4A462B466C
:102528000520872101F0AEFE52462B460520D22118
:1025380001F0A8FED2215A462B46502001F0A2FEF7
:10254800DDF808C09B20D22162462B4605B0BDE8C5
:10255800F04F01F097BE00BF040F0020B00C002020
:10256800EDB00508F7B0050871AE050873B10508A8
:1025780075B10508C1AE0508ED23000849AC05088A
:10258800D525000859AC0508D526000800B105086E
:10259800DD27000808B105089927000810B10508CB
:1025A8005527000808B50CF007F94FF441400CF026
:1025B80047FE044B186807F07DF9034B09221A708F
:1025C80008BD00BFE42600207126002010B50C4C81
:1025D800FFF7E8FF0B4A0023B420052103F00EFFA4
:1025E800A0684FF6E07101F079F8A068064901F09B
:1025F80023F80CF0E1F8BDE8104002F0ADB900BFD7
:10260800B00C00207BB1050818B10508264B2DE950
:10261800F7431888C00014F08BFC054628B905203C
:10262800B421224A2B4603F0E9FE214BDFF87880DB
:102638001D6000240CF0C0F826461E4FDFF8889075
:1026480023E009F029FA3B68D9F8000045F8083C6E
:102658007B6845F8043C184B1B68C01807F02AF93A
:10266800164B186809F0E6FAB8F8000094FBF0F089
:1026780080B24FF4FC63009328210246322303F012
:102688000FFD04F59E7401360334B8F800300835A0
:10269800B342D6DA0A4B186807F00CF9094B09223D
:1026A8001A70BDE8FE8300BFDC3A002031B105088E
:1026B800D03600209C380020682600209C26002068
:1026C800E426002071260020D836002010B5094CD9
:1026D800FFF79CFFA0684FF6E07100F0FFFFA068CD
:1026E800054900F0A9FF0CF067F8BDE8104002F0BA
:1026F80033B900BFB00C00203FB1050810B5074C36
:102708004FF6E071A06800F0E9FFA068044900F006
:1027180093FFBDE8104002F01FB900BFB00C0020C5
:1027280059B1050810B5074C4FF6E071A06800F0E4
:10273800D5FFA068044900F07FFFBDE8104002F013
:102748000BB900BFB00C00206FB1050810B50C4CD8
:102758000B2323700B4B01221A70002003F00EF894
:102768000948FFF7EAFA2078FEF758FA074B0320E2
:1027780093ED000A0CF02FF8BDE81040D2E700BF37
:10278800FC2C00207A0D0020FC17002024030020D8
:1027980038B50C4D0C232B700B4B01241C700020FA
:1027A80002F0ECFF0948FFF7C8FA2878FEF736FA76
:1027B800074B204693ED000A0CF00DF8BDE83840B1
:1027C800B0E700BFFC2C00207A0D0020FC17002089
:1027D8002403002010B50C4C092323700B4B012255
:1027E8001A70002002F0CAFF0948FFF7A6FA2078FD
:1027F800FEF714FA074B022093ED000A0BF0EBFFEB
:10280800BDE810408EE700BFFC2C00207A0D0020A8
:10281800FC170020240300200CF064BB034A044882
:1028280000231370034A1370FFF787BAE4380020B7
:10283800A0180020712600202DE9F743384D394EA5
:10284800DFF8FC800024284601F04DFE224623468E
:1028580047F6FF7134480094019400F003FF4FF6E7
:10286800FF77814639462246234630480094019432
:1028780000F0F8FE39463060224623464046009470
:10288800019400F0EFFE3946706022462346404628
:102898000094019400F0E6FE2346B06039462246D3
:1028A80040460094019400F0DDFE2149F060214A81
:1028B800204601F0CFFB2049204A0746204601F078
:1028C800C9FB214680464A462B46204601F0DAFCE1
:1028D8003C2132682B46282001F0D4FC5A2172682A
:1028E8002B46192001F0CEFC7821B2682B4619201E
:1028F80001F0C8FC9621F2682B46192001F0C2FCB1
:10290800D2213A462B46EC2001F0BCFC0520D2210E
:1029180042462B4603B0BDE8F04301F0B3BC00BF0C
:10292800F0100020C00C002089B1050891B10508FD
:10293800C1AE0508252800089CB105082128000813
:1029480075B1050870B5064600200D46144603F01B
:102958001DFD4FF6FF7003F017FCF2B273208621BD
:10296800002303F02DFDEAB27320AE21002303F00B
:1029780027FDE2B27320D6210023BDE8704003F0A2
:102988001FBD08B5084B20201860084B1860084B7D
:1029980058221A600146FFF7D5FF0648064B186013
:1029A800BDE8084006F086BFD8010020D401002009
:1029B800D0010020C0E1E4009026002008B5094BB2
:1029C80020201860084B58211960084B02461860EF
:1029D800FFF7B8FF0648074B1860BDE8084006F047
:1029E80069BF00BFD8010020D4010020D001002019
:1029F800809698009026002008B5094B582018604A
:102A0800084B20211960084B0A461960FFF79AFF06
:102A18000648074B1860BDE8084006F04BBF00BFEA
:102A2800D8010020D4010020D0010020404B4C00E8
:102A380090260020034A044800231370034A1370A9
:102A4800FFF77BB9E4380020A01800207126002089
:102A58002DE9F74F444D454EDFF83C8100242846C8
:102A680001F041FD2246234647F6FF714048009495
:102A7800019400F0F7FD4FF6FF778346394622466A
:102A880023463C480094019400F0ECFD3946306040
:102A98002246234640460094019400F0E3FD39465F
:102AA80070602246234640460094019400F0DAFD07
:102AB8002346B0603946224640460094019400F00F
:102AC800D1FD2D49F0602D4A204601F0C3FA2C496A
:102AD8002C4A0746204601F0BDFA2B492B4A80466E
:102AE800204601F0B7FA2A492A4A8146204601F0D1
:102AF800B1FA214682465A462B46204601F0C2FBCF
:102B08003C2132682B46192001F0BCFB5A2172681F
:102B18002B46192001F0B6FB7821B2682B46192004
:102B280001F0B0FB9621F2682B46192001F0AAFBB0
:102B3800D2213A462B46EC2001F0A4FB82214246E2
:102B48002B46192001F09EFBAA214A462B46192044
:102B580001F098FB19205246D2212B4603B0BDE85C
:102B6800F04F01F08FBB00BF44190020D00C0020AB
:102B7800A4B10508B2B10508C1AE05083D2A000890
:102B8800BFB10508012A0008C8B10508C529000811
:102B9800D1B105088B29000875B1050810B50B4C93
:102BA800204601F0A0FC00200146224600F0BAFDB4
:102BB80000200749074A01F04DFAD2210246234670
:102BC8004FF48270BDE8104001F05CBBFC17002098
:102BD800DAB10508052C000870B5C9240AE0A8B2C6
:102BE80000223146013502F06BFCF02DF7D101349B
:102BF800EF2C02D00025A6B2F1E770BD10B51A4C33
:102C08002378092B08D1194A00231370184A137026
:102C1800FFF7E2FF174823E00A2B0ED1164B18687E
:102C280014F08EF9154A00231370114A1370144AD0
:102C38001370FFF7D1FF134812E0002002F09EFD49
:102C4800114A00231360114A13800D4B02221A7097
:102C58000F4B186806F02EFE22780E4B0E481A709D
:102C6800BDE81040FFF769B8712600207A0D0020F2
:102C7800770D0020040F0020D03600207B0D0020A7
:102C8800E4380020F0100020C40D0020D20D0020F0
:102C9800E42600208E26002038120020034B012253
:102CA8004FF4FC601A7003F06FBA00BF770D002074
:102CB800044B054800221A70044B0C221A70FFF7C7
:102CC8003CB800BF770D0020441900207126002071
:102CD800044B054800221A70044B0D221A70FFF7A6
:102CE8002CB800BF770D0020A80F00207126002007
:102CF80007B50A4A0023137004228DE80C00C62089
:102D08001022232356210CF00DFC054B05480A22FE
:102D18001A7003B05DF804EBFFF70FB8770D0020C9
:102D280071260020F010002007B50A4A002313700E
:102D380004228DE80C0097201022232356210CF042
:102D4800F1FB054B054809221A7003B05DF804EB46
:102D5800FEF7F3BF770D002071260020040F002036
:102D680007B50B4B00221A70082203238DE80C00CC
:102D78004920102223233D210CF0D4FB054B0648A3
:102D880001221A7003B05DF804EBFEF7D6BF00BF4E
:102D9800770D0020712600206C15002008B50D4B1A
:102DA800002018700C4B18700C4B18700C4B082234
:102DB8001A700C4B187003F013FA0B4B01211970A1
:102DC8004FF080400EF00FFE0848BDE80840FEF7BF
:102DD800B4BF00BF95260020D40D0020770D002039
:102DE80071260020FC2C0020E8360020600E002010
:102DF80070B51F4C1F4E20684FF6E075294600F04D
:102E08006DFC20681C4900F017FC6068294600F03A
:102E180065FC6068194900F00FFCA068294600F0BD
:102E28005DFCA068164900F007FC01F095FD4FF421
:102E38007A6008F0FFFE2068294600F04FFC206801
:102E4800314600F0F9FB6068294600F047FC6068ED
:102E5800314600F0F1FBA068294600F03FFCA0686D
:102E6800314600F0E9FBBDE8704001F075BD00BFD8
:102E7800E00C002078B10508F0AD050804AE05089F
:102E880014AE05080C4B10B500241C700B4B012226
:102E98001A70204609F00EF8204603F0A1F9084BF5
:102EA8000B221A7009F064FB0AF0E5F80548BDE842
:102EB8001040FEF742BF00BF770D0020FC2C002019
:102EC80071260020101600200F4A002310B5137039
:102ED8000E4A13700BF080FF044628B1FFF788FFF5
:102EE800BDE8104001F038BD03F07AF909F066FA40
:102EF800074B1C70074B07221A7009F059FA06484D
:102F0800BDE81040FEF719BFD40D0020770D002052
:102F1800FC2C00207126002024140020144A0023D1
:102F280010B51370134A1370134A13700BF054FF43
:102F380028B1FFF75DFFBDE8104001F00DBD03F0BB
:102F48004FF90E4B01241C7009F038FA06F020FDE9
:102F58000B4B06221A7009F02BFA4FF080402146DD
:102F68000EF041FD0748BDE81040FEF7E6BE00BF81
:102F780095260020D40D0020770D0020E83600208B
:102F8800712600204C1000202DE9F04F734DDFF81A
:102F980030928BB000244FF6FF78284601F0A3FA50
:102FA8004146224623466E480094019400F05AFB9D
:102FB8004FF6E076042703903146224623466948B7
:102FC8000097019400F04EFB3146049022462346B8
:102FD80065480097019400F045FB4146059022465C
:102FE800234648460097019400F03CFB5F4E41465B
:102FF80030602246234648460097019400F032FB91
:10300800234670604146224648460097019400F0E6
:1030180029FB5749B060574A204601F01BF856492A
:10302800564A8046204601F015F85549554A074644
:10303800204601F00FF85449544A8146204601F0D1
:1030480009F85349534A8246204601F003F8524989
:10305800524A8346204600F0FDFF5149514A8446B2
:103068002046CDF808C000F0F5FF4F4906904F4ABA
:10307800204600F0EFFF4E4907904E4A204600F0E8
:10308800E9FF4D4908904D4A204600F0E3FF2146EC
:103098000990039A2B46204601F0F4F82146049A39
:1030A8002B46C82001F0EEF80A21059A2B46C820C5
:1030B80001F0E8F8552132682B46782001F0E2F853
:1030C800692172682B46782001F0DCF8B2682B463B
:1030D8007D21782001F0D6F828213A462B46052094
:1030E80001F0D0F8962142462B46052001F0CAF897
:1030F800D2214A462B46052001F0C4F8D221524677
:103108002B46562001F0BEF8D2215A462B46A6205F
:1031180001F0B8F8DDF808C0B42162462B46052056
:1031280001F0B0F8B421069A2B46562001F0AAF80F
:10313800B421079A2B46A62001F0A4F8B421089AD6
:103148002B46F62001F09EF8099AF620D2212B464C
:103158000BB0BDE8F04F01F095B800BFA0180020F3
:10316800DFB10508E8B10508F5B10508E00C002055
:1031780000B20508D92C00080EB20508692D000810
:1031880016B205088D2E00081FB20508252F000865
:1031980028B20508D12E000831B20508A52D00086F
:1031A8003AB20508312D000843B20508F92C000889
:1031B8004CB20508B92C000854B20508A52C000823
:1031C80075B1050807B5032308228DE80C004920CE
:1031D800102223233D210CF0A5F9044B04480122B9
:1031E8001A7003B05DF804EBFEF7A7BD7126002046
:1031F8006C1500202DE9F743314E324F324D002433
:10320800304601F070F92246234647F6FF712F48F1
:103218000094019400F026FA4FF6FF788146414663
:103228002246234638460094019400F01BFA414692
:1032380028602246234638460094019400F012FA8A
:10324800414668602246234638460094019400F0BF
:1032580009FA2346A860414622463846009401945C
:1032680000F000FA1A49E8601A4A204600F0F2FE17
:10327800214607464A463346204601F003F83C21DA
:103288002A683346192000F0FDFF5A216A68334640
:10329800192000F0F7FF7821AA683346192000F0BA
:1032A800F1FF9621EA683346192000F0EBFFEC2085
:1032B800D2213A46334603B0BDE8F04300F0E2BFFE
:1032C8009411002075B10508EC0C00205CB20508CB
:1032D800C1AE0508CD3100081C4B1A781C4B10B53F
:1032E8001A7009F04BF91B4B1B4A00241C60022082
:1032F8002346CA2103F082F8204608F0DBFD174B6D
:103308001C80174B1C70174B1B78023B052B1CD8D5
:10331800DFE803F003070B13170FBDE81040FEF7B3
:1033280077B9BDE81040FEF761B9BDE81040FEF777
:103338004BB9BDE81040FEF723B9BDE81040FEF7D1
:1033480031B9BDE81040FEF709B910BD8E2600203E
:1033580071260020C40D002074B10508E436002051
:10336800E4380020FC2C002008B5084B186806F04B
:10337800A1FA002002F034FF09F0FAF8044B0548DE
:103388000B221A70BDE80840FEF7D7BCE4260020DF
:103398007126002010160020114B10B500241C7057
:1033A800104B186806F086FA204602F019FF0E4BFB
:1033B8001B780B2B0ED8DFE803F006060D0D0D0D5C
:1033C8000A080D0D0D06094802E0094800E0094801
:1033D800FEF7B3FC084B1C70BDE8104009F0C8B8F4
:1033E800FC2C0020E426002071260020A0180020D4
:1033F800241400204C100020E43800202DE9F0416E
:10340800144C204601F06FF800201349134A00F0CD
:1034180021FE1349134A0746002000F01BFE1249FB
:10342800124A0646002000F015FED22105463A460B
:103438002346E62000F026FF4B213246234664202F
:1034480000F020FF642069212A462346BDE8F041A8
:1034580000F018BF3812002016AB0508A133000889
:1034680064B205087133000870B20508E13200083B
:1034780008B508B143682BB90348044A044B9B219B
:1034880001F092FC586908BD7DB20508282C040893
:103498009FB2050808B5FFF7EBFF8068123080B2CD
:1034A80008BD08B5FFF7E4FF4068063080B208BDE4
:1034B8002DE9F84F04468846FFF7DAFF6689E58963
:1034C800074606F1030905F10F0AB8F1000F1FD0EE
:1034D8001F2002F059FE2046FFF7DCFF83462046F6
:1034E800FFF7DFFF294603465FFA8BF2F0B202F0DE
:1034F8008BFE042002F04AFF0B364FF6FF700335AF
:1035080002F042FEB0B2A9B23A68012302F076FF97
:103518003D69204641464A465346A847BDE8F88FCC
:1035280013B504460DF1060101A803F09FF92046E2
:10353800FFF79EFF6389BDF80410BDF80620C91A7D
:10354800E389D21A0339C3680F3A204698471CBD4D
:10355800F7B5044614200D4616461F4613F0E8FC3E
:10356800089BC7600361064B0649074A80E870005C
:1035780000930190054B002000F05DFEFEBD00BFEA
:10358800B9340008AB3400089D3400082935000818
:10359800704708B508B143682BB90448044A054B7D
:1035A800AD2101F001FC586908BD00BFBEB2050895
:1035B800402C04089FB20508F8B505460E46FFF7EB
:1035C800E8FF836B04461BB128463146984700E064
:1035D80018466F8994F83C30ED890EB9034310D032
:1035E800208E02F0D1FD608E02F0E4FD94F83500E3
:1035F80002F0CCFE94F8343038462946224602F0D0
:10360800FDFE002384F83C30F8BD08B5FFF7C1FF84
:1036180090F83500BDE8084002F0CDBE38B5FFF798
:10362800B8FF044614F07CF8054694F8350002F01B
:10363800BDFE684380B238BD38B50D46FFF7A9FF17
:1036480029462E22044614F09BF850B120462946FC
:103658002E2214F0E7F8002384F82E30012384F892
:103668003C3038BD2DE9F743074640200E46154645
:10367800984613F05DFC044628B91148114A124BCC
:103688004E2101F091FB114B114A12498DE81800A7
:103698000020114B00F0CFFD39468146FFF7CCFFE3
:1036A8009DF82830268684F835300B9B6586A36301
:1036B800002384F8348084F83C304846BDE8FE8313
:1036C800BEB20508582C0408DCB20508C13500084C
:1036D80013360008253600089935000810B50C4641
:1036E800FFF757FF0123048680F83C3010BD00BF68
:1036F8004FF4A0707047C82070477047074B1B787D
:10370800022B07B508D1064B1B78022B04D001A861
:103718000DF1060103F0AAF80EBD00BFE438002041
:10372800FC2C002073B50A4B06460D461446009340
:1037380000200849084A094B019000F07CFD294601
:1037480002462346304602B0BDE8704000F09ABDFC
:1037580003370008F9360008FF3600080537000867
:1037680013B502AB03E90600436843B1027C0124A8
:10377800082A9C7004D11B692146984700E01C4622
:1037880020461CBD30B500282BD0058B002425E031
:10379800036A1A7C012A05D15B681A888A421BD100
:1037A800187F30BD052A06D15B681A888A4213D172
:1037B80093F82C0030BD032A06D15B681A888A4228
:1037C8000AD193F8250030BD062A05D15B681A880E
:1037D8008A4201D1D87A30BD01340430AC42D7D303
:1037E800002030BD08B1817501207047F8B5044646
:1037F8000D46D0B1E175D0F898309847012D0DD11C
:103808002746002606E0F86900F10802436906CA5F
:1038180098470136238B04379E42F4D3D4F8983066
:103828002046294698470120F8BDF8BDF8B5054659
:10383800084617460E4613F073FF013FB84234BFDF
:1038480004463C463CB128463146224613F0EAFF7E
:1038580000232B55F8BD2C70F8BDF7B504460020A1
:103868000090019000296CD00E8B68E000F10803ED
:1038780051F823301D7C042D04D15D682D889542B4
:1038880047D0013000F1080351F823301D7C012D89
:1038980004D15D682D8895423BD0013000F10803C2
:1038A80051F823301D7C052D04D15D682D88954283
:1038B8002FD0013000F1080351F823301D7C032D6F
:1038C80004D15D682D88954223D0013000F10803AA
:1038D80051F823301D7C022D04D15D682D88954256
:1038E80017D0013000F1080351F823301D7C072D53
:1038F80004D15D682D8A95420BD0013000F1080390
:1039080051F823301D7C062D08D15D682D8895421D
:1039180003D103F10801204615E0013000F1080346
:1039280051F823502B7C082B09D16F683F889742A8
:1039380004D105F1080120461A4605E00130B042DD
:1039480094D320466946082213F0A2FD2046FEBD06
:10395800F8B505460F461646002830D04388032B95
:103968002FD0202013F0E4FA044600282BD040F88A
:103978000C5B39460C22FFF759FF1820E66113F05B
:10398800D7FA0646B8B102230374012363760F4BB6
:10399800446063600E4BA360002323766B8805EBBD
:1039A800830201339BB2012B50606B800CD16A6893
:1039B8005268137608E0204613F0C2FA04E006467F
:1039C80002E0002600E006463046F8BDA4AB040835
:1039D80042A8040837B5456802AB03E906003DB3C1
:1039E800037C0124042B85F8314022D1688E02F033
:1039F800CBFB95F8300002F0C9FC95F8343043B998
:103A0800BDF80200BDF80610AA1C234602F0F6FC19
:103A18000FE0012B03D1084840F2395104E0022B92
:103A280007D1054840F24151044A054B01F0BCF961
:103A38002C4620463EBD00BFEFB2050818770408A3
:103A4800EDB20508F8B504460F46164610B3838A4A
:103A58000A2B20D0202013F06BFA0546E8B1446009
:103A6800102200F108003946FFF7E0FE4FF6FF7319
:103A7800A08A2B801F236B8000232B76831D0130A7
:103A880080B20128EE6144F82350A08207D1A369CF
:103A98001876F8BDF8BD0020F8BD0120F8BD01205A
:103AA800F8BD2DE9F3471D464B1C984282460C464B
:103AB8001746BDF828600DDD95420BDC01320AF18E
:103AC80001035B1A521BC8B2D2B29BB229460096B8
:103AD80002F092FBAAF1020A3046C4EB0A0A02F08D
:103AE80053FB4FF000084FF001091FFA8AFA0BE068
:103AF800601C08EB050180B289B25246002300968B
:103B080002F072FB09F101097B1B08F101089945D4
:103B18001FFA88F8ECD3BDE8FC87F8B5C7B214469D
:103B280038461E460D4602F071FB621E92B23846B8
:103B3800294602F06BFB304602F026FB022606E01F
:103B4800A21B92B23846294602F060FB0136A64213
:103B5800F6D3F8BD73B504460E4600F11E001546AF
:103B6800009200233C2280B21E3E02F03DFBB1B21F
:103B780020463C220123009502F036FB7CBD73B53C
:103B880004460E460138154600920023032280B2EF
:103B9800013E02F029FBB1B2204603220123009521
:103BA80002F022FB7CBDF7B5089D2E7BEF7A1C4600
:103BB8003604AB7A06EB0726F618431A687B06EB41
:103BC80000602D1800200190121B08462146009520
:103BD80001F002FFFEBD30B5456885B004AB03E9CE
:103BE80006007DB101242C736D68BDF80800BDF88E
:103BF8000A109DF80C209DF80E300095FFF7D3FFB2
:103C0800204600E0284605B030BD2DE9F04385B0D8
:103C180004AB03E906004468BDF80860BDF80C7001
:103C2800002C41D0012384F8263094F825300BB9B4
:103C3800A26800E06268FFB2BDF80A109DF80E3075
:103C4800009230463A46FFF7AEFF04F10C08022016
:103C580002F09CFB404613F063FD054600B1451E8B
:103C68000F3F0024153E1FFA87F90DE002F098FB7C
:103C780002F09CFB04FB106189B248462022002315
:103C880002F0D6FB0134E4B2AC42EFD3002002F0DC
:103C98007BFAB8B2B1B24246012302F0C9FB002058
:103CA80002F074FB012000E0204605B0BDE8F08377
:103CB8002DE9F04385B004AB03E906004568BDF87B
:103CC8000860BDF80C70002D3CD001236B762B7E6C
:103CD800BDF80A10012B0CBF6A68AA689DF80E305F
:103CE8000092FFB23A463046FFF75DFF0C350220DE
:103CF80002F04CFB284613F013FD0E3F81460024CA
:103D0800163E1FFA87F80DE002F04AFB02F04EFB60
:103D180004FB106189B240462022002302F088FB90
:103D28000134E4B24C45EFD9002002F02DFAB8B2C4
:103D3800B1B22A46012302F07BFB002002F026FBE9
:103D4800012000E0284605B0BDE8F0832DE9F04FDA
:103D580085B00546DDF840900291484690460393A9
:103D680013F0DEFCDDF838A0DDF83CB00646294645
:103D780000242F4611E024B1B4420CBF5B465346E1
:103D880000E0039B01F10805ADB200932846029AB2
:103D98004346FFF708FF01342946B442EBDD002013
:103DA80002F0F2F9022002F0F1FA7D1D08F105088F
:103DB800A8B21FFA88F14A46012305B0BDE8F04FC2
:103DC80002F01CBB70B5406886B006AB03E906007C
:103DD80000282ED0012380F82D308668164BF21A61
:103DE800534243EB020390F82C205AB1002B134D99
:103DF800134B144A08BF1D46134B00F11C0418BF8F
:103E080013460AE0002B0D4D0D4B0E4A18BF1D46F8
:103E18000D4B00F10C0408BF1346BDF81200BDF8A5
:103E28001410BDF81620009601950294FFF78EFF36
:103E3800012006B070BD00BF88800408C47C040857
:103E48006A820408A67E04084C84040870B5446895
:103E580086B006AB03E9060004B301236377A668BE
:103E6800104B227FF11A4B4243EB01030AB10BB905
:103E780004E01BB966680C4D0C4B01E00C4D0D4B72
:103E8800BDF81200BDF81410BDF8162000960C34C9
:103E980001950294FFF75AFF012000E0204606B082
:103EA80070BD00BFD48B040810880408F289040888
:103EB800AA8D0408808F04082DE9F04385B004AB6F
:103EC80003E906004468BDF80860BDF80A90BDF82B
:103ED8000C50BDF80E80002C00F08C800123A374D8
:103EE8000220676802F052FA4FF6FF7002F062F99A
:103EF800002002F049F9EDB25FFA88F8A6F1160140
:103F080089B230462A4643460097FFF74CFE277A87
:103F1800002F2ED1A28A234600E00137974204D20F
:103F28009969097E04330029F7D002F039FA02F0C2
:103F38003DFAA9F116091FFA89F90E2101FB109122
:103F48004FF6FF7208F101085FFA88F389B2009210
:103F580048462A46FFF7A5FD022002F017FA1F205F
:103F680002F012F9A38A002B38D0103DE8B2303E97
:103F78002CE0E3685C68A28A2346013A002700E047
:103F88000137974204D29969097E04330029F7D092
:103F980002F006FA02F00AFA0E2101FB10914FF620
:103FA800FF7208F101085FFA88F389B20092484667
:103FB8002A46FFF776FD022002F0E8F91F2002F0FA
:103FC800E3F8A38A53B1103DE8B21A3E0637B1B2FE
:103FD80054F827200123083202F02AFA002002F0C0
:103FE800D5F94FF6FF7002F0E5F81F2002F0CCF883
:103FF800012000E0204605B0BDE8F0832DE9F0413E
:1040080005463620884614461F4612F091FF06469C
:10401800E0B120F8025B41462E22FFF707FCBDF80D
:10402800183086F8344073861820012386F83070DB
:1040380086F8313012F07CFF044618B1042346603C
:10404800037404E0304612F07BFF00E0044620468B
:10405800BDE8F081F8B5064624200F46154612F053
:1040680067FF0446D8B10F4B068083600E4B394674
:104078004360102200F10C00FFF7D8FB0126002353
:10408800182025622377667712F052FF054610B193
:104098004460067404E0204612F052FF00E0054632
:1040A8002846F8BDD48B04082E860408F8B50646C1
:1040B8002C200F46154612F03BFF0446E8B120F8C5
:1040C8000C6B39461922FFF7B1FB0D4BA562A360B3
:1040D8000C4B6360002384F825301820012384F8F2
:1040E800263012F025FF054618B1032344600374F7
:1040F80004E0204612F024FF00E005462846F8BDFB
:10410800E0A404087EA1040810B50446142012F0A7
:104118000FFF20B100234380014B0480036110BDD1
:104128005939000838B50546442012F001FF044605
:10413800C0B10E4B058243600D4B036001238374AD
:104148000023037283820B4B0364182012F0F0FEE5
:10415800054618B107234460037404E0204612F0B2
:10416800EFFE00E00546284638BD00BF749D0408F0
:104178006A9904084D3A00082DE9F04105463420B3
:10418800884614461F4612F0D3FE064620B3144B49
:1041980005808360134B41464360102200F10C00F8
:1041A800FFF744FB214606F11C001022FFF73EFBF7
:1041B800002386F82C3018200123376386F82D3029
:1041C80012F0B6FE044618B105234660037404E0F5
:1041D800304612F0B5FE00E004462046BDE8F08106
:1041E80088800408E27A04082DE9F0410446142086
:1041F8000D461646984612F09BFE0746B8B1069B38
:10420800048003610023C37201234560068180F89E
:104218000A800373182012F08BFE044618B1062397
:104228004760037404E0384612F08AFE00E0044652
:104238002046BDE8F0812DE9F041044618200D46DE
:104248001646984612F074FE0746B8B101238370EB
:10425800069B04800361079B45608660C0F80C805C
:104268004361182012F064FE044618B10823476021
:10427800037404E0384612F063FE00E0044620466A
:10428800BDE8F0812DE9F34198461B8B1D2B0546AF
:104298000C4617464FF0000000F2B480B5F5A07F39
:1042A8000090019000F2AE80F02900F2AB80127C01
:1042B800ADF80610511EADF80250072900F28A80A9
:1042C800DFE801F045595E04456A14767B684E4A7A
:1042D8007A611A8893F834303A80013BDBB2012BBB
:1042E8007FD8ADF80240ADF806507AE005F1160225
:1042F800ADF8002004F11602ADF8042002AE434ADE
:1043080016E903007A6107F1080282E8030003F165
:104318000802013348F82270A8F818307B681A8A16
:10432800187A3A8000286CD1FFF7FCFE38494368B8
:1043380059603849DF600126163D196002461E7231
:10434800A8B2E1B24346FFF79DFF30465AE0012A82
:104358000CBF314B314B78687B6130F80C3B3B80AC
:1043680013F0DEF9431CDB001A34ED18ADF80440F5
:10437800ADF8005035E07B68294A1B687A6102E095
:10438800284A7B687A611B8814353B80ADF8005059
:104398001434ADF8044024E07B68234A7A611A8813
:1043A8003A801A899B7AAD18ADF80050E418F0E706
:1043B8007E681E4B7B61338838463B80736898471C
:1043C800013D4519ADF80050B36838469847013C9F
:1043D8000419DEE71648174A174B40F21A3100F065
:1043E800E3FC02AA12E9030007F1080383E80300CB
:1043F800B8F8183003F10802013348F82270A8F819
:1044080018300120BDE8FC81DD390008C13E0008F4
:104418006095040856910408553E0008CD3D0008F3
:10442800B93C0008133C0008DF3B00086937000866
:10443800EFB2050828770408EDB20508F8B5164666
:10444800002834D01378002B2ED0028B002327E0CD
:10445800046A257C042D21D165682F888F421DD1DF
:1044680095F8313053B16F8E01F0B4FE04F10802B3
:1044780068866369204606CA98476F86A81C314635
:104488002E22FFF7D3F995F831307BB104F10802F9
:104498006369204606CA98470120F8BD01330430F5
:1044A8009342D5D30020F8BD1846F8BD0120F8BDC9
:1044B80070B5B8B1068B0446002310E0256A287C45
:1044C80004280AD16D682888884206D11046A91C9C
:1044D8002E22FFF7ABF9012070BD01330434B3423B
:1044E800ECD3002070BD38B5044620B3134BC3612C
:1044F800134BC0F89830134BC0F89C30124B002572
:104508007822C0F8A0308575C5750583294600F165
:10451800200012F0FFFFD4F898302046294698472B
:104528000A4A1388312B07D8094941F82340013337
:104538001380012038BD38BD284638BDF53700083E
:10454800ED3700088D37000863380008FC0C0020A0
:10455800E81900202DE9F0410446002800F0B38056
:10456800078B02460025A8E0136A1E7C042E00F083
:104578008780012E23D1586803888B4240F09B80A6
:1045880005F1080712F0DCFC54F827004FF000088A
:10459800C0F8048012F0D4FC228B531E9D4208D030
:1045A8000732238354F8221044F8271044F8228055
:1045B80002E044F8278025833046BDE8F081052EC7
:1045C8005ED0032E5CD0022E13D15B681868038876
:1045D8008B4270D14388013B9BB243800BB912F0E8
:1045E800AFFC05F1080654F82630586812F0A8FC0C
:1045F8004EE0072E21D15E68338A8B425BD10027BB
:1046080006E0BB1D013756F8230012F099FCFFB2F3
:10461800B38ABB42F5D80027B78205F1080654F8DB
:104628002630586812F08CFC54F8260033E044F821
:10463800267025830120BDE8F081062E1ED158681A
:1046480003888B4237D105F1080612F079FC54F83B
:1046580026000027476012F073FC228B531E9D42F0
:1046680009D00833013A54F82310228344F826105D
:1046780044F82370DEE744F826701AE0082E1AD1B1
:10468800586803888B4216D112F05AFC05F10806C7
:1046980054F826000027476012F052FC228B531E64
:1046A8009D42C4D0073254F8221044F8261044F82A
:1046B80022702383BEE701350432BD42FFF454AFB4
:1046C8000020BDE8F081BDE8F08170B504460028FF
:1046D8002AD0068B751E083600EB86061EE056F8B3
:1046E800043D1A7C042A13D0012A11D0052A0FD0C0
:1046F800032A0DD0022A02D15B681B6809E0072A49
:1047080002D15B68198A05E0062A01D0082A04D17B
:104718005B6819882046FFF71DFF013D681CDED144
:1047280000232383012070BD70BDF0B528B300239A
:10473800068B1A461EE0046A257C072D18D164688A
:10474800258A8D4214D1A78A002504EB83040DE045
:1047580004EB050C0435DCF818C09CF818C0BCF153
:10476800010F03F1010301D1D8B2F0BDBB42EFD371
:1047780001320430B242DED30020F0BD70B508B378
:10478800048B00231BE0026A157C072D15D15268A3
:10479800158A8D4211D10023958A11461C460120A5
:1047A80007E013B99669307601E08E6934760133F3
:1047B8000431AB42F5D3012070BD01330430A3426C
:1047C800E1D3002070BD2DE9F04128B30023078B09
:1047D8001A461EE0046A257C072D18D16468258ACC
:1047E8008D4214D1B4F814C0002504EB83040CE006
:1047F80066190435B66996F81880B8F1010F03D127
:1048080006F10800BDE8F08101336345F0D30132B9
:104818000430BA42DED30020BDE8F0812DE9F0472C
:1048280000282FD00023B0F818C01D4627E0046ADE
:10483800267C072E21D16468268A8E421DD1B4F8C1
:104848001480002604EB830915E009EB0604A76928
:104858003C7E012C0DD192F800A0BAF1000F08D0CF
:1048680007F1080011461022FEF7E0FF2046BDE8D8
:10487800F087013304364345E7D3013504306545F5
:10488800D5D30020BDE8F087F0B5B0B1068B002580
:1048980010E0046A277C062F0AD1646827888F42B3
:1048A80006D123819DF814306260A3720120F0BD07
:1048B80001350430B542ECD30020F0BD10B500211D
:1048C8000446FEF793FF20460121BDE81040FEF79D
:1048D8008DBF38B598B1048B024600230CE0106AEE
:1048E800058804328D4206D100F10802436906CAE0
:1048F8009847012038BD0133A342F0D3002038BDCA
:1049080010B50C460021FEF771FF20460121BDE8D5
:104918001040FEF76BBF13B502AC04E90C00BDF8FC
:104928000230834206D8BDF80030834234BF0020ED
:10493800012000E00020BDF806308B4206D8BDF803
:1049480004308B4234BF0021012100E000210028FF
:1049580018BF0846C0B21CBD38B5114B114A19889A
:10496800002319E052F8045FA87D012812D1002421
:104978000CE004F1080355F82300037C082B03D14D
:10498800436800211B6998470134A4B22B8BA342CA
:10499800EFD838BD01339BB28B42E3D138BD00BF9D
:1049A800FC0C0020E4190020704770B5094CA5786C
:1049B8007DB9094B1E78012E0BD163680133636002
:1049C8006268064B9A4204D9284601F0A1FCA670F9
:1049D800656070BDFC0C00209801002040420F006B
:1049E800054A9060134602E0996801399960916818
:1049F8000029F9D1704700BFFC0C0020F0B585B044
:104A080001F032FF002800F04981002502A80DF1CD
:104A18000A01ADF80850ADF80A5001F027FF03A8C5
:104A28000DF10E01ADF80C50ADF80E5001F06AFF13
:104A3800BDF80C10BDF808200091BDF80E10BDF8A7
:104A48000A3001912C46964D964908200AF0D0FF6D
:104A5800A878012803D101F05BFCAC7019E1924BF6
:104A68005B78012B40F01581AB78002B40F0118169
:104A78006B6029888D4A09E152F8046FB07D0128DE
:104A880040F002810025FAE005F10803BDF80800AE
:104A980056F82340BDF80A1004F108030CCBFFF7C1
:104AA8003AFF002800F0E980237C013B062B00F246
:104AB8009F80DFE803F00429159D1F9D4C00666860
:104AC800012304F10805337795E806006369204659
:104AD8009847002333772046636995E8060086E007
:104AE800636893F8252012F1FF3218BF012283F87A
:104AF800252077E0636893F82C2012F1FF3218BF65
:104B0800012283F82C206DE06268137E1568002B63
:104B18006ED16E882F462946184606E051F804EFF4
:104B2800DEF804E001338EF81800B342F6D301230F
:104B38001376002607E057F8040F00F108024369CE
:104B480006CA984701366B889E42F4D350E06568E0
:104B580020892E68A37B227B0096A0F1160189B2DA
:104B6800FFF721F81420FFF73BFF2B7AC3B9AF8A70
:104B780029461A461E4609E0886990F818E0067624
:104B8800BEF1010F08BF134604310132BA42F3D314
:104B980001220BB9AB6924E0053355F8233020E036
:104BA8006368DB685A680023908A154619461F46D1
:104BB80009E0AE6996F818E03776BEF1010F08BF34
:104BC8000B46043501318142F3D3411E8B4203D198
:104BD800053052F8203003E004D2073352F823306E
:104BE80001221A7604F1080206CA6369204698472A
:104BF800237C013B072B4CD8DFE803F00410074B5C
:104C08000A0D123A63681B6A34E063689B6A2DE0F8
:104C180063681B6B2AE063681B6927E0636824E00C
:104C280063681A7A7AB9988A1946013800E001321D
:104C3800824204D28C69247E0431002CF7D00632DB
:104C480053F8223011E0DB685A68908A114601381F
:104C5800002300E00133834204D28C69247E0431AE
:104C6800002CF7D0063352F82330DB69984710E060
:104C78006368DB68204698470BE00135ADB2338B9B
:104C8800AB423FF601AF04E001339BB28B427FF4A5
:104C9800F3AE01F02FFE0F20FFF7A2FE05B0F0BD26
:104CA800FC0C002015B3050898010020E419002029
:104CB800034B9A6812B19A68013A9A60704700BF2C
:104CC800FC0C00202DE9F3470120DFF8D080DFF845
:104CD800D09001460CF026FA012400254FF4807686
:104CE80002274046694600968DF804708DF8054005
:104CF8008DF806508DF807400BF06CFE40460821F1
:104D080022460BF0E7FE244BDFF898801A6844F23D
:104D1800A243B2FBF3FA0AF1FF3A204621461FFAF2
:104D28008AFA0CF02FFAC8F804A048464146A8F8B9
:104D38000050A8F80250A8F8085088F80A500CF05B
:104D4800BDFD7023A8F80C300423A8F810300AF130
:104D5800FF3A6323642203FB0AF3B3FBF2F39BB22B
:104D6800C8F8143008F10C014846A8F80E40A8F815
:104D78001870A8F81A50A8F81C60A8F81E500CF073
:104D8800BBFE484621460CF02EFE484621460DF053
:104D980034F9BDE8FC8700BFE401002000000240B0
:104DA800000001400C0D002083B50E46074615494A
:104DB80010201C4615460AF01BFE102012490AF066
:104DC80017FE102011490AF013FE10200E490AF0B0
:104DD8000FFE002310200E4901930AF009FE334606
:104DE80010200C493A460AF003FE10200A492A46C8
:104DF8000AF0FEFD1020094922460AF0F9FD019B40
:104E08000133E7E74FB3050854B3050874B3050841
:104E180084B3050894B30508A9B30508BAB305080F
:104E280008B5164B1A6A01321A621A6A012A1A461A
:104E380003D0134840F21E210FE05862194602E0E1
:104E48004B6A013B4B62506A0C4B0028F8D11A6A36
:104E5800012A06D00A4840F229210A4A0A4BFFF7DC
:104E6800A3FF1A6A013A1A621B6A2BB10448054A61
:104E7800064B40F22B21F2E708BD00BF0C0D0020C5
:104E8800CBB3050806AF0408F5B3050806B4050852
:104E980010B5084C0221002220460BF010FE44F603
:104EA800FF70FFF7BDFF204602210122BDE8104038
:104EB8000BF005BE000402400C4B0D491A6844F281
:104EC800A2436428B2FBF3F3D4BF20EAE070642065
:104ED800013B9BB24B60013B58436422B0FBF2F0AC
:104EE80080B2486103480C310CF089BDE401002010
:104EF8000C0D00200000014010B5134B93F828203A
:104F08002AB11248124A134B40F209310EE001222D
:104F180083F8282066234FF0C042013BDBB21080A3
:104F280033B90A480A4A0C4B40F21331FFF73CFFE9
:104F38001488A4B28442F0D1084B1980024B002295
:104F480083F8282010BD00BF0C0D0020CBB3050846
:104F580010AF040817B40508EDB205080000026098
:104F680010B5FFF7AFFE6420FFF7A6FF2121072049
:104F7800FFF7C2FF3220FFF753FF01210020FFF7A0
:104F8800BBFF3220FFF74CFF23210720FFF7B4FFB8
:104F98003220FFF745FF00211020FFF7ADFF41F257
:104FA8008830FFF73DFF33210720FFF7A5FF3220A8
:104FB800FFF736FF112046F63001FFF79DFF32203C
:104FC800FFF72EFF4FF4C0610220FFF795FF322054
:104FD800FFF726FF122046F6EB41FFF78DFF322040
:104FE800FFF71EFF03204AF6A401FFF785FF3220D2
:104FF800FFF716FF00210C20FFF77EFF3220FFF796
:105008000FFF0D2040F60C01FFF776FF3220FFF767
:1050180007FF0E204FF42C51FFF76EFF3220FFF7E9
:10502800FFFEB0211E20FFF767FF3220FFF7F8FED2
:10503800012042F63F31FFF75FFF3220FFF7F0FE15
:1050480005200021FFF758FF3220FFF7E9FE002175
:105058000620FFF751FF3220FFF7E2FE16204EF63A
:105068001C71FFF749FF3220FFF7DAFE172040F2E4
:105078000311FFF741FF3220FFF7D2FE00210B207A
:10508800FFF73AFF3220FFF7CBFE00210F20FFF792
:1050980033FF3220FFF7C4FE41200021FFF72CFF29
:1050A8003220FFF7BDFE42200021FFF725FF322006
:1050B800FFF7B6FE00214820FFF71EFF40F23F141D
:1050C8003220FFF7ADFE21464920FFF715FF3220B9
:1050D800FFF7A6FE00214A20FFF70EFF3220FFF758
:1050E8009FFE00214B20FFF707FF3220FFF798FEB5
:1050F80044204FF46F41FFF7FFFE3220FFF790FE88
:1051080000214520FFF7F8FE3220FFF789FE2146EF
:105118004620FFF7F1FE3220FFF782FE302040F2F2
:105128000771FFF7E9FE3220FFF77AFE31204FF4CE
:105138000171FFF7E1FE3220FFF772FE32204FF4D3
:105148000171FFF7D9FE40F202543220FFF768FEE2
:1051580021463320FFF7D0FE3220FFF761FE3420CE
:1051680040F20751FFF7C8FE3220FFF759FE3520FD
:105178004FF40171FFF7C0FE3220FFF751FE3620D1
:105188004FF40171FFF7B8FE3220FFF749FE2146C0
:105198003720FFF7B1FEA4F500743220FFF740FE78
:1051A80021463A20FFF7A8FE3220FFF739FE2F20CC
:1051B80041F2BE21FFF7A0FE3220FFF731FE214663
:1051C8003B20FFF799FE3220FFF72AFE002123201B
:1051D800FFF792FE3220FFF723FE00212420FFF77D
:1051E8008BFE3220FFF71CFE25204FF40041FFF70D
:1051F80083FE3220FFF714FE00214F20FFF77CFECC
:105208003220FFF70DFE4E200021FFF775FE3220F9
:10521800BDE8104004E608B5124B93F829202AB1DE
:105228001148124A124B40F223310FE0012283F851
:105238002920222166234FF0C042013BDBB21180B6
:1052480033B90948094A0B4B4FF44F71FFF7ACFDCE
:10525800108880B22228F0D1024B002283F829203E
:1052680008BD00BF0C0D0020CBB305081DAF040816
:1052780017B40508EDB2050810B51B4B032826D84E
:10528800DFE800F0021A080E1C8841F2280246F6F0
:1052980028000AE01C8841F2080246F6080004E0EB
:1052A8001C8841F2300246F6300049F241318C4206
:1052B80014BF014611460BE0188846F6200249F251
:1052C8004131884214BF11464FF4815100E000215A
:1052D8001A8848F689139A4202D11120FFF70CFE6A
:1052E800BDE8104097E700BF9A010020014B1880E5
:1052F8000A2095E5000002604FF0C043188003F5CE
:1053080000331A881A88188880B270474FF0C04353
:1053180022221A8003F5003382B01A8892B2ADF8BF
:1053280006201B889BB2ADF80630BDF8060080B297
:1053380002B07047072040F27311DDE50720002115
:10534800DAE582B0044BADF80600BDF8062092B24B
:105358005A8502B0704700BF0C0D002082B0044B84
:10536800ADF80600BDF8062092B25A8002B0704728
:105378009A010020014B80B218807047000002603B
:105388004FF0C04380B218807047024B80B218803B
:10539800704700BF000002604FF0C04380B2188021
:1053A8007047024B80B21880704700BF000002604F
:1053B80082B0044B0190019ADA62DA6A002AFCD1C1
:1053C80002B070470C0D002070B54FF0C0452A247C
:1053D8002C800A4C060AC0B226802080100AD2B25D
:1053E800208022802B222A800A0A2280C9B21A0A27
:1053F800DBB221802280238070BD00BF00000260E4
:1054080010B50B4614460246FFF7DEFF4FF0C043C7
:105418002C22A0B21A80BDE8104067E70B4B1A880F
:1054280048F689139A4210B504460AD1C1F1EF0132
:105438004E2089B2FFF760FD4F202146BDE810409D
:105448005AE502460B46BDE81040BDE79A01002028
:1054580008B5FFF7E3FF0F4B1B78012B4FF0C04255
:105468000D4B0FD12E2111801A881A881B8892B2F1
:1054780002F0FC0002F4784242EAC000C3F3C423FD
:10548800184308BD222111801A881A88188880B20A
:1054980008BD00BFB81A00200000026070B5074DB3
:1054A8000646012421463046FFF7D2FF0134A4B254
:1054B800C82C25F8020FF5D170BD00BFE6380020D2
:1054C80010B5084B1B78012B144602D1BDE81040DB
:1054D80096E7FFF7A3FFFFF79EFE2046BDE81040C2
:1054E80004E700BFB81A002070B5074D064601242E
:1054F8002146013435F8022F3046A4B2FFF7E0FF09
:10550800C82CF5D170BD00BFE638002070B505463F
:105518000E46FFF7C3FF01242146013428463246D0
:10552800A4B2FFF7CDFFC82CF6D170BD2DE9F84F16
:105538000C4693460546C718DFF82CA00AE0BAF8CF
:105548002A20B1B292B24046FFF7BAFF01364E4563
:10555800F5DB0135BD4205DA264604EB0B091FFAD7
:1055680085F8F4E7BDE8F88F0C0D00202DE9F0412F
:1055780004460D461646BDF81880032B39D8DFE8D7
:1055880003F00B351927381980B2294642460137EE
:10559800FFF796FFBFB200E00027B742F3D1BDE89E
:1055A800F081E01B80B2294642460137FFF788FFA9
:1055B800BFB200E00027B742F3D1BDE8F081E91B94
:1055C80089B2204642460137FFF77AFFBFB200E0B2
:1055D8000027B742F3D1BDE8F081791989B2204696
:1055E80042460137FFF76CFFBFB200E00027B74221
:1055F800F3D1BDE8F08170B5194B1A4A598E92F96A
:10560800004064180025A4B28AB0AC4208BF012447
:10561800C62C28BFC62415700F264FF6FF721E86AB
:105628005C865A8519202B46009221460A22FFF7EC
:105638009DFF21463046FFF70BFF224603460A49E5
:1056480002A811F0E7FF02AA06A8084911F0E2FF34
:105658003220D22106AA2B4600F0D0FE0AB070BD37
:105668000C0D0020251B00202CB4050834B40508B7
:105678002DE9F341BDF820500C4690461F461A46C6
:10568800002306460095FFF771FF611E414430462E
:105698003A46002389B20095FFF768FF3046214655
:1056A800424601230095013EFFF760FFBF19B8B2DB
:1056B800214642460123089502B0BDE8F04155E76E
:1056C80070B50D461C490446088848F68911884279
:1056D8002CD1C5F1F001661E9E198A1AC5F1EF0397
:1056E80092B29BB29A422CBF11461946EF2928BFA5
:1056F800EF219A4238BF134643EA0121B6B289B274
:105708004420FFF7F9FBA64234BF31462146452025
:10571800FFF7F2FBA64238BF264640F23F139E42EF
:1057280034BF314619464620FFF7E6FB2046294696
:10573800BDE8704072E600BF9A01002000200146D3
:10574800F0224FF4A073BBE770B54FF0C0452A2490
:105758002C80094C060A26802080080A2080218097
:105768002B212980110A218022801A0A2280238075
:105778002C232B8070BD00BF0000026070B5114B58
:105788001B78012B044607D1002040F23F11024646
:10579800EF23FFF7D9FF04E0FFF7D0FF0020FFF762
:1057A8006BFDF02509E0013E2046B6B2FFF79EFDED
:1057B800002EF8D1013DADB215B14FF4A076F2E755
:1057C80070BD00BFB81A00202DE9F04F1C463E4BB3
:1057D80087B01B78039183469DF844101098059173
:1057E800012B039B049092461FFA8BF09AB208D1C2
:1057F800411E531E0919534489B29BB2FFF7A4FFF7
:1058080009E01FFA8AF51146A3B22A46FFF758FFA6
:105818000020FFF731FD0027DDF80C803E4640F2FE
:105828003F1CA14639E0BBF1000F2EDB65452CDC9F
:105838000398002829DBB8F1EF0F26DC220702D1F4
:10584800002CC8BF013621492140002903DA01395B
:1058580061F00F010131059A0AB1C1F10F010498F5
:1058680030F8162003FA01F10A4012B26AB1184959
:105878004A8D029392B2A8B21FFA88F1CDF804C0FB
:10588800FFF71EFEDDF804C0029B013401354C45CC
:10589800C9DB0136013708F10108574503DA5D46CF
:1058A80000240123F3E7084B1B78012B08D10020C3
:1058B80040F23F110246EF2307B0BDE8F04F43E73F
:1058C80007B0BDE8F04F39E7B81A00200F00008094
:1058D8000C0D00202DE9F74F1F463B4BDDF83080BB
:1058E8001B7816469DF83420012B044601920D467C
:1058F80080B28AB208D1411E531EC9199B1989B2B8
:105908009BB2FFF721FF09E01FFA86FE1146BBB2E2
:105918007246FFF7D5FE0020FFF7AEFC4FF0000BF4
:10592800DA463DE0002C30DB09EB040340F23F127D
:1059380093422ADC002D28DB0BEB0503EF2B24DC3C
:1059480019F00F0F04D1B9F1000FC8BF0AF1010A0D
:105958001E4B09EA0303002B03DA013B63F00F0334
:105968000133019A0AB1C3F10F03012202FA03F3CA
:1059780038F81A2013401BB213B1154B588D01E0AB
:10598800144A508880B2FFF7B1FC09F1010901E01F
:105998004FF00009B945C5DB0AF1010A0BF1010B0B
:1059A800B345F5DB084B1B78012B08D1002040F2EA
:1059B8003F110246EF2303B0BDE8F04FC4E603B041
:1059C800BDE8F04FBAE600BFB81A00200F0000800B
:1059D8000C0D00209A0100202DE9F0411C4F069C77
:1059E8003F789DF81C60012F02FB03F580B28FB24F
:1059F80009D1411ECB1899B27B1E9A1893B23A4628
:105A0800FFF7A2FE07E092B29BB23946FFF758FEB5
:105A18000020FFF731FC002709E034F8020B1EB123
:105A2800030A43EA002080B2FFF760FC0137AF4267
:105A3800F3DB074B1B78012B07D1002040F23F1105
:105A48000246EF23BDE8F0417EE6BDE8F04175E689
:105A5800B81A00202DE9F0431F2093B0FFF78EFEFF
:105A68004FF47840FFF78AFE4FF6E0754FF4FC607C
:105A7800FFF784FE2846FFF781FE0020514CFFF710
:105A88007DFE00204FF6FF79014664220346A4F804
:105A98002A90CDF80090FFF769FD00200A216422C2
:105AA8000346CDF80090FFF761FD0020014664220F
:105AB80001234FF4784765850095FFF757FD772058
:105AC800EF21C82200234FF4FC6667850097FFF793
:105AD8004DFDBD213222012340F23F10668500961C
:105AE800FFF744FDA0203222002378216785009724
:105AF800FFF73CFDA0207821322201234FF01F0838
:105B080066850096FFF732FDA02078213222022315
:105B1800A4F82A80CDF80080FFF728FDA02078217E
:105B28003222032365850095FFF720FD264B274980
:105B3800A3F8028002AD3C22284611F0A9FCEB2014
:105B4800C3210522302300950025A4F82A90019549
:105B5800FFF7C0FE32210A2096220B466785009780
:105B6800FFF786FD32213C2096220B46668500967B
:105B7800FFF77EFD32210B4696226E20A4F82A807C
:105B8800CDF80080FFF774FDFFF7D8FBFFF7D2FBD5
:105B98003220FFF791F92846FFF78EF96420FFF7C6
:105BA8008BF90B4B03F110028DE8240028465A6844
:105BB8001B682946FFF710FF1195119B01331193BC
:105BC800FBE700BF0C0D00209A01002032AF04084B
:105BD800F0D301082DE9F14FFFF774F84FF0C045F5
:105BE8006420FFF769F90127FFF752F94FF02809F8
:105BF8006D48FFF715F92F800520A5F8009003F0F0
:105C080059FACF232B80694B002683221E801A80E5
:105C180030221A80ED222A804FF064080322A3F86C
:105C280000801A8012221A8081221A80E8222A8093
:105C380085221A8079221F801A80CB222A80392255
:105C48001A804FF0340C02242C21F72219801E8070
:105C5800A3F800C01C802A8020221A80EA222A8009
:105C6800C0221E80C1211E802A8026221A802980F7
:105C780011211980C5212980352119803E211980DB
:105C8800C7212980BE211980362129803A20552133
:105C9800A3F8009028801980B12129804FF0100BBB
:105CA800F2211E80A3F800B02980082119802A80DB
:105CB800E0221F804FF01F092A801A22A3F80090C3
:105CC8004FF0180A1A800F210A22A3F800A01A80A0
:105CD80019800621198045211980872119803221D0
:105CE800198007211A804FF0E10E19801C800524C5
:105CF80019801C801E80A5F800E04FF0250E1E803C
:105D0800A3F800E04FF0270EA3F800E01C80A3F8EA
:105D180000B04FF0090BA3F800B04FF0780B1880D3
:105D2800A3F800B04FF04D0BA3F800B01C800D2471
:105D3800A3F800A01C8038241C8018802A20A3F80F
:105D48000090EF2428802B201E801E801E801C803F
:105D580028803F201E801E801F801880B720A5F84D
:105D680000C028801980B62129801A8082221A80D2
:105D78001122A3F800E040461E8029272A8003F05C
:105D880099F940462F8003F095F90948FFF748F83C
:105D98002C232F8030462B8040F23F113246234679
:105DA80001B0BDE8F04FCFE4400D030000000260F1
:105DB80040420F002DE9F041022098B00121002453
:105DC8000BF0B0F9012502268048169616A98DF821
:105DD8005D408DF85E408DF85F408DF85C500AF0AC
:105DE800F9FD182029460BF09DF9284629460BF0A5
:105DF800B1F921460C2276480AF06CFE0C22744850
:105E080029460AF067FE04210C2271480AF062FE56
:105E180005210C226E480AF05DFE07210C226C4811
:105E28000AF058FE08210C2269480AF053FE09219D
:105E38000C2267480AF04EFE0A2165480C220AF037
:105E480049FE0B2162480C220AF044FE0E210C2266
:105E58005F480AF03FFE0F210C225D480AF03AFE27
:105E680007210C225B480AF035FE08210C2259480C
:105E78000AF030FE09210C2256480AF02BFE0A21AE
:105E88000C2254480AF026FE0B210C2251480AF035
:105E980021FE0C210A464F480AF01CFE0D210C2257
:105EA8004C480AF017FE0E210C224A480AF012FE4E
:105EB8000C2248480F210AF00DFE4CF6B3734448F3
:105EC800169316A98DF85C608DF85E408DF85F40DA
:105ED8008DF85D500AF07EFD16A94FF680733D4897
:105EE80016938DF85C608DF85E408DF85F408DF8F4
:105EF8005D500AF06FFD40F6B830FEF791FFFEF7EF
:105F0800C7FF40F6B830FEF78BFF0F2311934FF40D
:105F1800805310270DF13C08099368464FF400237D
:105F28001094129414941594009401940294039775
:105F380004940694079408940A9405940B940C937B
:105F4800CDF834800F9513950AF0BDFA05236846FD
:105F580011930F961094129414941594CDF83880D8
:105F680013950AF0B0FA294620460AF02CFB40F6B1
:105F7800B830FEF755FF2046FFF7BEF9044616492C
:105F8800164E3846224609F033FD41F289239C42D9
:105F980048F68918124F01D044450ED1FEF7E0FFAC
:105FA80000233B70A6F8008010200E4948F689129D
:105FB80041F2892309F01CFD05E0FFF70BFE49F2C9
:105FC80041333D70338018B0BDE8F08100040240D1
:105FD800000C02400010024039B405089A01002064
:105FE800B81A002050B405084FF0C04336221A8072
:105FF80003F50033012814BF682048201880704733
:1060080070B5244B01228CB01A7000240AE0A9B2A2
:106018001F2230460135FFF753FA642DF7D10134BA
:10602800642C02D00025A6B2F1E7322001460246D0
:106038000346FFF7C9F94FF0C0432E221A8003F533
:10604800003300201E881C881D88A4B2B6B200F058
:106058009BF8ADB2234610490095324603A811F0CB
:10606800D9FA00230A20C82103AA00F0C7F904F0CE
:10607800FC0204F4784444EAC20242EAD522074901
:1060880003A811F0C7FA0A20DC2103AA002300F0B4
:10609800B5F9FEE7B81A00208FB40508A7B40508BB
:1060A8002DE9F04F40F23F19484534BF04464C46AD
:1060B800EF2B34BF98464FF0EF084A4538BF91465A
:1060C800EF2934BF0D46EF25C4EB090AC5EB0807D5
:1060D80085B0BAF1000FB8BFCAF1000A002FB8BFE7
:1060E8007F424FF6FF734C452CBF1A4601221FFA18
:1060F8008AFA454538BF0123BFB202930FFA8AF6E0
:106108003BB29E42BDF838B0019202DDC6F34F069D
:1061180007E0022693FBF6F67642B6B201E01E4689
:1061280003E00FFA8AF35B420393144A1378022BB5
:10613800204629465A4602D1FDF721FD01E0FFF726
:10614800BFF94C4501D1454514D0039A33B2934267
:1061580005DD019AF31BA4189BB2A4B200E03346F4
:1061680036B23AB29642DADA029A5344AD189BB282
:10617800ADB2D4E705B0BDE8F08F00BFFC2C00201D
:1061880000487047C01A002082B0064BADF80600E0
:10619800BDF8062092B21A80188880B202B0FFF7C4
:1061A800D0B800BFBC1A0020014B188880B27047D5
:1061B800BC1A002082B0064BADF80600BDF80620D8
:1061C80092B21A80188880B202B0FFF7C7B800BF31
:1061D800BE1A0020014B188880B27047BE1A0020F2
:1061E800FFF7CCBAFFF76CBA10B5BDF808400294B7
:1061F800BDE81040FFF7BAB910B5BDF808400294E1
:10620800BDE81040FFF734BAFFF790B92DE9F04F19
:106218004FEA420800253D4C85B082468B46C8F1BE
:10622800030817462E461FFA87F909EB0B0C22883C
:1062380005EB0A031FFA8CFC9BB26146184692B222
:10624800CDF804C00293FFF73BF9C9EB0B0292B2F9
:106258000392029B22880399184692B2FFF730F9FD
:10626800DDF804C02288C5EB0A039BB261461846D4
:1062780092B20293FFF724F9029B228803991846E9
:1062880092B2FFF71DF905EB0B0292B2039209EBEC
:106298000A03228803999BB2184692B20293FFF729
:1062A8000FF9029B2288C5EB0B0C1FFA8CFC1846D1
:1062B800614692B2CDF804C0C9EB0A09FFF700F9AC
:1062C800228803991FFA89F992B24846FFF7F8F82D
:1062D8002288DDF804C092B248466146FFF7F0F81C
:1062E800B8F1000F04DA08EB860808F1060805E0A3
:1062F800F31B08F10A0808EB8308013F0136013552
:10630800BE42ADB28FD905B0BDE8F08FBC1A0020EF
:1063180008B9FFF713B8012801D1FFF70BB8704788
:10632800704700200146F0224FF4A073FFF7C8B968
:10633800704708B505280CD8DFE800F012140305EB
:106348000709094808BD094808BD094808BD0948A2
:1063580008BD0948094A0A4B40F24111FEF724FDDD
:10636800084808BD084808BD8801002078010020B9
:106378007001002068010020B2B405086EAF04085F
:10638800EDB20508900100208001002010B50446F8
:10639800FFF7CFFF014B18601C7110BDA001002052
:1063A800014B1879704700BFA001002008B5FFF71E
:1063B800C0FF808808BD08B5FFF7BBFFC08808BDCF
:1063C800F7B51F460B4B0C4E1D681446EA882B6820
:1063D800203C5443A4B2AE1B03EB440418BF01266F
:1063E800AB888DE8500017B1FFF7EEF901E0FFF731
:1063F80071FAFEBDA0010020900100202DE9F041B6
:106408000F46984615460446084E08E0204643467F
:106418003946FFF7D5FF33689B88E418A4B215F80E
:10642800012B002AF2D1BDE8F08100BFA0010020B5
:1064380010B5044608462146BDE81040DEE7094B82
:1064480070B5044618790E461546FFF7B4FFC6F135
:10645800F001091A89B220462A460023BDE8704097
:10646800CCE700BFA0010020704700BF044B1A68AA
:106478000AB9044A1A601A6810181860104670475A
:10648800400D0020843D00204FF0FF30704708B5D4
:106498000248034A034B3721FEF786FCD1B40508AE
:1064A80084AF0408EDB205080120704710B5044612
:1064B8000A4802210BF0BCF80028F9D00748214609
:1064C8000BF07FF8054801210BF0B2F80028F9D04D
:1064D8000248BDE810400BF071B800BF003800401A
:1064E80010B5194802210BF0A3F80028F9D0164876
:1064F80000210BF066F8144801210BF099F80028E8
:10650800F9D011480BF05AF80402A4B2002301E0B4
:1065180001339BB2002BFBD00B4802210BF088F80B
:106528000028F9D0084800210BF04BF80648012153
:106538000BF07EF80028F9D003480BF03FF8204311
:10654800C0F3CB0010BD00BF003800402DE9F04774
:106558008AB00AAF0A2001210AF0E4FD4FF4604333
:1065680047F8143D474EDFF824A1012400254FF0D9
:106578000208304639468DF81A508DF818808DF883
:1065880019808DF81B400AF025FA30460D210522A6
:106598000AF0A0FA30460E2105220AF09BFA0522DD
:1065A80030460F210AF096FA21464FF480400AF04F
:1065B800DDFD50460AF0B8FE4FF48273ADF80230A4
:1065C8004FF40073ADF80A303823ADF80C3050465C
:1065D80007236946ADF81030ADF80050ADF8045007
:1065E800ADF80650ADF80850ADF80E500AF0CEFEE2
:1065F800504621460AF065FFA9468DF81A503046E4
:106608004FF48055394605958DF818408DF8198056
:106618008DF81B400AF0DEF9304629460AF04BFA9D
:106628004025394618488DF818908DF819808DF84E
:106638001A908DF81B4005950AF0CCF921464FF4C5
:1066480080400AF09FFD062103200BF029F80C2357
:1066580007A88DF8213007958DF820908DF82240F5
:1066680009F0ACFE17238DF8243009A80F238DF804
:1066780025308DF826308DF8274002F039FF0AB012
:10668800BDE8F08700040240000C024000380040DA
:10669800014B1878704700BF440D0020024B5A8800
:1066A8009B8802800B807047440D0020014B00221C
:1066B8001A707047440D0020F0B593B06846002169
:1066C800482210F027FF6D46002464484FF480519B
:1066D8000AF0F3F9002301E001339BB2002BFBD051
:1066E8009020FFF7E3FE002301E001339BB2002B6B
:1066F800FBD0FFF7F5FE4FF48051074657480AF0E4
:10670800DAF9002301E001339BB2002BFBD0534898
:106718004FF480510AF0D1F9002301E001339BB214
:10672800002BFBD0D020FFF7C1FE002301E001338E
:106738009BB2002BFBD0FFF7D3FE4FF480510646E7
:1067480046480AF0B8F945F8047B01342E624448FB
:106758004021E4B20AF09DF910B9092CB5D101E045
:10676800092C78D19DE80C00D218029B0398069951
:10677800D218049BC018059BC018079BCB18089912
:10678800032490FBF4F092FBF4F25B1893FBF4F310
:10679800151AC11A9C1A002DB8BF6D420029B8BF3E
:1067A8004942002CB8BF6442502D03DD502909DD51
:1067B800502C50DC8D4205DAAC424FF0020405DB68
:1067C800111806E08C424FF0020401DAD11800E0FB
:1067D800C1180A9B099A0C980F9DD2180B9BD218C6
:1067E8000D9BC0180E9BC018109BEB18119D91FBB8
:1067F800F4F1032492FBF4F290FBF4F05B1993FBA1
:10680800F4F3161AC41A9D1A002EB8BF7642002C4B
:10681800B8BF6442002DB8BF6D42502E89B203DD67
:10682800502C09DD502D16DCA64205DAB5424FF092
:10683800020405DB131806E0A5424FF0020401DA52
:10684800D31800E0C318074A93FBF4F39BB2938074
:1068580001235180137013B0F0BD00BF0004024043
:10686800000C0240440D0020FFF712BFF7B50546A3
:106878000C4601A80DF10601FFF710FF1B4BBDF8F0
:106888000660BDF8040093E80600724301FB00228D
:1068980099685218164992FBF1F207EE102AF8EEA1
:1068A800C77A40F23F17FCEEE77A17EE902A92B2C9
:1068B800B2F5207F28BF3A462A801D69DA685B69ED
:1068C8006E4302FB0060C01890FBF1F107EE101A4E
:1068D800F8EEC77AFCEEE77A17EE903A9BB2B3F57A
:1068E800F07F28BFEF232380FEBD00BF4C0D0020A2
:1068F80040420F00FFF7DABE014B187E704700BF19
:106908004C0D0020FFF7CABE042808B505D9074872
:10691800074A084B7D21FEF747FA054B03EB800039
:10692800038B0B80438B138008BD00BFF2B40508AE
:106938008AAF040810B5050808B5082001F0BAF9AF
:1069480042F69643C31A584240EB030008BD10B5FF
:106958000A2001F0D7F90C4C20600E2001F0D2F982
:106968006060122001F0CEF9A060162001F0CAF98B
:10697800E0601A2001F0C6F920611E2001F0C2F97A
:1069880001236061237610BD4C0D002010B5FFF780
:10699800DDFD01F06DFA044601F076FA0749034679
:1069A8002246202009F024F8FFF7C6FF28B101F09D
:1069B80079FA10B9BDE81040C9E710BD4CB5050813
:1069C80010B5104C0A20216801F083F961680E2087
:1069D80001F07FF9A168122001F07BF9E168162027
:1069E80001F077F921691A2001F073F961691E2015
:1069F80001F06FF9082042F69641BDE8104001F019
:106A08004BB900BF4C0D00202DE9F04F0346A7B04D
:106A1800B0F800C01C898688DF885D89CDF810C071
:106A2800B249B0F802C0B3F80C90B3F80E80CDF8B4
:106A380024C00FFA84FB30B201220FFA87FE0BEB59
:106A4800000C0A7629B20FFA89FACDF888C001EB52
:106A58000E0C0FFA88F2CDF890C00AEB0B0CCDF8AB
:106A680030C002EB010CCDF858C0B3F810C05B8AF7
:106A7800CDF800C00FFA8CFC06910CEB00010A91CE
:106A880002930CEB0A011BB2239103EB0E010E914A
:106A980099182591049900FA81F0584450446044AB
:106AA800DDF824C006990EFA8CFEDDF810C01FFA36
:106AB80080FB1CFB0CF08E4416FB0600964414FB6E
:106AC8000400009A19FB09009E4412FB02001FFAF9
:106AD8008EFA0BF0B7FEDDF824C0029ACDE9120158
:106AE8001CFB0CF017FB070015FB050018FB080042
:106AF80012FB02000BF0A6FEDDF824C0029ACDE9D5
:106B0800140104991CFB01F317FB063615FB0466F8
:106B1800009B18FB096612FB03600BF093FEDDE98E
:106B28001423CDE90001DDE912010BF001FF044651
:106B38000D46DDE9000102460B460BF0F9FE024660
:106B48000B46204629460BF03FFDCDE91801584673
:106B58000BF088FECDE91001DDE91023DDE9000125
:106B68000BF0E6FECDE9060150460BF07BFE8046B1
:106B780089464246DDE912014B460BF0D9FEDDE9B4
:106B88001023CDE91C01DDE914010BF0D1FE002230
:106B980006460F46564BDDE918010BF0C9FE424682
:106BA80004460D464B46DDE906010BF0C1FE0246E0
:106BB8000B460BF00BFD02460B46204629460BF010
:106BC80005FD424604460D464B46DDE91C010BF027
:106BD800AFFE02460B46204629460BF0F5FCDDE9E0
:106BE800102304460D46304639460BF0A1FE0246F6
:106BF8000B46204629460BF0E7FCDDF828C0CDE916
:106C080002014FEA8C10DDF830C000EB0C20DDF8F3
:106C180010C0A0241CFB04000BF014FEDDF838C0E3
:106C2800CDE90A014FEA8C10DDF858C000EB0C20C2
:106C3800DDF824C01CFB04000BF004FECDE90C01B8
:106C480050460BF0FFFDDDE91023CDE91601DDE923
:106C58000C010BF06DFE4246CDE91E014B46DDE905
:106C68000A010BF065FE4246CDE920014B46DDE9FD
:106C780000010BF05DFE32463B460BF0A5FCCDE96A
:106C88000E0158460BF0DEFDDDE91C23CDE91A01A3
:106C9800DDE906010BF098FCDDF88CC0C024CDE9D5
:106CA800060104FB0CF0DDF888C0302505FB0C005C
:106CB800DDF810C078261CFB06000BF0C3FDDDF8DC
:106CC80094C0824604FB0CF0DDF890C005FB0C0074
:106CD800DDF824C01CFB06008B460BF0B3FDDDE994
:106CE800102306460F460BF023FE03E04C0D002050
:106CF800000014404246CDE904014B46504659462F
:106D08000BF016FEDDE9142380468946DDE90A0109
:106D18000BF00EFEDDE9002304460D46DDE90C010B
:106D28000BF006FE02460B46204629460BF04CFCAB
:106D38000022A14B0BF0FCFDDDE9202304460D46A3
:106D4800DDE91E010BF040FC02460B46DDE91601A9
:106D58000BF0EEFD02460B46204629460BF036FCAA
:106D6800002204460D46954BDDE90E010BF0E0FDCF
:106D780002460B46204629460BF028FCDDE9022393
:106D88000BF000FF88A3D3E900230BF0D1FD0CF032
:106D980069F88B490860DDE91223DDE90C010BF085
:106DA800C7FDDDE9002304460D46DDE90A010BF0C5
:106DB800BFFD02460B46204629460BF005FC002283
:106DC8007D4B0BF0B5FDDDE91E2304460D46DDE9DC
:106DD80020010BF0F9FB02460B46DDE91A010BF026
:106DE800A7FD02460B46204629460BF0EFFB002282
:106DF80004460D46714BDDE906010BF099FD02468C
:106E08000B46204629460BF0E1FBDDE902230BF097
:106E1800B9FE65A3D3E900230BF08AFD0CF022F834
:106E2800674A5060DDE90E23DDE90A010BF080FDB9
:106E3800DDE9062304460D46DDE90C010BF078FD7B
:106E480002460B46204629460BF0C0FB00220446AA
:106E58000D465A4BDDE918010BF06AFD02460B4658
:106E6800204629460BF0B2FBDDE902230BF08AFE2F
:106E78004DA3D3E900230BF05BFD0BF0F3FF504B60
:106E880059469860DDE9142350460BF051FDDDE9C1
:106E9800002304460D46304639460BF049FD0246AC
:106EA8000B46204629460BF08FFB0022424B0BF085
:106EB8003FFD424604460D464B46DDE904010BF012
:106EC80083FB02460B46DDE916010BF031FD024655
:106ED8000B46204629460BF079FB35A3D3E900235E
:106EE80004460D46DDE90E010BF022FD02460B4675
:106EF800204629460BF06AFBDDE902230BF042FE2F
:106F080029A3D3E900230BF013FD0BF0ABFFDFF847
:106F1800B0C0DDE91223CCF80C00394630460BF03E
:106F280007FDDDE9002304460D46504659460BF09F
:106F3800FFFC02460B46204629460BF045FB002283
:106F48001D4B0BF0F5FCDDE9042304460D464046D5
:106F580049460BF039FB02460B46DDE91A010BF0F6
:106F6800E7FC02460B46204629460BF02FFB10A3F0
:106F7800D3E9002304460D46DDE906010BF0D8FCF1
:106F880002460B46204629460BF020FBDDE902238A
:106F98000BF0F8FD04A3D3E900230BF0C9FC0BF0B8
:106FA80061FF074908610DE00000000080842E4160
:106FB8000000000000C0824000001440000089402A
:106FC8004C0D0020DDE90E23504659460BF0B0FC6D
:106FD800DDE9062304460D46304639460BF0A8FC89
:106FE80002460B46204629460BF0F0FA11A3D3E9D6
:106FF800002304460D46DDE918010BF099FC024612
:107008000B46204629460BF0E1FADDE902230BF096
:10701800B9FD0AA3D3E900230BF08AFC0BF022FF89
:10702800034A506127B0BDE8F04FC9E4AFF30080D0
:107038004C0D00200000000000C08240000000004D
:1070480080842E41AFF30080064A074B1A60074A36
:10705800074B1A60074B42F210721A60064B642203
:107068001A60704740420F00F026002080C3C90113
:10707800082D0020E42C00209C260020012808B5BB
:1070880003D05AD3022851D13CE02C4B1B78012B5A
:1070980003D013D3022B49D121E0294BC82019680A
:1070A80000F017FE274BCC20196800F012FE264B83
:1070B800D020196800F00DFED42033E0204BD820F2
:1070C800196800F006FE1F4BDC20196800F001FE6D
:1070D8001D4BE020196800F0FCFDE42022E0184B6D
:1070E800F820196800F0F5FD164BFC20196800F02F
:1070F800F0FD154B4FF48070196800F0EAFD4FF46D
:1071080082700FE00E4BE820196800F0E2FD0D4B8D
:10711800EC20196800F0DDFD0B4BF020196800F039
:10712800D8FDF420094B196800F0D3FD04F0F4FEF3
:1071380018B9BDE8084004F000BF08BD1C0E0020C7
:10714800F0260020082D0020E42C00209C2600209A
:1071580008B52E4B1B78012B02D0022B55D140E0ED
:107168002B4B1B78012B03D013D3022B4DD121E0DD
:10717800C82000F0C7FD274B1860CC2000F0C2FDE6
:10718800254B1860D02000F0BDFD244B1860D4209A
:1071980022E0D82000F0B6FD1E4B1860DC2000F07D
:1071A800B1FD1D4B1860E02000F0ACFD1B4B1860D2
:1071B800E42011E0F82000F0A5FD164B1860FC2033
:1071C80000F0A0FD144B18604FF4807000F09AFD99
:1071D800124B18604FF4827000F094FD104B186049
:1071E80008BDE82000F08EFD0A4B1860EC2000F086
:1071F80089FD094B1860F02000F084FD074B1860EA
:10720800F42000F07FFD064B186008BDC90100207E
:107218001C0E0020F0260020082D0020E42C002061
:107228009C26002008B504F077FE10B1BDE80840A0
:107238008EE7BDE8084007E7064B07495960C021BB
:10724800002219721E211A70D9601A745A611A76AE
:10725800DA617047EC1A002040787D0110B50321EF
:10726800FF22C02001F02CFC1F4C1021802220603E
:10727800C02001F025FC112180222060C02001F0EF
:107288001FFC122180222060C02001F019FC13216C
:1072980080222060C02001F013FC1421802220608D
:1072A800C02001F00DFC152180222060C02001F0D3
:1072B80007FC802220601621C02001F001FC20601C
:1072C800C0201721802201F0FBFB80222060B7211B
:1072D800C02001F0F5FB054B00221A745A611A769A
:1072E800DA6101221A7010BDC4260020EC1A0020B1
:1072F80038B5C0200321FF2201F0E2FB0B4D00242A
:107308002B19615D5A78C020023401F0D9FBC82CD2
:10731800F6D1B121AC22C02001F0D2FBC02003215C
:10732800002201F0CDFB002038BD00BFB6AF040835
:107338002DE9F34706460F4692461D461AB90C1F1B
:10734800E401914635E005EE902A06EE903AB8EE53
:10735800657AF8EE667AFC01C7EE277AA4F5007420
:107368009FED5C7A67EE877A17EE900A0BF08CFA3D
:1073780041EC100B0DF0ECFB59EC108B49464046E4
:107388000BF098FD24184FEACA100BF05BFACDE910
:10739800000128460BF056FA4B4642460BF0C8FA55
:1073A80002460B46DDE900010BF00EF90BF082FDF9
:1073B8008146002E14BF4FF022084FF01A08C5F37B
:1073C80007224146C02001F07BFB08F10101EAB227
:1073D800C02001F075FBC4F3014208F10201C0208E
:1073E80001F06EFBC4F3072208F10301C02001F08D
:1073F80067FBE2B208F10401C02001F061FBC9F3A8
:10740800034305F4702243EA123208F10501C02053
:1074180001F056FB08F10601C9F30722C02001F06C
:107428004FFB08F107015FFA89F2C02001F048FB21
:10743800C020B121A02201F043FB07EE107A264CB0
:10744800F8EEC77A0EBBD4ED015A06EE90AAB8EE54
:10745800657A05EE905AB8EE666AF8EE656A012319
:10746800C6EE266A237477EEA67A67EE277A17EEB9
:10747800900A0BF009FA41EC100B0DF069FB51EC86
:10748800100B0BF017FD606120E005EE90AAD4ED1B
:10749800016AB8EE656A05EE905AB8EE667AF8EEBB
:1074A800656A0123C6EE266A237677EEA67A67EE2A
:1074B800277A17EE900A0BF0E7F941EC100B0DF064
:1074C80047FB51EC100B0BF0F5FCE0610020BDE828
:1074D800FC8700BF00000043EC1A002000220123B3
:1074E80026E7012838B50D4604D002280CBF3C24F5
:1074F8002C2400E034242146C02001F05BFB05F079
:10750800070200F00F0040EA02122146C020BDE841
:10751800384001F0D5BA2DE9F3470A9C1D460746C5
:107528008A461646524B01E06D0864089C42FBD817
:107538002DB906F10076043EF601A94634E006EEC0
:10754800905AB8EE667A06EE904AF8EE667AF60138
:10755800C7EE277AA6F500769FED467A67EE877A1A
:1075680017EE900A0BF090F941EC100B0DF0F0FAC1
:1075780059EC108B494640460BF09CFC3618E80144
:107588000BF060F9CDE9000120460BF05BF94B46A2
:1075980042460BF0CDF902460B46DDE900010BF03F
:1075A80013F80BF087FC8146022F9BBF324BDB1987
:1075B8004FF0000893F8C880C4F307224146C02062
:1075C80001F07EFA08F10101E2B2C9B2C02001F06F
:1075D80077FA08F10201C9B2C6F30142C02001F0EE
:1075E8006FFA08F10301C9B2C6F30722C02001F0FF
:1075F80067FA08F10401C9B2F2B2C02001F060FADA
:1076080004F47024C9F3034308F1050143EA143272
:10761800C9B2C02001F054FA08F10601C9B2C9F391
:107628000722C02008F1070801F04AFA5FFA89F238
:107638005FFA88F1C02001F043FABAF1010F0CBFDC
:107648002F220F220DB942F04002012F06D002D39B
:10765800022F0AD105E0C020102104E0C02011212A
:1076680001E0C020122101F02BFA0020BDE8FC87C0
:10767800FFFF0F0000000043B6AF040807B5012361
:1076880000930023FFF747FF0EBD00280CBFFF2221
:10769800002208B5C020032101F012FA002008BD1D
:1076A80008B5C020B121AC2201F00AFA002008BDBB
:1076B80008B50420012109F035FD4FF4807001213F
:1076C800BDE8084009F05EBD07B502230093032317
:1076D8008DF804300348002369468DF8073009F017
:1076E80079F90EBD0008024030B5124D8BB0002468
:1076F80006A8069407940894099408F039FB0094A6
:107708008DF804408DF805400294039404942846AB
:10771800012469468DF8144008F0FBFA28460B212D
:107728002246062308F070FB2846214608F03AFB5B
:107738000BB030BD0020014010B5002104460122E5
:10774800302001F0BDF9C0B9012001F0B3FC002CD4
:10775800B8BF4034E4B210212246302001F0B0F91D
:10776800012001F0A7FC30201121224601F0A8F9E0
:107778000120BDE8104001F09DBC10BD10B50021EE
:1077880004460122302001F09BF9C0B9012001F024
:1077980091FC002CB8BF4034E4B2122122463020BC
:1077A80001F08EF9012001F085FC302013212246DA
:1077B80001F086F90120BDE8104001F07BBC10BD46
:1077C80038B5012205460C463020002101F078F931
:1077D800F0B9012001F06EFC25EAE5725F2AA8BF26
:1077E8005F223B21D2B2302001F06AF9012001F07A
:1077F80061FC24EAE4725F2AA8BF5F22D2B230207B
:107808003C2101F05DF90120BDE8384001F052BC8F
:1078180038BD302810B504460ADC10F17F0F02DBB2
:10782800002802DB05E06FF07E0404F5807400E0B8
:107838003024002130200A4601F042F9A8B901207D
:10784800E4B201F037FC41212246302001F038F93A
:10785800012001F02FFC30204221224601F030F9AE
:107868000120BDE8104001F025BC10BD282810B546
:10787800044609DC10F1180F02DB002802DB04E0E3
:107888006FF017047F3400E02824002130200A46D6
:1078980001F016F9A8B90120E4B201F00BFC53215C
:1078A8002246302001F00CF9012001F003FC3020C1
:1078B8005421224601F004F90120BDE8104001F0EE
:1078C800F9BB10BD08B530200021012201F0F8F8FD
:1078D80060B9012001F0EEFB30203321402201F095
:1078E800EFF80120BDE8084001F0E4BB08BD10B581
:1078F80030200021012201F0E3F8044660B901209C
:1079080001F0D8FB30203321224601F0D9F80120BC
:10791800BDE8104001F0CEBB10BD10B530200021ED
:10792800012201F0CDF80446A0B9012001F0C2FB04
:1079380034212246302001F0C3F8012001F0BAFBBF
:1079480030203721224601F0BBF80120BDE8104065
:1079580001F0B0BB10BD4020EEE640200EE708B5B0
:1079680000210122302001F0ABF8012001F0A2FB38
:1079780030203421024601F0A3F8012001F09AFBDF
:1079880030203721024601F09BF80120BDE808406D
:1079980001F090BB08B500210122302001F090F8D9
:1079A800012001F087FB302034210C2201F088F8F7
:1079B8000120BDE8084001F07DBB00000000000088
:1079C8002DE9F04F984B994A1968994B002914BF33
:1079D80091469946974B2DED048BC3F80090964B32
:1079E8000025002287B01A80AA46AB46A8465AE06E
:1079F800A2004046CDF804C002920AF045FF0746AF
:107A0800584601F100460AF03FFF02460B46384649
:107A180031460AF0D9FD39F9243007EE103AF8EE6C
:107A2800C77A064617EE900A0F460AF02DFF02465F
:107A38000B46304639460AF0C9FD0BF05BFA07469B
:107A480050460AF021FF0446284601F100460AF094
:107A58001BFFCDE90401DDE90423204631460AF085
:107A6800B3FD029A09EB02030446B3F9023007EEAC
:107A7800103AF8EEC77A0D4617EE900A0AF004FF9E
:107A880002460B46204629460AF0A0FD0BF032FAC2
:107A9800DDF804C0684A0CF1010CC3465546A2F84B
:107AA80000C08246B846644BB3F800C00FFA8CF4A5
:107AB800B32C9DDD58460AF0E7FECDE902014046A9
:107AC8000AF0E2FE002206460F465C4BDDE90201A1
:107AD8000AF02EFF02460B46304639460AF076FD7C
:107AE8000022574B0BF04EF80BF004FA4CA3D3E9E5
:107AF800002309EE900ADDE902010AF019FF0022CD
:107B08004F4B0BF03FF80BF0F5F909EE100A284639
:107B18000AF0BAFE044650460D460AF0B5FE0022A9
:107B280006460F4620462946444B0AF001FF024606
:107B38000B46304639460AF049FD0022404B0BF00F
:107B480021F80BF0D7F936A3D3E9002308EE900A01
:107B5800294620460AF0ECFE0022394B0BF012F8B9
:107B68000BF0C8F908EE100A69EE287A58EE297A5F
:107B780017EE900A0AF088FE68EE097A48EEA97AAC
:107B8800044617EE900A0D460AF07EFE45EC104BAF
:107B980041EC110B0DF0E0F851EC100B0BF0AAF9C9
:107BA80028EE088A08EEA88A07EE100A254B264C0C
:107BB800F1EE477AC3ED007A18EE100A0AF064FE77
:107BC80041EC100B0DF0D6F929EE099A51EC100B87
:107BD80009EEA99A0BF08EF9206019EE100A0AF046
:107BE80053FE41EC100B0DF0C5F951EC100B0BF0E6
:107BF80081F9D4ED007A07EE100A87EE877A134BE5
:107C08001860134BFDEEE77A83ED007A114BC3ED54
:107C1800007A07B0BDEC048BBDE8F08FAFF30080AD
:107C2800912B50E67AB6EB3F141B002096230020D8
:107C3800F61D0020101B00201C1B00200000E03F48
:107C4800000059400C2D0020242D0020182D002064
:107C5800142D0020181B002010B5084C204608F0F1
:107C680006FB074B1860FFF7ABFE064B06490122DF
:107C780020461A80BDE8104008F07ABB1060024028
:107C8800141B0020680D002020800010014B18688C
:107C9800704700BF181B002038B505460C46013553
:107CA800C1F3072101F014FAA8B2E1B201F010FA09
:107CB80000B238BD38B5044601F044F80134054631
:107CC800A0B201F03FF8EDB2C0B240EA052000B220
:107CD80038BD37B50B0E8DF804300B0C8DF8053018
:107CE8000B0A8DF806308DF80710002400E02846AE
:107CF80001AB451CE15C013401F0EAF9042CADB29A
:107D0800F5D13EBD37B5002400E02846451C01F0FA
:107D180019F801ABADB2E0540134042CF5D19DF84B
:107D280005009DF80430000440EA03609DF8073020
:107D380018439DF8063040EA03203EBD37B50023BE
:107D48000193002400E02846451C00F0FBFF01AB2E
:107D5800ADB2E0540134042CF5D19DED010A3EBDCD
:107D68007047000038B50446642001F0A3F925786F
:107D78006068AD00EDB2257008F091FE237A40FAF4
:107D880003F000F003000543104B257005F00F05C4
:107D98005A5D6378D218D2B2D3B20132D2B2022A73
:107DA800637001D80022A2705BB2012B03DD0123AE
:107DB800A3700023637094F90130013303DAFF23C1
:107DC800A3700023637094F9020038BD82B00408E0
:107DD800F7B504200121234F09F0A4F902AD0121D0
:107DE8004FF48040012409F0CDF900264FF4B07318
:107DF8003846694645F8083D8DF804608DF8074017
:107E080008F0E8FD1020214609F08CF9782369462E
:107E1800154800938DF804608DF8074008F0DAFDE6
:107E28000420214609F07EF921464FF4804009F0EC
:107E3800A9F91C233846694600938DF804608DF82B
:107E4800074008F0C7FD0220214609F06BF9B0236E
:107E580006488DF8046069468DF80740009308F0DD
:107E6800B9FDFEBD000802400010024000040240B7
:107E7800802108B5034808F00CFED0F1010038BF96
:107E8800002008BD0004024008B54FF48071044882
:107E980008F0FFFDD0F1010038BF002008BD00BF89
:107EA8000008024008B5FFF7E3FF08B1FFF7ECFF51
:107EB800C0B208BD70B500283AD01E4B1A78801899
:107EC8001D4AC0B292F90020187040B282421B4A83
:107ED80002DD11780139197093F9001092F9002028
:107EE80091FBF2F402FB14141549E4B21C700A88E1
:107EF800144B1A80144B154A18881080144A92F9AA
:107F0800000064B2013094FBF0F200FB1240114C07
:107F18002688114C258800FB065008800F490888E0
:107F28000F49098802FB00121A800E4B01221A70B1
:107F380070BD00BFBE3A0020E9360020C4360020DC
:107F4800F43A00200A370020BC3A0020BC38002050
:107F5800F63A002018380020583B0020843B0020C7
:107F68009A380020BC360020F0B5264A264C00235B
:107F78001370264A25681678254A12680FE0D45CE3
:107F88002F197F7817F0040F07D0302C02D1202347
:107F9800135431E01B4A137003E00133DBB29E42F5
:107FA800EDDA184B1B788342194B16D9A9B11A6818
:107FB800164C3121115430210BE01A681518125C47
:107FC8002E2A19D0303AD2B2092A88BF2970013036
:107FD800C0B222788242F0DA0EE01B681A5C79B1EE
:107FE8002E2A0DD05118C9B2392903D82F2998BF84
:107FF800302100E039211954BDE8F040FCF7ACBC51
:10800800F0BD00BF6C0D002048030020783C002024
:10801800E03A002010B5642001F04CF88648FFF7DC
:10802800A1FE864B1B7804460C2B00F26981DFE821
:1080380013F00D000D0067017500750037008C0006
:108048008E00BE00C100DB008E004301FFF71CFF5D
:1080580018B10120F9F75CFD52E1794B1888794B8A
:108068001B88C01A784B1B8890FBF3F0774B1A8853
:10807800774B1B88D31A774A128893FBF2F3DBB24B
:10808800C0B2032B00F2D380DFE803F00204060835
:10809800714A40E0714A3EE0714A3CE0714A3AE078
:1080A800FFF7F2FED8B100210A226F4810F002FC57
:1080B8006E4B002118600A226D4810F0FBFB6D4BD7
:1080C80018600420FEF762F9962005216A4A002309
:1080D800FEF794F90020FEF759F907F0E9F8584B34
:1080E8001888584B1B88C01A574B1B8890FBF3F015
:1080F800564B1A88564B1B88D31A564A128893FB3C
:10810800F2F3DBB2C0B21BB1012B40F0908001E06A
:10811800554A00E0564A594B1A6088E0002800F09A
:10812800EF80574B1A7806DD0132D2B2102A1A7046
:1081380008D9112205E0013AD2B2112A1A7001D9E0
:1081480000221A70F9F7CEFEDAE04E4B1870002CB8
:1081580000F0D6804C4B1B78022B40F0D1804B4B63
:108168001A78A418E4B20322B4FBF2F102FB11441A
:10817800E4B21C70464B474A1B5D022B137009D0B2
:10818800052B0CD0012B40F0BB804FF49170692176
:10819800414A08E04FF491706921404A03E0404A9F
:1081A8004FF4917069210023FEF728F9A8E0354BB8
:1081B8001870A5E0FFF768FEA0B10021394810F05B
:1081C800C5FA394B042083ED000AFEF7DFF8B42026
:1081D8000521364A0023FEF711F9FAF78FFA002035
:1081E800FEF7D4F82F4A16E0FFF74EFE90B10021B3
:1081F8002F4810F0ABFA2F4B042083ED000AFEF74E
:10820800C5F896200521294A0023FEF7F7F8002033
:10821800FEF7BCF8264A194B1A60094B1888094B17
:108228001B88C01A084B1B8890FBF3F0C0B221468C
:10823800FFF79AFE64E000BFA80100207126002025
:10824800F43A0020583B002018380020BC3A00209F
:108258009A380020843B0020B4260020D82600202D
:10826800EE2C0020A0260020603B0020C401002046
:10827800D03A0020C001002087B50508E03A002068
:10828800EA260020EC3A0020E4380020D50D002032
:10829800300300201C03002097B505089AB505088F
:1082A8009DB50508DC36002024030020A0B505088C
:1082B8000037002020030020FFF7E6FD08B107F093
:1082C800CFF914B1264B01221A70264B1A68A4184C
:1082D80014F5967FB8BF244A1C60B8BF1A601B68A3
:1082E800B3F5967F03DD1F4B4FF496721A601C4C52
:1082F80023782BB11D4B186801F0DCFA002323709A
:108308001B48FFF72FFD1B4B1B78013B0C2B25D877
:10831800DFE803F007242424211616241212162459
:108328001600FFF7C7FDFFF7A3FD002816D00220AF
:10833800BDE81040F9F7ECBB0F4B1B78022B0AD1B4
:1083480000280E4B01D1187010BD01DD012200E09C
:10835800FF221A7010BDBDE81040ABE510BD00BF8C
:10836800EC260020F03A0020D4FEFFFF90260020E3
:10837800B401002071260020E4380020251B0020CD
:1083880010B58CB01E490F2268460FF081F81D49C0
:108398000F2204A80FF07CF81B490F2208A80FF041
:1083A80077F800210822302000F08AFB012000F035
:1083B80081FE002404AB1DF80420E15C302000F0AD
:1083C8007FFB0134012000F075FE0F2CF2D1002153
:1083D8000922302000F074FB012000F06BFE00241D
:1083E80008AB1DF80420E15C302000F069FB013483
:1083F800012000F05FFE0F2CF2D10CB010BD00BFC1
:1084080094B00408A3B00408B2B0040810B58CB046
:108418001E490F2268460FF03BF81D490F2204A899
:108428000FF036F81B490F2208A80FF031F8002189
:108438000822302000F044FB012000F03BFE00241D
:1084480004AB1DF80420E15C302000F039FB013456
:10845800012000F02FFE0F2CF2D10021092230203C
:1084680000F02EFB012000F025FE002408AB1DF8CB
:108478000420E15C302000F023FB0134012000F0EF
:1084880019FE0F2CF2D10CB010BD00BFC1B004080A
:10849800D0B00408DFB0040810B58CB01E490F2214
:1084A80068460EF0F5FF1D490F2204A80EF0F0FFF4
:1084B8001B490F2208A80EF0EBFF002108223020EC
:1084C80000F0FEFA012000F0F5FD002404AB1DF8D1
:1084D8000420E15C302000F0F3FA0134012000F0C0
:1084E800E9FD0F2CF2D100210922302000F0E8FA32
:1084F800012000F0DFFD002408AB1DF80420E15C3A
:10850800302000F0DDFA0134012000F0D3FD0F2CFB
:10851800F2D10CB010BD00BFEEB00408FDB00408E5
:108528000CB1040807B50220012108F0FBFD012366
:1085380000938DF8043002238DF805300448002399
:1085480069468DF806308DF8073008F043FA0EBDFD
:108558000004024010B5084C01210022204608F012
:10856800AEFA40F2FF4000F0A5FD012120460A4680
:10857800BDE8104008F0A3BA0004024008B5FFF7B0
:10858800E9FF00210A46302000F09AFA012000F0A5
:1085980091FD01210A46302000F092FA012000F0F6
:1085A80089FD00210122302000F08AFA012000F024
:1085B80081FD01210822302000F082FA012000F01C
:1085C80079FD02210122302000F07AFA012000F022
:1085D80071FD00210A46302000F072FA012000F0F7
:1085E80069FD1B21CD22302000F06AFA012000F03D
:1085F80061FD04210322302000F062FA012000F01E
:1086080059FD06210922302000F05AFA012000F015
:1086180051FD07210822302000F052FA012000F015
:1086280049FD08217022302000F04AFA012000F0AC
:1086380041FD1E213020B02200F042FA012000F056
:1086480039FD05219122302000F03AFA012000F08E
:1086580031FD0D210322302000F032FA012000F014
:1086680029FD0E210022302000F02AFA012000F016
:1086780021FD14218022302000F022FA012000F090
:1086880019FD0B218822302000F01AFA012000F091
:1086980011FD0C218222302000F012FA012000F096
:1086A80009FD12218822302000F00AFA012000F08A
:1086B80001FD13218C22302000F002FA012000F085
:1086C800F9FC00210A46302000F0FAF9012000F0F8
:1086D800F1FC3D210222302000F0F2F9012000F0E7
:1086E800E9FCFFF74DFEFFF791FEFFF7D5FE3020BE
:1086F8000021012200F0E4F9012000F0DBFC3D211B
:108708006422302000F0DCF9012000F0D3FC0321C2
:108718000022302000F0D4F9012000F0CBFC042125
:108728000022302000F0CCF9012000F0C3FC002129
:108738000122302000F0C4F9012000F0BBFC0C211C
:108748000822302000F0BCF9012000F0B3FC0D2114
:108758000822302000F0B4F9012000F0ABFC0E2113
:108768000822302000F0ACF9012000F0A3FC0F2112
:108778000822302000F0A4F9012000F09BFC002121
:108788000A46302000F09CF9012000F093FC0222F8
:108798004021302000F094F9012000F08BFC3020BB
:1087A8004121002200F08CF9012000F083FC3F21D8
:1087B800D422302000F084F9012000F07BFC002155
:1087C8000122302000F07CF9012000F073FC102118
:1087D8000F22302000F074F9012000F06BFC112109
:1087E8000F22302000F06CF9012000F063FC122108
:1087F8000022302000F064F9012000F05BFC132116
:108808000022302000F05CF9012000F053FC09211F
:108818003C22302000F054F9012000F04BFC0021EC
:108828000122302000F04CF9012000F043FC3020F8
:108838003421024600F044F9012000F03BFC3020CE
:108848003721024600F03CF9012000F033FC3621C4
:108858000322302000F034F9012000F02BFC3921EC
:108868000322302000F02CF9012000F023FC3B21EA
:108878003C22302000F024F9012000F01BFC3C21B0
:108888000A46302000F01CF9012000F013FC0021FA
:108898000A46302000F014F9012000F00BFC5121A9
:1088A800C022302000F00CF9012000F003FC522116
:1088B8003020002200F004F90120BDE8084000F053
:1088C800F9BB00BF2DE9F04F454E464D93B001214D
:1088D8004FF4001008F026FC304607F0C9FB4FF0B3
:1088E800C0630293404B0393404B002404934FF41E
:1088F800B4794FF400334FF480684FF400674FF4B5
:10890800005A4FF4807B304602A90C9301930997D3
:10891800CDF8189005940794CDF82080CDF828A0BC
:10892800CDF82CB00D9407F02FFC22463046304984
:1089380007F085FC3046012107F08BFC01210A462F
:108948004FF0402008F05CFE284607F091FB294ACA
:10895800019B0392284A0C9304922846402202A9BC
:10896800059209970294CDF818900794CDF82080C5
:10897800CDF828A0CDF82CB00D9407F005FC2246C0
:1089880028461E4907F05BFC2846012107F061FCD8
:1089980042F2107701220221194808F031FE3846C8
:1089A80000F088FB3046012107F029FC0121284608
:1089B80007F025FC384600F07DFB0B238DF844308A
:1089C80011A801238DF845408DF846408DF84730B1
:1089D80000F08EFD384600F06DFB13B0BDE8F08F57
:1089E80010600240886002400C400040962300203E
:1089F800F61D00200C3C0040C6200020261B00204D
:108A0800003C004002481021012207F06FBC00BF63
:108A18001060024013B50220012108F083FB4FF4D7
:108A280010730E4C009302238DF804308DF8053036
:108A380001238DF806302046002369468DF807305B
:108A480007F0C8FF20460621042208F043F8204614
:108A58000921042208F03EF81CBD00BF00040240B2
:108A680030B5154D85B001214FF4001008F07EFB9C
:108A7800284608F045F80023ADF804304BF6FF739C
:108A8800ADF806303323ADF808304FF48063ADF805
:108A98000A304FF48043ADF80C3004AC074B28463D
:108AA800012144F8103D08F0CDF82846694608F041
:108AB80055F805B030BD00BF00540040801A0600CC
:108AC80073B54FF4961306460D461446019304E019
:108AD800019B5A1E0192002B57D031484FF40031A8
:108AE80008F0C8F90028F3D12D48012108F0B6F89C
:108AF8004FF48053019304E0019B5A1E0192002B0E
:108B080045D02748274908F0A0F90028F4D0244880
:108B18003146002208F0BAF84FF48053019304E07C
:108B2800019B5A1E0192002B33D01D481E4908F0A4
:108B38008CF90028F4D01A48294608F02AF94FF48D
:108B48008053019303E0019B5A1E01921BB3144802
:108B5800164908F07AF90028F5D01148214608F09E
:108B680018F94FF49613019303E0019B5A1E0192E2
:108B78009BB10B480E4908F07DF90028F5D008484C
:108B8800012108F077F8002008E0012006E0022023
:108B980004E0032002E0042000E005207CBD00BFC3
:108BA8000054004001000300820007008000070015
:108BB8000400001037B54FF4961304460D46019390
:108BC80005E0019B5A1E0192002B00F09B8056483D
:108BD8004FF4003108F04EF90028F2D15248012133
:108BE80008F03CF84FF48053019305E0019B5A1EAE
:108BF8000192002B00F088804B484C4908F025F979
:108C08000028F3D048482146002208F03FF84FF4E6
:108C18008053019304E0019B5A1E0192002B75D0EA
:108C28004148434908F011F90028F4D03E48294644
:108C380008F0AFF84FF48053019304E0019B5A1EEB
:108C48000192002B64D038483A4908F013F90028FB
:108C5800F4D03548012108F001F84FF4805301930E
:108C680004E0019B5A1E0192002B53D02E482F4935
:108C780008F0EBF80028F4D02B482146012208F030
:108C880005F84FF48053019304E0019B5A1E0192AA
:108C9800002B41D0244C2849204608F0EBF8002846
:108CA800F3D02046002107F0F9FF20460121238B4D
:108CB80007F0E0FF4FF48053019304E0019B5A1E34
:108CC8000192002B2AD018481C4908F0D3F8002834
:108CD800F4D0154808F05FF84FF480530193124A16
:108CE80003E0019B591E0191D3B113889B05F8D469
:108CF800012104460C4807F0D1FF0B48104908F041
:108D0800D3F80EE001240CE002240AE0032408E072
:108D1800042406E0052404E0062402E0072400E019
:108D2800082420463EBD00BF005400400100030057
:108D3800820007000400001002000010400000102C
:108D48000004001013B54FF496130446019305E090
:108D5800019B5A1E0192002B00F0AF8060484FF42F
:108D6800003108F087F80028F2D15D48012107F0AA
:108D780075FF4FF48053019305E0019B5A1E019241
:108D8800002B00F09C805648564908F05EF80028F1
:108D9800F3D05348A021002207F078FF4FF4805306
:108DA800019305E0019B5A1E0192002B00F0898077
:108DB8004B484D4908F049F80028F3D0210A4848A3
:108DC80007F0E7FF4FF48053019304E0019B5A1E1C
:108DD8000192002B77D04248444908F04BF800280C
:108DE800F4D0E1B23E4807F0D4FF4FF4805301932A
:108DF80004E0019B5A1E0192002B66D038483B497B
:108E080008F038F80028F4D03548012107F026FF8B
:108E18004FF48053019304E0019B5A1E0192002BEA
:108E280055D02F482F4908F010F80028F4D02C48C6
:108E3800A121012207F02AFF4FF48053019304E097
:108E4800019B5A1E0192002B43D0254C28492046ED
:108E580008F010F80028F3D02046002107F01EFF84
:108E680020460121238B07F005FF4FF4805301931F
:108E780004E0019B5A1E0192002B2CD018481D4972
:108E880007F0F8FF0028F4D0154807F084FF4FF4E6
:108E980080530193124A03E0019B591E0191E3B1EB
:108EA80013889905F8D4012104460D4807F0F6FE09
:108EB8000B48114907F0F8FF10E001240EE00224E6
:108EC8000CE003240AE0042408E0052406E0062454
:108ED80004E0072402E0082400E0092420461CBD21
:108EE8000054004001000300820007000400001045
:108EF80002000010400000100004001013B54FF4E9
:108F080096130446019305E0019B5A1E0192002B1B
:108F180000F0AF8060484FF4003107F0ABFF002845
:108F2800F2D15D48012107F099FE4FF48053019377
:108F380005E0019B5A1E0192002B00F09C805648C8
:108F4800564907F082FF0028F3D05348A021002299
:108F580007F09CFE4FF48053019305E0019B5A1ED5
:108F68000192002B00F089804B484D4907F06DFFB6
:108F78000028F3D0210A484807F00BFF4FF480532C
:108F8800019304E0019B5A1E0192002B77D04248BE
:108F9800444907F06FFF0028F4D0E1B23E4807F0DB
:108FA800F8FE4FF48053019304E0019B5A1E01928E
:108FB800002B66D038483B4907F05CFF0028F4D006
:108FC8003548012107F04AFE4FF48053019304E02D
:108FD800019B5A1E0192002B55D02F482F4907F0AC
:108FE80034FF0028F4D02C48A121012207F04EFEBE
:108FF8004FF48053019304E0019B5A1E0192002B09
:1090080043D0254C2849204607F034FF0028F3D0E8
:109018002046002107F042FE20460121238B07F05D
:1090280029FE4FF48053019304E0019B5A1E0192DC
:10903800002B2CD018481D4907F01CFF0028F4D03D
:10904800154807F0A8FE4FF480530193124A03E035
:10905800019B591E0191E3B113889C05F8D40121A5
:1090680004460D4807F01AFE0B48114907F01CFF8B
:1090780010E001240EE002240CE003240AE004249A
:1090880008E0052406E0062404E0072402E008249A
:1090980000E0092420461CBD0054004001000300E4
:1090A80082000700040000100200001040000010B9
:1090B8000004001082B0002304E0019B01330193F7
:1090C800009B01330093009B8342F6D302B07047A4
:1090D80037B54FF4805304460D46019304E0019BD5
:1090E8005A1E0192002B6DD03C484FF4003107F016
:1090F800C1FE0028F3D13948012107F0AFFD4FF434
:109108008053019304E0019B5A1E0192002B5BD00F
:109118003248334907F099FE0028F4D02F48A0219F
:10912800002207F0B3FD4FF48053019304E0019B44
:109138005A1E0192002B49D028482A4907F085FE7B
:109148000028F4D0210A254807F023FE4FF4805365
:10915800019304E0019B5A1E0192002B38D01F484E
:10916800214907F072FE0028F4D0E1B21B4807F04D
:1091780010FE4FF48053019303E0019B5A1E0192A5
:1091880043B31648184907F060FE0028F5D0134885
:10919800294607F0FEFD4FF49613019303E0019B67
:1091A8005A1E0192C3B10D48104907F063FE00280A
:1091B800F5D00A48012107F05DFD0D48FFF77AFF59
:1091C80000200AE0012008E0022006E0032004E075
:1091D800042002E0052000E006203EBD00540040C7
:1091E800010003008200070080000700040000104F
:1091F800A0860100F7B54FF4805304460D46164685
:10920800019304E0019B5A1E0192002B74D0404840
:109218004FF4003107F02EFE0028F3D13C4801211D
:1092280007F01CFD4FF48053019304E0019B5A1E84
:109238000192002B62D03648364907F006FE002816
:10924800F4D03348A021002207F020FD4FF48053CA
:10925800019304E0019B5A1E0192002B50D02C4828
:109268002D4907F0F2FD0028F4D0210A284807F01C
:1092780090FD4FF48053019304E0019B5A1E019224
:10928800002B3FD02248254907F0DFFD0028F4D005
:10929800E1B21F4807F07DFD4FF48053019304E0CD
:1092A800019B5A1E0192002B2ED019481B4907F02A
:1092B800CCFD0028F4D000244FF4961710E0295D67
:1092C800134807F066FD019703E0019B5A1E0192BF
:1092D800E3B10F48124907F0CDFD0028F5D001345D
:1092E800E3B2B342EBD30A48012107F0C3FC0D48AF
:1092F800FFF7E0FE00200AE0012008E0022006E077
:10930800032004E0042002E0052000E00620FEBD62
:10931800005400400100030082000700800007009D
:1093280004000010A086010013B50520012107F0F4
:10933800F9FE184C4FF4E053009302238DF80430E3
:109348008DF805302046002369468DF806308DF8E3
:10935800073007F03FFB20460A21062207F0BAFB38
:1093680020460C21062207F0B5FB062220460B21D9
:10937800A4F5006407F0AEFB4FF4004320466946AD
:10938800009307F027FB20460F21062207F0A2FBD7
:109398001CBD00BF000802401FB50446FFF7C2F815
:1093A800FFF75EFBFFF7EAF8FFF7BEFF01214FF476
:1093B800004007F0DBFE02940F4C1023ADF802309A
:1093C800204600236946ADF80430ADF80C30ADF8FE
:1093D8000030ADF8063007F0F8FF69464FF040203E
:1093E80008F0C7F82046012108F077F84FF0402030
:1093F800012108F072F81FBD003C004082B0002334
:1094080004E0019B01330193009B01330093009B0F
:109418008342F6D302B0704707B50420012107F054
:1094280081FE01214FF4804007F0ACFE4FF4007339
:10943800009300238DF804300348012369468DF812
:10944800073007F0C7FA0EBD000802400D4B07B5FC
:109458001A680D484FF47A73B2FBF3F20B4B013ADA
:109468005A600B4AF02182F8231000229A600722E2
:109478001A60084B084A00930121084B02F012F8C1
:109488000EBD00BFE4010020F426002010E000E03B
:1094980000ED00E000030020E40200204C02002060
:1094A800054B1A6812B11A68013A1A60034B1A6818
:1094B80001321A60704700BFB0260020C82600207D
:1094C80082B0044B0190019A1A601A68002AFCD1F4
:1094D80002B07047B0260020704700BF40F0BE6061
:1094E800024B40F42020D860704700BF00ED00E038
:1094F800C37810B503B3164B4278DB688478DB4336
:10950800C3F30223C3F10401C9B202FA01F10F2225
:1095180042FA03F2C9B222400A430E4B0178120103
:10952800CB18D2B283F8002303780122590903F03B
:109538001F0302FA03F307E003780122590903F035
:109548001F0302FA03F32031024A42F8213010BD0A
:1095580000ED00E000E100E021F0604121F07F0132
:10956800014B08439860704700ED00E0044B1A690E
:1095780009B1104301E022EA00001861704700BFFA
:1095880000ED00E0044B1A6804280CBF42F0040206
:1095980022F004021A60704710E000E0014B93EDDE
:1095A800000A7047142D0020014B93ED000A704704
:1095B8000C2D0020014B93ED000A7047202D002050
:1095C800014B93ED000A7047102D0020014B93EDDD
:1095D800000A7047242D0020014B93ED000A7047C4
:1095E800182D00200000000008B5FDF737FE002008
:1095F800012324210246FDF79BFE124B1B78013BF9
:10960800DBB20020012B05D80146FDF76AFF0120D7
:10961800002104E00721FDF764FF01200721FDF781
:1096280060FF63221221C020FFF74AFA02200121BD
:10963800FDF757FFFEF734F80120BDE80840FEF7B4
:1096480024B800BF1C0E00200E4B1B78062B05D13A
:109658000D4B0E4A196812688A181A600C4B1B7851
:10966800013BDBB2012B084B196805D8094A914226
:1096780007DD01321A607047074A914201DD013265
:109688001A60704771260020E82C00206826002008
:109698001C0E00207FD1F008FF27ED080F4B1B7828
:1096A800062B05D10E4B0F4A196812688A1A1A60E0
:1096B8000D4B1B78013BDBB2012B094B05D80B4A3C
:1096C8001968914208DC1A6070471A68B2F57A2F57
:1096D800DCBF4FF47A221A60704700BF7126002061
:1096E800E82C0020682600201C0E002020A107007E
:1096F8002DE9F04F6A4B6B4C1B688DB019220A900C
:1097080069485343B0FBF1F01C190D4609F09AF86B
:1097180041EC100B0BF01CFA51EC100B09F0CAFBD2
:1097280010F0010F804618BF00F1FF3805FB08F064
:1097380009F088F8064620460F4609F083F80246E5
:109748000B463046394609F01DFA04460D4645ECED
:10975800104B0BF0FDF957EC106B204632463B4698
:10976800294608F031FFCDE902013946304609F0B3
:10977800A1FB47A3D3E900230B90DDE9020109F01F
:1097880053FB002858D1012000264FF01509314617
:1097980007464FF0000A4FF0000B03E03046394609
:1097A800069E049FA7FB0A23541807FB0B333F4A66
:1097B80043F100050023A242AB41CDE904453ED365
:1097C800A6FB0A23141806FB0B33384843F100059F
:1097D8000021A042A941CDE9064530D3DDE90201C7
:1097E8002DA3D3E90023049C069D09F01DFB40BB73
:1097F800DDE9022300202E4909F0C4F982468B4690
:109808004BEC10AB0BF0A4F95046594653EC102B17
:109818008DED080B08F0D8FECDE90201DDE908015D
:1098280009F016FE09F1FF395FFA89F982468B467D
:10983800B9F1000FB2D104E00125002401E035465A
:109848003C460B9A0A9BD1B25BB9184622462B4676
:10985800FDF76EFD0A980123009301464246034630
:1098680009E022462B460120FDF762FD0120009009
:10987800014642460023FDF74EFEFDF711FF012089
:109888000DB0BDE8F04FFDF700BF00BFAFF300809B
:10989800956479E17FFDA53DBBBDD7D9DF7CDB3D74
:1098A800F03A002040787D0100E9A435FFFF0F0061
:1098B8000000F03F2B4A2C4B1278012A10B5186093
:1098C8000BD12A4A904201DD01321A60284A1B68EE
:1098D80093420EDC244B1A600BE0022A09D1254A78
:1098E800904201DD01321A60234A1B6893420FDC63
:1098F8000CE01D4B214A1968914201DD01321A60C2
:109908001B68B3F57A2F03DC4FF47A22164B1A60E2
:10991800154B1B4A19681B4B1B4C1B68CB189342F1
:1099280023601ADC0020FFF7E3FE01202168FFF71F
:10993800DFFE0C4B1B78013BDBB20020012B05D866
:109948000146FDF7CEFD0120002104E00721FDF7C7
:10995800C8FD01200721FDF7C4FD034B1A680B4B16
:109968001A6010BD1C0E0020E82C00207FD1F008E2
:1099780020A107007F74D21A60E31600FF27ED08C4
:1099880080D1F008002D0020042D0020D8360020BA
:10999800014B18688EE700BFE4260020AFF3008073
:1099A8007047FEE7FEE7FEE7FEE77047704770473F
:1099B80002F036B910B5094CA37A4BB1084B1A68B6
:1099C80022F006021A6000F013F8204600F047FE65
:1099D8004FF48020BDE8104006F058BDF426002062
:1099E80010ED00E0014801F009B800BFF42600209E
:1099F800364BD3F8882042F47002C3F88820344BE1
:109A08001A6842F001021A6000229A60196821F06F
:109A1800847121F4803119602E495960196882B027
:109A280021F480211960DA60009201921A6842F4E8
:109A380080321A601A6802F400320192009A0132E8
:109A48000092019A1AB9009AB2F5A06FF2D1204B90
:109A58001B6813F4003318BF01230193019B012BEA
:109A68002ED11B4B1A6C42F080521A641A4A1168A4
:109A780041F4804111609A689A609A6842F4004201
:109A88009A609A6842F4A0529A60144A5A601A6816
:109A980042F080721A6019680D4A8901FBD5104B93
:109AA80040F205611960936823F00303936093689B
:109AB80043F002039360936803F00C03082BFAD178
:109AC800024B4FF000629A6002B0704700ED00E070
:109AD800003802401030002400700040085440074D
:109AE800003C0240184B194A996801F00C010429FE
:109AF80003D0082903D0164B19E0164B17E0596814
:109B08005A6811F4800F596814BF124B104B02F0B9
:109B18003F02B3FBF2F30C4A5268C2F30142C1F3AD
:109B28008811013252004B43B3FBF2F3074A13602A
:109B3800054B9A68054BC2F303129A1819681279F3
:109B480021FA02F21A60704700380240E40100204E
:109B58000024F40000127A0037B51C2301240025E4
:109B680001A88DF804308DF805508DF806408DF861
:109B78000740FFF7BDFC2046214607F0F7FA0A49DF
:109B880040F2E1434B6040F24F130B800D814D8052
:109B98004FF0804007F092FE4FF080402146224669
:109BA80008F051FA3EBD00BF282D002008B54FF03F
:109BB8008040012108F05CFA80B101214FF080401B
:109BC80008F061FAFEF726FA054B064A11781A786A
:109BD8008A181A70044B1A8801321A8008BD00BF0F
:109BE80095260020EC3A0020780D002008B540208A
:109BF80006F03EFC30B1FCF75FFD4020BDE80840B0
:109C080006F044BC08BD0000014608B5044808F049
:109C1800F9FB0348402108F0A2FC0028F9D008BD50
:109C280000440040F0B589B04FF4E13301200193BE
:109C380000232B4CADF808301E460146ADF80A301B
:109C4800ADF80C30ADF810300C23ADF80E3007F03D
:109C580069FA4FF40030012107F088FA20680221E0
:109C6800072206F037FF07226068032106F032FF5B
:109C78000125022704232068059305A98DF81A6099
:109C88008DF81B508DF818708DF8197006F0A2FE2B
:109C980008236068059305A98DF8187006F09AFEE8
:109CA800A06801A908F004FB2A4640F225510D4896
:109CB80008F03CFC262307A88DF81C308DF81D60A1
:109CC8008DF81E608DF81F50FFF712FCA06829461A
:109CD80008F06BFB044A054B1A6009B0F0BD00BFE1
:109CE800F801002000440040119C00087C3C002042
:109CF800024B9868002108F058BB00BFF80100200B
:109D080010B5094C40F22551204608F032FC50B1FC
:109D1800A288D2B2112A02D1044B01211970044B36
:109D280019884A401A8010BD004400407F0D002069
:109D3800880D00207047704773B50120014607F071
:109D4800F1F9264C4FF4D8530093022303268DF8DB
:109D580004302046002369468DF806308DF8073018
:109D68008DF8056006F036FE204608210A2206F026
:109D7800B1FE204609210A2206F0ACFE20460B213E
:109D88000A2206F0A7FE0A2220460C2106F0A2FEAF
:109D980001254FF480632046694600938DF80650EC
:109DA8008DF807508DF8056006F014FE0A210A4662
:109DB800204606F08FFE29464FF4804007F0E2F96E
:109DC8008020294607F0BAF94FF08050294607F05D
:109DD80009FA284606F05AFB7CBD00BF0000024085
:109DE80007B54FF4C060FFF779FB43238DF80430C3
:109DF8000322012301A88DF805308DF806208DF87F
:109E08000730FFF775FB0EBD782358430723B0FBD7
:109E1800F3F0002301338342FCD970474FF47A737F
:109E28005843F1E737B50023104C0193054603204A
:109E3800FFF7EAFFEB681A69013C019213D0019A17
:109E4800002AF4DA019A42F001020192019A1A6199
:109E5800064A1969013A019102D00199C907F8D453
:109E68000320FFF7D1FF00203EBD00BF410D0300D6
:109E780010B5C47874B900EB820003339B10D0F896
:109E8800D000224603E051F8044C0132046004314A
:109E98009A42F8D1002010BD033230B59210D0F8A4
:109EA800D0400B46002003E02568013043F8045CED
:109EB80004339042F8D101EB800030BD0122F0B5A7
:109EC8000023827040220129C37082800CD10823AC
:109ED8000370042343704FF4A073C38002230372FA
:109EE800C1724FF0A04309E041B90C230370062367
:109EF80043704FF4A063C3801F4BC17203F5006227
:109F08000261C3604678044601461A46002508E007
:109F180002F5106C02F530620A65C1F814C001350B
:109F28003A460431B54202F12007F1D303F58062C5
:109F3800426103F58862C0F8CC20067803F5A06575
:109F48000146002203E0C1F88C500132203504316B
:109F5800B242F8D31946002202E0C4F8CC1001320C
:109F68000434B24201F58051F7D303F56063C0F8B9
:109F78000C310020F0BD00BF0000044038B5037A62
:109F8800C2680025012B044625D1936B417A65F3FD
:109F9800104309B143F480139363D36823F4800317
:109FA80023F0500343F010036FF3C3036FF3C71399
:109FB8006FF351436FF3D343D3602046FFF732FF6B
:109FC800E378012B3ED1052363F34405E36845F0AC
:109FD80020059D6036E0D36843F04003D360FFF767
:109FE80021FF237A627A032B14BF4FF434134FF402
:109FF8003C130AB143F48013E26814209363FFF71B
:10A008000DFFE268217AD368032908BF43F480333F
:10A01800D360237A032B15D1156B012363F39B655A
:10A028006FF3D7552D2345F0805563F31645156317
:10A03800C820FFF7F3FEE36845F400051D63C82058
:10A04800FFF7ECFEE378012B07D1E3689D68052252
:10A0580062F3440545F020059D60002038BDC368C3
:10A068009A6842F001029A6000207047C3689A68B3
:10A0780022F001029A600020704707B5002301937F
:10A08800019B43F020030193019B61F38A13019321
:10A09800019BC2681361064B1169013B019102D013
:10A0A80001998806F8D40320FFF7AEFE00200EBD04
:10A0B800410D030007B500230193019B43F01003F2
:10A0C8000193019BC2681361064B1169013B019121
:10A0D80002D00199C906F8D40320FFF795FE0020A5
:10A0E8000EBD00BF410D030008B5C268D368012941
:10A0F8006FF35D736FF39E7302D143F0005302E078
:10A1080009B943F080433220D360FFF787FE00206F
:10A1180008BDC368586900F001007047C3685B69EF
:10A1280013F0010F14BF002001207047C36858695D
:10A1380000F001007047C3685A6998691040704779
:10A14800C3685868704703691A6861F301021A60A6
:10A158007047C268002393614FF0FF335361536027
:10A1680053610B4B9361C3789169002B14BF4FF473
:10A1780000634FF4016343F4701343F4405343F016
:10A18800080321EA03010B4393610020704700BFD5
:10A1980000080080F8B5D0F80C3100221A60036975
:10A1A80015461A6865F3CC221A60C37A012B044657
:10A1B8001BD10321FFF7C7FFE36880214FF480021A
:10A1C80061F30F0259629A62C02262F30F0561F3CC
:10A1D8001F454FF4A072C3F8045162F30F056FF3E3
:10A1E8001F45C3F80851C3F80C5110212046FFF74A
:10A1F80044FF2046FFF75EFF226900234FF0FF313E
:10A208001361204653611E469161FF25D3612146A3
:10A2180010E082691768C7F3076707F08007FFB285
:10A22800002F14BF4FF090470027176001331661C5
:10A238000430956062789342EBD300231D46FF20DB
:10A2480010E04A6D1668C6F3076606F08006F6B297
:10A25800002E14BF4FF0904600261660013315619A
:10A268000431906062789342EBD323691A6942F40F
:10A2780080721A61E278012A04D1054A402161F30B
:10A2880059421A632046FFF764FF0020F8BD00BF5B
:10A298000301010003699B68C3F34103013B022BDF
:10A2A8009ABF024AD05C0320704700BF50B104082F
:10A2B80010B5036981699C680A68C4F341000228E3
:10A2C80002D06FF30A0202E0032060F30A020A6078
:10A2D8005A6842F480725A60002010BD30B54D783B
:10A2E8000B780022012D00EB830405D105FA03F356
:10A2F800A46963F30F0205E0012505FA03F3646D11
:10A3080063F31F422368C3F3072505F08005EDB208
:10A318006DB98D6865F30A03CD78C98865F39343F1
:10A3280061F3995343F0805343F400432360036976
:10A33800D9690A43DA61002030BD30B54D780B7811
:10A348000024012D224600EB830105D105FA03F311
:10A35800896963F30F0205E0012505FA03F3496DE6
:10A3680063F31F4203696FF3CF340C60D96921EAA4
:10A378000202DA61002030BDF8B54F780B78012F62
:10A3880000EB830349D19E694C69356833692A46D5
:10A3980064F3120314B967F3DC430BE08F68E41924
:10A3A800013CB4FBF7F7CC7867F3DC43012C08BF1A
:10A3B80064F35E733361C378012B06D10B780C69A3
:10A3C80000EB83039B695C610CE0CB78012B09D01F
:10A3D8004B693BB103690C785E6B012707FA04F4FB
:10A3E80034435C63CB78012B07D103699B68DB0599
:10A3F80054BF45F0005245F080520B7800EB8303C0
:10A4080042F004429B691A60CB78012B38D10A7854
:10A418008B8AC968FFF72CFD32E05E6D4F6935689D
:10A428008C6833692A462FB964F31203012464F354
:10A43800DC430AE03F19013FB7FBF4F7BF05BF0D46
:10A4480067F3DC437C4364F312033361C378012B65
:10A4580005D10B780C6900EB83035B6D5C61CB78ED
:10A46800012B06D14B7913B145F0005201E045F0BC
:10A4780080520B7800EB830042F00442436D1A606F
:10A488000020F8BD73B54D78012D3DD183694A6927
:10A498001E681C690094E4B242B962F306048DF8A0
:10A4A80000409DF8024065F3C4040EE08D68AA429E
:10A4B80086BF4D6165F3060462F306048DF800401B
:10A4C8009DF80240012262F3C4048DF80240009A0C
:10A4D8001A61C278012A05D10A780C6900EB820258
:10A4E8009269546146F004421A60C378002B34D153
:10A4F8004B69002B31D003690A78586B012101FAA6
:10A5080002F202435A6328E00B784E698C6800EB2C
:10A5180083035B6D1A681D690095EDB206B14C6145
:10A5280064F306059DF802408DF80050012565F397
:10A53800C4048DF80240009C1C61C378012B05D12E
:10A548000B780C6900EB83035B6D5C610B7800EBA7
:10A55800830042F00442436D1A6000207CBD4B78B2
:10A56800012B0B7800EB83000AD182691368C3F3CF
:10A57800076101F08001C9B221B143F0804301E0D5
:10A58800426D136843F400131360002070474B7842
:10A59800012B0B78C97800EB83000CBF8269426DF0
:10A5A80002391368C9B26FF35553012998BF43F0B4
:10A5B800805313600020704703699A69D869104076
:10A5C800000C704700EB810102694B6D9B68506974
:10A5D8001840704703699869DB69184080B2704772
:10A5E80082B000230093C0238DF80330012200239A
:10A5F80062F3C4038DF8023018238DF80030009AF6
:10A60800436D1A61C278012A06D100F5B960586114
:10A618001A684FF080221A6002B07047D0F81431DF
:10A6280010B50446D3B103699A68D20716D5827A61
:10A6380042B1D0F80C21D0F80C116FF341026FF33E
:10A6480000020A605A6842F001025A600520FFF7CA
:10A65800E5FB23695A6822F001025A6010BD837A2B
:10A6680063B103699B68D90708D5D0F80C31D0F8D5
:10A678000C216FF341036FF300031360704701234C
:10A6880010B5002280F8123104460346FF2104E089
:10A6980058698160186D01328160607804338242A4
:10A6A800F6D3236900221A615A61DA614FF0FF324A
:10A6B8009A612046FFF7FEFC20461021BDE81040B5
:10A6C800DBE44B78012B0B7800EB83000FD1836917
:10A6D8001868C0F3074000F02003DBB2CBB900F0E4
:10A6E8000200C0B200280CBF302020207047436D04
:10A6F8001868C0F3074000F02003DBB25BB900F034
:10A708000200C0B200280CBF4FF440504FF4005074
:10A718007047102070474FF4805070474B78012BDA
:10A728000B7810B500EB83030AD19C69102A2368C3
:10A7380002D1BDE8104012E7202A0CD0302A0FE0E1
:10A748005C6DB2F5805F236802D143F400131BE00F
:10A75800B2F5005F02D143F0006315E0B2F5405F47
:10A768000FD1C3F3074202F02002D2B222B1002374
:10A778004B71BDE810400AE743F0806343F0802343
:10A7880002E00AB962F3CF33236010BDF8B504467E
:10A79800FFF794FB0122002384F8122184F8133177
:10A7A80028271646194640250CE007FB03F000F55C
:10A7B8008C7022182354D3805670D1709560D16064
:10A7C8005161013362789342EFD30023282619465A
:10A7D80040250CE006FB03F000F55C7022182354BA
:10A7E800D3805170D1709560D16051610133627826
:10A7F8009342EFD32046FFF739FC2046FFF7BEFB14
:10A8080000212046FFF770FC2046FFF7C3FC2046D6
:10A81800BDE8F840FFF723BC70B5CDB20C464FF049
:10A82800280601F07F0106FB010115F0800F14BF17
:10A8380001F58C7101F55C7104F07F04ED090C7071
:10A848004D708A60CB7005B1CC80022B01D10023FA
:10A858000B71FFF743FD002070BD10B5CAB201F0BF
:10A868007F034FF0280404FB030312F0800F14BF8A
:10A8780003F58C7303F55C7301F07F01D20919703D
:10A888005A701946FFF759FD002010BD38B501F080
:10A898007F0528246C4304F55C7401194B6100237F
:10A8A8008B614B70EBB20355CA60C478012C08BFAA
:10A8B8000A6113B9FFF7E6FD01E0FFF75DFD00202F
:10A8C80038BD70B501F07F042825654305F58C7502
:10A8D80041190126E4B2CA600A6100224E7044554B
:10A8E8008A614B6114B9FFF7CDFD01E0FFF744FD24
:10A8F800002070BDCAB212F0800F10B54FF02803C7
:10A9080006D001F07F0403FB040303F58C7303E016
:10A9180003FB010303F55C73D209012401F07F01F5
:10A9280019709C705A701946FFF719FE002010BD67
:10A93800CAB212F0800F10B54FF0280306D001F00C
:10A948007F0403FB040303F58C7303E003FB01039B
:10A9580003F55C730024D20901F07F0119709C7023
:10A968005A701946FFF713FE204610BD08B50B06AE
:10A9780004D501F07F01FFF780FB01E0FFF79AFBA8
:10A98800002008BD0369002261F30A1219680A430E
:10A998001A60704703695A6803206FF341025A60CE
:10A9A800FFF73CBA03695A68032042F002025A6072
:10A9B800FFF734BA11F0800F4FF0280306D001F0EA
:10A9C8007F0103FB010101F58C7103E003FB010129
:10A9D80001F55C71FFF775BE11F0800F4FF0280389
:10A9E80006D001F07F0103FB010101F58C7103E042
:10A9F80003FB010101F55C71FFF790BE2DE9F74FEC
:10AA08000446FFF78BFB002800F03F822046FFF743
:10AA180092FB0546002800F03882C0F3074000F09A
:10AA28000800C0B2002861D02046FFF7C5FDA14646
:10AA3800824627464FF00008DFF86CB32E4650E0F8
:10AA48001AF0010F46D05FFA88F2114620460092AC
:10AA5800FFF7B8FD10F0010F0546009A20D07B6D76
:10AA680001259D60E178A94207D11B69D9F87813BF
:10AA7800C3F31203CB1AC9F88833DBF80030204639
:10AA88001B6811469847E378012B09D1B8F1000FEC
:10AA980006D194F81131052B02D12046FFF7A0FD0D
:10AAA80005F00203DBB213B17B6D02259D6005F052
:10AAB8000403DBB213B17B6D04259D6005F0080526
:10AAC800EDB23DB1DBF8003020469B6898477B6DBE
:10AAD8000820986008F101084FEA5A0A043709F17A
:10AAE8002809BAF1000FABD135460120C5F3074359
:10AAF80003F00403DBB2002B00F0AF802046FFF721
:10AB080069FD264683464FF0000801959FE01BF03B
:10AB1800010F00F0978023695FFA88F919695D6B66
:10AB280004EB890225FA09F59269ED019268EDB204
:10AB38000D431540EA071CD55A6B012000FA08F1AD
:10AB480022EA01025A63B369974A98601368054676
:10AB58005B68204649469847E378AB4209D1B8F18B
:10AB6800000F06D194F81131042B02D12046FFF7CB
:10AB780037FD05F00403DBB213B1B36904259D600A
:10AB880005F00803DBB213B1B36908259D6005F031
:10AB98001003DBB213B1B36910259D6005F02003E3
:10ABA800DBB213B1B36920259D6005F04003DBB229
:10ABB80013B1B36940259D6005F00203DBB213B100
:10ABC800B36902259D6025F07F0515F0FF0F39D088
:10ABD800282505FB084505F58C75C246AB696A69E9
:10ABE800C3EB020CAB689C4528BF9C460CF1030CD8
:10ABF800B3694FEA9C0C9B696746A04614E0AA68B3
:10AC0800E9681C1B944228BF1446A3B240464A4632
:10AC1800FFF72EF9EB681B19EB60AB69E71C1C19F1
:10AC2800AC61B3699B69BF089BB2BB4205D9AC69EB
:10AC38006B699C4201D2002BE1D1B369802544465F
:10AC48009D60D04608F101084FEA5B0B0436BBF162
:10AC5800000F7FF45CAF019D012005F00203DBB219
:10AC680013B1E36802225A61C5F3076303F0800356
:10AC7800DBB2CBB1A37A43B1D4F80C31D4F80C21B0
:10AC88006FF341036FF30003136023695A6822F0DE
:10AC980001025A60444B1B6820469B699847E36849
:10ACA8004FF000425A610120C5F3072303F008035F
:10ACB800DBB2F3B13C4B1B6820465B6998472369BC
:10ACC800E2689B684FF400615161A27A82B1DB07A8
:10ACD8000ED5D4F80C311A6842F001021A601A68CD
:10ACE80042F003021A60314B1A6942F006021A61F7
:10ACF800012005F00803DBB243B12B4B1B6820464B
:10AD0800DB689847E36808225A61012005F01003C0
:10AD1800DBB2002B33D0E3689A6922F010029A6103
:10AD28001F6A282607F00F0306FB0346C7F34343B1
:10AD3800022B06F55C7602D0062B1AD10EE047F6F8
:10AD4800F0733B40ABB1C7F30A172046F1683A46A7
:10AD5800FFF7A2F8F368DB19F36007E004F5B961BF
:10AD680020460822FFF798F8C7F30A17B369DF19D6
:10AD7800B761E3689A6942F010029A610120C5F34D
:10AD8800072303F01003DBB2002B39D023695A687C
:10AD9800002622F001025A6031462046FFF76DF97D
:10ADA80023463246FF2108E09402002000ED00E02F
:10ADB80058698160186D013281606078043382427D
:10ADC800F6D3236901274FF0FF3267F30F069A6124
:10ADD80067F31F460F22DE615A612F221A611A6833
:10ADE8006FF30A121A602046FFF7FAFBE3684FF484
:10ADF80080525A61264B1B6820461B699847384683
:10AE0800C5F3072303F02003DBB2EBB12046FFF7BD
:10AE18004FFAE3682046DE68FFF73CFA032806D1BC
:10AE28000023A3704FF40073A380092304E00123D7
:10AE3800A3704023A380052363F38D26E3684FF4B2
:10AE48000052DE6001205A61C5F3074303F0100386
:10AE5800DBB24BB10E4B1B682046DB699847E368B1
:10AE68004FF480125A610120C5F3074505F020050B
:10AE7800EDB255B1064B1B6820461B6A9847E3683C
:10AE88004FF400125A610120FFE7BDE8FE8F00BFB2
:10AE98009402002043230B800048704704020020DE
:10AEA80038B51F4B1A68511C052A196035D1197914
:10AEB800002201291A6030D09968B1F5006F08BFE7
:10AEC8009A60174B9968DC68A1421A4602D10022A1
:10AED8001A7122E086BFC1F500631361C1EB040457
:10AEE800D0F8EC3598BF14611569B3F839300C4CBB
:10AEF8009D428AB204D95918ED1AA160256104E06F
:10AF08006918A1600021ABB22161054901240C71C7
:10AF180004498A188121FFF7D4FC002038BD00BFFE
:10AF28008C0D0020C72D002038B528230A4D03FBBF
:10AF380001010A4BB1F888131B6904462846984753
:10AF4800D4F8EC352046B3F8403001212A46FFF703
:10AF58009DFC002038BD00BF7F2D0020800200200E
:10AF680070B50B7813F0600506460C4625D0202DE9
:10AF78001FD1CD88B5B113F0800F487808D0214B88
:10AF880021499B682A469847E2881F49304625E0B0
:10AF98001E4B1D4958641E4B30465D612A4600F021
:10AFA80022FB1DE0174B48789B6829462A4698479C
:10AFB80025E000F077FB022521E04B780A2B11D021
:10AFC8000B2B14D0062B1AD14B881B0A212B03D12B
:10AFD800CA883A2A28BF3A220E49304600F0EAFACF
:10AFE80000250CE00C49012200F0E4FA07E08B7818
:10AFF8001BB9074A1D46936101E000F053FB284640
:10B0080070BD00BF80020020BF2D00200402002078
:10B018008C0D002016020020A40D002010B58121FF
:10B028000446FFF71AFC01212046FFF716FC82218F
:10B038002046FFF712FC024B5B689847002010BDC2
:10B048008002002038B5D0F8EC350446B3F8392032
:10B0580081210223FFF7E0FBD4F8EC350121B3F896
:10B06800402020460223FFF7D7FB82210822032332
:10B078002046FFF7D1FB094B022200251A715D71AA
:10B08800074B1B689847D4F8EC35064AB3F84030AC
:10B0980020460121FFF7FAFB284638BDC4020020EC
:10B0A800800200207F2D002010B5074C606CFF281F
:10B0B80007D0064B064A9B68064952699847FF2302
:10B0C8006364002010BD00BF04020020800200203D
:10B0D8008C0D0020BF2D002038B510490B79012BAD
:10B0E80019D10C690CB90C7115E0D0F8EC358D68E4
:10B0F800B3F839309C42AAB203D95D198D60E41ABD
:10B1080003E0A3B22C198C6000240C610449521886
:10B118008121FFF7D6FB002038BD00BF8C0D002031
:10B12800C72D002000207047002070470023F0B58D
:10B13800084A094E1D4609E01468C75C37550134B2
:10B148000133B4F5006F146008BF15608B42F3D16A
:10B158000020F0BD980D0020C72D0020104B114A8B
:10B16800D3F800C000232DE9F0410F4F16461D46C5
:10B178000DE0146810F8038007F804800134802C6F
:10B1880008BF2C4614603468644505D001338B42EF
:10B19800EFD10020BDE8F0810220BDE8F08100BFBA
:10B1A800483600205C360020C835002021280FD101
:10B1B800084B1A680A701A68120A4A705A888A7004
:10B1C800DA78CA701A790A715A794A719B798B713F
:10B1D800002070477802002007B502AB012103F870
:10B1E800010D1846FFF7A2FF0EBD002100E0013156
:10B1F800435C002BFBD199E798E70B4B0B491A6886
:10B20800096891420BD00A498A5C02701A680132B7
:10B21800802A1A6005D100221A6001207047002098
:10B2280070470120704700BF483600205C36002078
:10B23800C8350020204B1A68204B1B689A42F0B58D
:10B2480009D135E00133802B08BF00239A4203D18E
:10B258001A4B1A602CE01A4CE15C0029F2D00A293A
:10B26800F0D00D29EED0154C1549134D23600E462C
:10B278000023CF182268BA5CC254226801339F1891
:10B28800802F08BF53422F689A18974210D0B25C9B
:10B298001AB10A2A01D00D2AEBD10022C254074A5A
:10B2A800116859187F29116003D98039116000E0AD
:10B2B80000231846F0BD00BF5C3600204836002049
:10B2C800C8350020704700BFD0F8E43510B51B69B9
:10B2D80004469847032384F81231002010BD08B5AE
:10B2E800042380F81231D0F8E435DB689847002051
:10B2F80008BD08B5D0F8E035DB6903B198470020F0
:10B3080008BD08B5D0F8E0351B6A9847002008BD8D
:10B3180008B5D0F8E0355B6A9847002008BD0021E1
:10B3280010B5402204460B46FFF776FA80214022EA
:10B3380000232046FFF770FA012384F81231D4F86D
:10B34800E435A0785B689847002010BD13B56946BE
:10B35800044600F085F99DF8001001F01F03012B49
:10B3680007D0022B0AD073B92046694600F026FAA6
:10B378000FE02046694600F007FA0AE020466946D1
:10B3880000F0A2F905E021F07F01C9B22046FFF7DD
:10B39800B1FA00201CBD38B5044600293DD190F80B
:10B3A8001131022B42D1D0F83421D0F820319A4201
:10B3B80011D9C178D21A0129C0F8342104D1D0F8A2
:10B3C8002411CB18C0F8243192B22046D4F82411A5
:10B3D80000F000F92AE0D0F83821B2FBF3F503FBBE
:10B3E800152565B99A420AD3D0F83C319A4206D25B
:10B3F80029462A4600F0EEF8C4F83C5116E0D4F885
:10B40800E035DB682BB194F81221032A01D12046DC
:10B418009847204600F00FF908E0D0F8E0355B695E
:10B4280023B190F81221032A00D19847002038BD93
:10B4380010B5044659BB90F81131032B30D1D0F820
:10B448008C23D0F878339A4214D9C178D21A0129BA
:10B45800C0F88C2304D1D0F87C13C918C0F87C1329
:10B468009A4228BF1A4692B22046D4F87C1300F0BC
:10B47800CAF815E0D0F8E0351B6923B190F812211D
:10B48800032A00D19847204600F0C6F808E0D0F813
:10B49800E0359B6923B190F81221032A00D198471F
:10B4A800002010BD2DE9F041069F04461646984637
:10B4B8000D46FEF741FC20462946C4F8E085C4F84D
:10B4C800E475C4F8E865FFF761F9D4F8E4351B685A
:10B4D80098472046BDE8F041FEF782BC002070473F
:10B4E800D0F8E03510B504461B689847D4F8E43521
:10B4F8009B689847002010BD08B5D0F8E0355B6818
:10B508009847002008BD000012230B8000487047B0
:10B51800C402002004230B8000487047D602002094
:10B5280010B5044C04480A46214600F075FA204636
:10B5380010BD00BF6036002068B605080A4608B589
:10B548000248034900F068FA014808BD7BB60508BF
:10B55800603600200A4608B50248034900F05CFA44
:10B56800014808BD89B605086036002008B50A46B6
:10B5780008B9044800E00448044900F04DFA0348BB
:10B5880008BD00BF94B60508A1B6050860360020BE
:10B5980008B50A4608B9044800E00448044900F020
:10B5A8003BFA034808BD00BFAEB60508CFB605088C
:10B5B8006036002010B513460C46C0F83821C0F894
:10B5C8003421022280F8112100212246FFF779F95F
:10B5D800002010BD10B50C46134600212246FFF787
:10B5E80070F9002010BD10B513460C46C0F8902322
:10B5F800C0F88C23032280F8112100212246FFF78E
:10B6080045F9002010BD10B50C461346002122460E
:10B61800FFF73CF9002010BD0021042310B50A46AD
:10B62800044680F811310B46FFF74BF92046FEF728
:10B63800D7FF002010BD0021052310B50A46044697
:10B6480080F811310B46FFF721F92046FEF7C8FFB5
:10B65800002010BD282303FB0100B0F888037047C1
:10B6680090F8C8350B7090F8C9354B7090F8CB2519
:10B6780090F8CA3503EB02234B8090F8CD2590F85B
:10B68800CC3503EB02238B8090F8CF2590F8CE358C
:10B6980003EB02239BB2CB80C0F83C31012380F836
:10B6A8001131704710B591F90030002B044601DBC9
:10B6B800CB880BB9802100E00021FFF71BF9204659
:10B6C800BDE81040FEF78CBF38B50D4604466B78D0
:10B6D8000979012B10D027D3032B51D190F81231BF
:10B6E800022B28D0032B47D16B889BB991B18029B5
:10B6F80010D0FFF7FFF80DE090F81231022B1AD0A6
:10B70800032B39D16B88002B3AD149B1802907D056
:10B71800FFF70EF9D4F8E03520469B68294698478C
:10B728002046FFF779FF2BE090F81231022B02D068
:10B73800032B21D106E019B3802921D02046FFF739
:10B74800D9F81DE011F0800F4FF0280306D001F062
:10B758007F0103FB010393F81A2103E003FB0101B6
:10B7680091F87223074B02B101221A60204605495D
:10B778000222FFF71FFF03E020462946FFF792FF4A
:10B78800002038BDA80D002038B590F81231032BE1
:10B7980004460D460CD10B79012B09D8D0F8E035B9
:10B7A8009B689847EB883BB92046FFF735FF03E0D5
:10B7B80020462946FFF776FF002038BD73B54B7841
:10B7C80004460D46092B00F21C81DFE813F0D10076
:10B7D80008011A01E4001A0172000A001A01C000E7
:10B7E80092004B881A0A013A062A00F20A81DFE819
:10B7F80012F007001A0027000801080108010801D3
:10B80800D4F8E835A0781B680DF106019847EB8855
:10B81800402B014603D094F81231012B3AD108236A
:10B82800ADF8063036E0D4F8E035A0789B6A0DF123
:10B8380006019847022343700146C4F8EC0529E045
:10B84800DBB2052B00F2DD80DFE803F003080D1200
:10B85800171CD4F8E835A0785B6817E0D4F8E83509
:10B86800A0789B6812E0D4F8E835A078DB680DE092
:10B87800D4F8E835A0781B6908E0D4F8E835A07852
:10B888005B6903E0D4F8E835A0789B690DF10601FF
:10B8980098470146BDF80630002B00F0B680EA88CC
:10B8A800002A00F0B2809A4228BF1A46ADF8062056
:10B8B8005CE08B88002B40F0A480CB88002B40F004
:10B8C800A08094F812214B88032A00F09A8003F094
:10B8D8007F05204684F813512946FFF753F8204680
:10B8E800FFF79AFE0DB1022300E0012384F812311C
:10B8F8008BE08978464E0129317100F2828094F8F4
:10B908001231022B02D0032B7BD108E0002962D030
:10B918000121032384F8101184F8123113E041B98E
:10B92800022384F8123184F810112046FFF7E4FD51
:10B9380051E094F81011012920464DD0FFF7DCFDA5
:10B94800317984F810112046FFF7CAFD43E0CA8810
:10B95800012A56D194F81231022B02D0032B50D170
:10B9680002E020462B4913E004F5887120460FE0D9
:10B9780094F81231023B012B43D8D4F814312449EE
:10B98800002B0CBF0123032341F80C3F2046012262
:10B99800FFF710FE39E04B88012B29D0022B34D158
:10B9A8008B8813F0FF0F30D121691B0A013B4A68CD
:10B9B800042B0FD8DFE803F0030507090B00012368
:10B9C80006E0022304E0032302E0042300E0052349
:10B9D80063F306124A602046FFF71EFE15E094F84E
:10B9E8001231023B012B0CD84B88012B0DD10023BF
:10B9F800C4F81431D4F8E03520469B6829469847A6
:10BA0800E9E720462946FFF74DFE00207CBD00BF30
:10BA1800A80D0020B00D002030B5C8B10023DDB25C
:10BA28000133C41814F8014C002CF8D16B1C5B00CE
:10BA380013800B7003234B70022305E0CA545A1C71
:10BA4800D2B202338C54DBB210F8012B002AF5D1A4
:10BA580030BD00BF704770477047704770477047E8
:10BA6800704700000000000008B5FCF701FA094B18
:10BA78005A78187002435A701AB19A7801329A703B
:10BA880030B99B78034A012B02D900235370937075
:10BA980008BD00BFB80D00202DE9F84F3F4B1B78BB
:10BAA800012B2DED028B09D002D3022B0FD108E018
:10BAB8003B4B1A68802392FBF3F206E0384B1A6876
:10BAC80003E0374B1B6803225A43364B5A61364B07
:10BAD8001A8892B2002AFBD0334B00221A80FDF755
:10BAE8005DFD10EE105AFDF75FFD284610EE104A76
:10BAF80006F0CAFE80462046894606F0C5FE41EC9F
:10BB0800100B41EC180B08F0CBFF57EC106BB0EEA4
:10BB1800480AF0EE680A09F0C3F832463B46404648
:10BB280049465BEC10AB06F003FF07F0E3F99FED25
:10BB38001F8A07EE100ADFED1E7A57EE087A194CB5
:10BB480052465B46C4ED007A4046494606F0F0FE90
:10BB580007F0D0F907EE900A27EE888A84ED018A6B
:10BB6800FDF734FD84ED020AFDF736FD84ED030A86
:10BB7800FCF78CF80F4B62691B68D31A0E4A07EE64
:10BB8800100A1268F8EEC77A93FBF2F3C4ED047A50
:10BB98002383BDEC028BBDE8F88F00BF1C0E00208C
:10BBA800E82C00209C380020680D00200000F0429E
:10BBB80000008C42E42600206826002007B50420F7
:10BBC800012105F0AFFA4FF46043009301238DF88B
:10BBD800043002238DF805300448002369468DF8A7
:10BBE80006308DF8073004F0F5FE0EBD000802405F
:10BBF800084B1A684FF47A73B2FBF3F2064B013A1A
:10BC08005A60064AF02182F8231000229A6007221F
:10BC18001A607047E401002010E000E000ED00E049
:10BC2800034B5A6812B15A68013A5A60704700BF0C
:10BC3800B80D0020024B58605A68002AFCD17047A2
:10BC4800B80D002030B585B004460D4601A86749F7
:10BC58000A220BF01DFC664B1B78032B10D8DFE87B
:10BC680003F00205080B01A8624907E001A8624930
:10BC780004E001A8614901E0614901A80BF0F2FC68
:10BC880004AA131913F80C3C5D19EDB22F2D01D835
:10BC98000A3502E0392D01D90A3DEDB204AB1C1971
:10BCA8004FF6FF7004F80C5CFAF76EFA0020FAF70A
:10BCB8006DFB0DF103050F24204623345A21002380
:10BCC80015F8012FA4B2FAF77BFBB4F5A57FF3D1E1
:10BCD80064205A212C220023FAF772FB0023CD207E
:10BCE8005A212C22FAF76CFB0020FAF74DFA404B48
:10BCF8001B78032B78D8DFE803F00233616C01A9C5
:10BD08003C480BF0AFFC0A2200213A480CF0D2FD67
:10BD18003C4A3D4B12781860012A0BD002D3022A04
:10BD28001AD10EE0B0F5FA5FBCBF4FF4FA521A60B0
:10BD3800364A0CE0364A904201DC01321A60354A34
:10BD480005E0354A904201DC01321A60334A1B682B
:10BD58009342C4BF2C4B1A60314B1A68314B2BE00D
:10BD680001A925480BF07EFC0A22002122480CF08C
:10BD7800A1FD244A2C4B12781860012A0BD002D35B
:10BD8800022A31D10EE0B0F5FA5FBCBF4FF4FA5287
:10BD98001A601E4A0CE01E4A904201DC01321A6009
:10BDA8001C4A05E01C4A904201DC01321A601B4A19
:10BDB8001B68934218DD1C4B1A6015E001A90F4857
:10BDC8000BF050FC0D4800210A220CF073FD174BB4
:10BDD80009E001A90A480BF045FC094800210A229C
:10BDE8000CF068FD124B186005B030BDF0B60508C0
:10BDF800E3260020B4260020D8260020EE2C0020C0
:10BE0800A02600201C0E0020F026002050DA110089
:10BE18001FA1070080D1F0085FE316008074D21AD2
:10BE2800E4260020E82C0020082D0020E42C002027
:10BE38009C26002010B50D4B0D4C1A680D48214664
:10BE48000BF0E8FB0C4B0D481A6821460BF0E2FB9F
:10BE58000B4B0C481A6821460BF0DCFB0A4B0B48CD
:10BE68001A682146BDE810400BF0D4BBF02600202C
:10BE7800B7AC0508B4260020082D0020D8260020DD
:10BE8800E42C0020EE2C00209C260020A026002078
:10BE98009FED010A704700BF000000009FED010AF6
:10BEA800704700BF000000009FED010A704700BF07
:10BEB8000000000018B1012801D1034B00E0034B3A
:10BEC8001868FDF7F7BC00BFD4260020E426002040
:10BED80010B9034B18687047024B1868704700BFC9
:10BEE800F0260020E426002010B9034B186870479C
:10BEF800024B1868704700BF082D0020D426002088
:10BF080008B54FF49570FBF7D5FE40F26523C31AC8
:10BF1800584240EB030008BD08B5C620FBF7CAFE2F
:10BF280040F28D13C21A504240EB020008BD4FF494
:10BF3800957040F26521FBF7AFBEC62040F28D1127
:10BF4800FBF7AABEDCE760EEA00AB7EE007AF0EED7
:10BF5800606A70EE077A40EE006A47EEA70A36EE8E
:10BF6800C77A08B5C7EE200A10EE900A06F08CFCD6
:10BF78000022084B06F0DCFC0022074B06F026FBEB
:10BF880006F0B8FF07EE900AFDEEE77A17EE900A82
:10BF98009F3008BD000059400000E03F38B52DED46
:10BFA800028BF7EE008AB0EE608A70EE288A10EEF7
:10BFB800900A28EE088A06F067FC08EEA88A002294
:10BFC8000F4B06F0B5FC044618EE100A0D4606F0B5
:10BFD8005BFC02460B462046294606F0D3FD0022AC
:10BFE800084B06F0F3FA06F085FF07EE900AFDEE1F
:10BFF800E77A17EE900A7730BDEC028B38BD00BFA8
:10C00800000069400000E03F2DE9F04F884F2DED1A
:10C01800068B97E80F0091B00CAC103784E80F003E
:10C028000FCF05AE0FC697E807004FF6FF7386E8F7
:10C0380007009F2077216422F7F76FFDA020772162
:10C0480064224FF6FF73F7F768FD9E20772164227C
:10C058004FF6FF73F7F761FD9F20762164224FF6B4
:10C06800FF73F7F75AFD4FF6FF73782164229F207C
:10C07800F7F753FD0020F9F764F99F20772165222F
:10C08800FAF7C4F80C349F2077216422FAF7BEF837
:10C098000DF12C0A0394F7EE009A4FF00F0B00E015
:10C0A8004D460AF1040AF7EE008A9AED009A002438
:10C0B800B0EE68AA01E0B846354618EE900A06F0D8
:10C0C800E3FB59A3D3E9002306F032FC06F012FF84
:10C0D80008EE900A38EEE98AB0EE490AF0EE480A0E
:10C0E800FFF731FFB0EE490AF0EE480A0646FFF7BF
:10C0F80055FFB2B2074683B22CB9104619460F2233
:10C10800F9F7DEF906E0A8B21FFA88F1CDF800B019
:10C11800F9F7C6FF0134B4F5967FCCD13D46F7EE6A
:10C12800008A002401E045464E4618EE900A06F0C3
:10C13800ABFB3DA3D3E9002306F0FAFB06F0DAFED9
:10C1480008EE900A39EEE88AB0EE490AF0EE480A9D
:10C15800FFF7F9FEB0EE490AF0EE480A8146FFF70C
:10C168001DFF1FFA89F2804683B22CB91046194682
:10C178000F22F9F7A5F905E0B0B2A9B2CDF800B0E1
:10C18800F9F78EFF0134B4F5967FCCD1039B9A451D
:10C1980086D104AD0DF12C0B4FF0000A01E0B84632
:10C1A800B146043595ED009AF7EE008A002401E0C7
:10C1B800B846B14618EE900A06F066FB1AA3D3E912
:10C1C800002306F0B5FB06F095FE08EE900A38EE5F
:10C1D800CA8AF0EE490AB0EE480AFFF7B4FEB0EE9C
:10C1E800480AF0EE490A0646FFF7D8FEB2B20746FB
:10C1F80083B22CB9104619462246F9F761F907E0CF
:10C208001FFA89F01FFA88F1CDF800A0F9F748FF66
:10C218000134B4F5C87FCBD15D45C0D111B0BDECB8
:10C22800068BBDE8F08F00BF295C8FC2F528F03F70
:10C2380054B10408121A06EE902A081AB8EEE67AE3
:10C2480006EE900AF8EEE67A08B5C7EE277A17EEFA
:10C25800900A06F019FB0022044B06F069FB002245
:10C26800034B06F0B3F906F0FDFD08BD000074406D
:10C278000000E03F8A1A06EE902A081AB8EEE67A1D
:10C2880006EE900AF8EEE67A08B5C7EE277A17EEBA
:10C29800900A06F0F9FA0022044B06F049FB002246
:10C2A800034B06F093F906F0DDFD08BD0000694078
:10C2B8000000E03F70B506460D460024610704D52E
:10C2C800A0B231462A46F9F7FBF80134B4F5A07F4D
:10C2D800F4D170BD70B506460D460024600704D53C
:10C2E800A1B230462A46F9F7EBF80134C82CF5D14B
:10C2F80070BD234B1B78012B03D011D3022B3DD1EA
:10C3080023E0204B1A68204B1A60204B1A68204BF8
:10C318001A60204B1A68204B1A60204B1A6811E0EB
:10C32800184B1A68184BD2011A60184B1A68184B28
:10C33800D2011A60174B1A68174BD2011A60174BB3
:10C348001A68D201164B1A6070470E4B0E4A1968CC
:10C35800032391FBF3F111600C4A11680C4A91FB1D
:10C36800F3F111600B4A11680B4A91FBF3F111606C
:10C378000A4A126892FBF3F3094A1360704700BF38
:10C388001C0E0020F0260020E4260020082D0020A6
:10C39800D4260020E42C002068260020C026002097
:10C3A800002D0020014B1868FDF784BAE426002010
:10C3B80008B5FFF79EFFBDE80840F3E770B5002118
:10C3C8000A222748274D284E284C0CF073FA0021E2
:10C3D8000A22286026480CF06DFA00210A223060F3
:10C3E80024480CF067FA00210A22206022480CF049
:10C3F80061FA224B326818602B682149D31A06EE7D
:10C40800903A2368B8EEE67A06EE903AF8EEE67AC5
:10C41800C7EE277AFCEEE77A17EE903A9AB20B80CD
:10C42800531C07EE903AB8EEE77ADFED167A67EE1E
:10C43800277A154BFCEEE76A16EE901A8AB206EEDA
:10C44800902AB8EEE67A198077EEC77AF5EEC07AC8
:10C45800F1EE10FA01DD01321A80BDE87040A7E75D
:10C46800B4260020F0260020082D0020E42C00200F
:10C47800D8260020EE2C0020A02600209C26002094
:10C48800DC3A00200000803D703B00200022F0B51F
:10C498001346202603254FF02C0C00E02646303E9C
:10C4A800F6B217460132092E10F8014B0AD897FB4D
:10C4B800F5F605FB16772FB9CE1801F803C074708E
:10C4C800023301E0CC540133092AE7D12022CA54AF
:10C4D800CB1848225A707A229A700022DA70F0BD7E
:10C4E800F0B51F46144B1E78012E8DB005460C463C
:10C4F80020D0A6F1030CDCF1000646EB0C06CEB901
:10C508000E4908A80BF086F808A86946FFF7BEFF91
:10C518000B496A4604A80BF07DF8BDF84800F9F706
:10C5280033FE3846F9F746FE2846214604AA334624
:10C53800F9F764FF0DB0F0BD71260020B7AC05080F
:10C5480034B4050810B501210446F8F7DFFF014BA4
:10C558001C8110BDB80D002008B50021C620FBF7CE
:10C568009BFB4FF495700021BDE80840FBF794BB96
:10C57800014B9F221A817047B80D00200020014608
:10C58800C82240F23F13F8F7D1BF07B50DF10700F5
:10C59800FEF733FE9DF807000EBD08B5FFF7F5FF5F
:10C5A8000028FBD108BD30B5044687B010EE100A4C
:10C5B8000D4606F069F902460B4601A805490BF03D
:10C5C80029F82046294601AA0023F9F717FF07B0E2
:10C5D80030BD00BFFAB6050808B5084803F05CFC92
:10C5E8000648022103F029FD0028F9D0034803F08A
:10C5F8007FFC07EE900AB8EE670A08BD00200140EC
:10C6080010B52DED028B9FED098A1924FFF7E4FF81
:10C61800013CE4B238EE008A002CF7D19FED040A01
:10C6280028EE000ABDEC028B10BD00BF0000000020
:10C63800ACC868392DE9F04F994B9A4C5D695E6832
:10C648002DED068B93ED00AAC7B007461AEE100A27
:10C6580093ED038AD3ED04AAD3ED028A93ED069AEB
:10C6680006F012F941EC100BCDE9040108F0FCFBCF
:10C678003A468D493BA88DED0C0B0AF0CBFFA0681C
:10C6880006F002F902460B462BA888490AF0C2FFB9
:10C69800E06806F0F9F802460B462FA884490AF02C
:10C6A800B9FF1AEE900A06F0EFF8CDE90A01DDE9C4
:10C6B8000A23804933A80AF0ADFF284606F0E4F8BB
:10C6C800CDE90601DDE906237B4937A80AF0A2FF78
:10C6D80018EE900A06F0D8F88046894642464B463E
:10C6E800764913A80AF096FF18EE100A06F0CCF85F
:10C6F80082468B46524672495B4617A80AF08AFF63
:10C70800DDE904236F491BA80AF084FF304606F0D0
:10C71800BBF85BA3D3E90023CDE9080106F008F9CB
:10C7280002460B461FA868490AF074FF49EC118BB2
:10C738004BEC10AB08F010FB51A3D3E9002351ECEC
:10C74800100B06F0F5F802460B4627A85F490AF0D9
:10C7580061FF19EE100A06F097F80B4602465C498D
:10C7680023A80AF057FFD4ED047AFDEEE77A594979
:10C7780017EE902A0FA80AF04DFF0022564BDDE96C
:10C788000C0106F0D5F806F0B5FB06F07DF8024678
:10C798000B4643A851490AF03DFFB5EEC08AF1EEB9
:10C7A80010FADFED4F9A37D5384606F05BF836A316
:10C7B800D3E9002306F0BCF8F1EE487A044617EEF8
:10C7C800900A0D4606F060F802460B4620462946B8
:10C7D80006F0AEF802460B462DA1D1E9000106F09D
:10C7E800D1F906F087FB9FED3F7A07EE900AF4EE49
:10C7F800C77AF1EE10FAC6BFC7EEA97A3A4C3B4C9D
:10C80800F4EEE97AF1EE10FA38DD9FED357A384D1D
:10C81800384CC7EE877A78E01FA3D3E90023504647
:10C82800594606F085F8044638460D4606F01AF8CB
:10C8380015A3D3E9002306F07BF802460B462046F1
:10C84800294606F09FF906F055FB07EE900AB7EE69
:10C85800007AF4EEC77AF1EE10FA46BF67EEA97ACD
:10C86800254C264CF4EEE97AF1EE10FA4CDD9FEDFA
:10C878001C7A234D234CC7EE877A46E01C4D44E0D2
:10C888006666666666A64C401F85EB51B81E194061
:10C89800000000A2941A6D420000000080842E411E
:10C8A8008C3A00209C3800201CB7050826B70508DC
:10C8B80031B705083CB7050846B7050850B705085D
:10C8C8005BB7050866B7050871B705087CB70508A2
:10C8D80087B7050893B70508000034C0A0B7050856
:10C8E80000007A44002474490BB7050808B7050806
:10C8F800ACB6050814B7050811B705080EB7050842
:10C9080017B7050819B705088B4D17EE900A05F0FB
:10C91800BBFF2A46CDE90001884902943FA80AF0E6
:10C9280079FE874B874D1868874B19688F42CCBFB3
:10C93800002301238742D8BF0023EB60834B1B7879
:10C948000D2B2ED13A46FFF775FC814B0646186829
:10C9580005F09AFF00227F4B05F0EAFF02460B46DE
:10C9680000207D4905F030FE06F07CFA4FF6E073B2
:10C978000093044600230520DC213A46FFF7B0FD6A
:10C98800EB6853B1754B1888754B4FF4FC651988E3
:10C998000095B2B2A3B2F9F783FB704B1E60704BDF
:10C9A8001C606A4B1B78082B40F0AE800220F9F718
:10C9B800EDFC4FF6FF70F9F7FDFB1F20F9F7E4FBDC
:10C9C80019210023674A2D20F9F718FD4FF6FF704B
:10C9D800F9F7F0FB00200024F9F7D6FB0F20B4216B
:10C9E8003A464FF6FF730094FFF77AFD0F206E2149
:10C9F80023462BAAF9F702FDB0206E2123462FAA61
:10CA0800F9F7FCFC0F20382123461BAAF9F7F6FC9E
:10CA1800B020382123461FAAF9F7F0FC0F205C212B
:10CA2800234633AAF9F7EAFC2346B0205C2137AA4B
:10CA3800F9F7E4FC0F204A21234613AAF9F7DEFC94
:10CA4800B0204A21234617AAF9F7D8FC0F209B21CA
:10CA5800234623AAF9F7D2FC0F20842123463FAAB4
:10CA6800F9F7CCFCB0208421234627AAF9F7C6FCA5
:10CA7800B0209B2143AA2346F9F7C0FC3A4B1B6818
:10CA8800B3F57A7FCCBF4FF4FC604FF47840F9F7E8
:10CA980091FB0023A020B4210FAAF9F7AFFC334B78
:10CAA8001C78012C0CD002D3022C1DD111E04FF6BA
:10CAB800E070F9F77FFB4FF48C7002212C4A10E0EC
:10CAC8004FF4FC60F9F776FB4FF48C700221294A89
:10CAD80007E04FF6E070F9F76DFB274A4FF48C70CA
:10CAE80021460023F9F78AFC0020F9F763FB4FF48D
:10CAF800FC60F9F749FBFFF783FD0F20DC21FFF706
:10CB080052FD1F20F9F756FB104B1B789A1FD2B223
:10CB1800012A02D90B2B40F05C82184B1B78023B90
:10CB2800052B00F25682DFE813F02D007D00EE00A1
:10CB38004701EF01640100BF17B70508AEB7050844
:10CB4800F0260020B80D0020082D002071260020B6
:10CB5800C03600200000044000003940D8380020CA
:10CB68007C3B0020BBB70508181B00201C0E0020CA
:10CB780015B605081AB605081EB60508FC2C0020CF
:10CB88000000C8425FED027A2AEE27AA1AEE100AC0
:10CB980005F07AFE9DED080B8046894607F080FF78
:10CBA800404653EC102B494605F0C2FED2A3D3E908
:10CBB800002305F00BFD06F055F99DED080B044622
:10CBC80008F06EF8404653EC102B494605F0B0FECD
:10CBD80002460B46CAA1D1E9000105F0F5FC06F0B2
:10CBE80041F94FF6E0730093054600230520DC2148
:10CBF8003A46FFF775FCB44BDB6853B1B34B188862
:10CC0800B34B4FF4784619880096A2B2ABB2F9F745
:10CC180047FAAE4B1C60AE4B4FF6E0701D60F9F75B
:10CC2800B3FAD6E1AB4B1868AB4B3A461968FFF735
:10CC380001FBAA4B1B784FF4FA7292FBF3F307EE51
:10CC4800903AB8EEE79ADFEDA67AF4EE498AF1EE6B
:10CC580010FAC8BFF0EE498AF5EE408AF1EE10FAF4
:10CC680048BFF0EE678AF4EEC98AF1EE10FA04467E
:10CC780020D8F4EEE78AF1EE10FA1BDBFDEEC97A54
:10CC8800FDEEE88A17EE901A18EE902A0020FFF7BA
:10CC9800F1FA8D4BDB68054653B18C4B18888C4BE9
:10CCA8004FF6FF7619880096A2B2ABB2F9F7F8F9F9
:10CCB800874B1D60B4EE498AF1EE10FAC8BFB0EE9A
:10CCC800498AF1EE497AB4EE678AF1EE10FA48BF64
:10CCD800B0EE678AB4EEC98AF1EE10FA00F27981F3
:10CCE800B4EEE78AF1EE10FAC0F27381FDEEE77A4E
:10CCF800BDEEC99ABDEEC88A17EE900A19EE101A51
:10CD080018EE102AAEE0734B1868734B3A46196850
:10CD1800FFF790FAF5EEC0AAF1EE10FA044627DD07
:10CD2800DDE90A015AA3D3E9002306F073F8F8B144
:10CD380059A3D3E90023DDE90A0105F0F9FD0B4603
:10CD480002466849002005F03FFC06F08BF85E4B70
:10CD5800DB68054653B15D4B18885D4B4FF6FF768F
:10CD680019880096A2B2ABB2F9F79AF9584B1D6030
:10CD7800DDE906014AA3D3E9002306F069F8002893
:10CD880000F02781DDE9060141A3D3E9002306F07D
:10CD980041F8002800F01D8143A3D3E90023DDE911
:10CDA800060105F0C5FD02460B4600204E4905F078
:10CDB8000BFC06F057F857E0464B1868464B3A46C6
:10CDC8001968FFF737FA3AA3D3E900230446DDE9E7
:10CDD800040106F03DF850B19DED040B08F044F84D
:10CDE800002251EC100B414B05F0A2FDDCE0C825F8
:10CDF800DDE031A3D3E90023DDE9080105F098FD62
:10CE08002FA3D3E9002305F0BDFE06F073F8314BDC
:10CE180008EE100A1868304B3A461968FFF70AFA04
:10CE2800DFED337A4AEE677A274BFDEEE77ADB6867
:10CE380017EE905A044625EAE57553B1234B188836
:10CE4800234B4FF6FF7619880096A2B2ABB2F9F7DA
:10CE580027F9BDEEC88A1E4B18EE102A1D606FF028
:10CE6800B300B421FFF706FA174BDB68054653B148
:10CE7800164B18881F4B4FF4FC6619880096A2B20F
:10CE8800ABB2F9F70DF91B4BA0E000BFAFF3008080
:10CE98009A9999999999B93F0000000000409F40DC
:10CEA8009A9999999999B9BF0000000000408F405C
:10CEB80089B5F81400E3693F00000000008076405F
:10CEC8001F85EB51B81E1940B80D0020D838002036
:10CED8007C3B0020F0260020082D00201C030020A9
:10CEE800000000000000694000005940000054C0E4
:10CEF80000004843C83600200000000000E06340FE
:10CF08000000000000C05D403B4B187805F0AAFC0B
:10CF180002460B460020394905F034FE05F0EAFFC9
:10CF280008EE100A05F0B0FC41EC100B07F09CFF6E
:10CF3800B4EE489AF1EE10FAC8BFB0EE489AB4EED3
:10CF4800C89AF1EE10FA5BEC10AB42D82C4B18687B
:10CF58002C4B3A461968FFF76DF9044619EE100A8A
:10CF680005F092FC41EC100B07F07EFF5946504645
:10CF780059EC108B05F0BEFF9FED237A07EE900A5F
:10CF8800C7EE277A17EE900A05F07EFC42464B461C
:10CF980005F0CEFC02460B4600201C4905F014FBA8
:10CFA80000221B4B05F012FB05F05CFF0546194BF0
:10CFB800DB6853B1184B1888184B4FF6FF76198861
:10CFC8000096A2B2ABB2F9F76BF8144B1D60124B86
:10CFD8001C60134B1B78022B09D043B14FF6FF732B
:10CFE80000930520DC213A460023FFF779FA47B081
:10CFF800BDEC068BBDE8F08F1C03002000005940F3
:10D00800F0260020082D0020000048430000694059
:10D018000000E03FB80D0020D83800207C3B0020FD
:10D02800FC2C002010B54FF4C770FAF743FEDB283C
:10D0380005D14FF4C870FAF73DFE84B219E041F209
:10D04800E104214644F20100FAF726FE44F2010009
:10D05800FAF730FEA04214BF80244FF4007421B2C6
:10D068004FF4C870FAF718FE4FF4C770DB21FAF7CF
:10D0780013FE204610BD024B00221A60704700BF05
:10D08800E436002070EEA10A88B030EE010A08B03C
:10D09800704770EEE10A88B030EE410A08B0704778
:10D0A800F0EE407A20EEA10A60EE810A47EEA10A6E
:10D0B80088B017EE810A08B07047D0B561EEA17A42
:10D0C80041EE017A2DED048B17EE900A88B0B0EE90
:10D0D800409AF0EE609AF0EE418AB0EE618A05F06F
:10D0E800D3FB0022002306460F4605F089FEE8B967
:10D0F80069EE887A49EE287A29EE088A17EE900AAE
:10D1080005F0C2FB32463B4605F03CFD19EEA88A05
:10D1180005F0F0FE044618EE100A05F0B5FB32469D
:10D128003B4605F02FFD05F0E5FE01E00448044606
:10D1380000EE900A00EE104A08B0BDEC048BD0BD9A
:10D148000050C347F0B58E4B2DED068B93ED001ABA
:10D15800D3ED011A8FB0F0EE408AB0EE608A8DED03
:10D16800060ACDED070A30EE410A70EEE10A38EE04
:10D17800811A78EE211A8DED0C1ACDED0D1A8DED70
:10D188000A0ACDED0B0AFFF798FF8DED040ACDEDE5
:10D19800050A04AA92E8030008AB83E80300DDED62
:10D1A800099A9DED08AA69EEA97A4AEE0A7A17EE5D
:10D1B800900A05F069FB41EC100B07F0DBFE51EC1F
:10D1C800100B05F097FE09EE100A19EE900A05F00B
:10D1D8005BFB04461AEE100A0D4605F055FB45ECBC
:10D1E800104B41EC110B07F0B7FD51EC100B05F09B
:10D1F80081FE68EE087A48EEA87AB1EE48AAC8EE31
:10D20800A79A604B604D5A691B8B6860EA612B8452
:10D2180004468AEE27AA85ED009A19EE100AC5ED94
:10D22800028A85ED038AC5ED049A85ED05AA05F005
:10D238002BFB4DA3D3E9002305F00AFEDFED537A5B
:10D24800002818BFB0EE679AB7EE007A79EE077A31
:10D2580037EE497A4E4BC7EE877A1B78033BC5ED0C
:10D26800067A042B71D8DFE803F0032738664F00ED
:10D2780018EE100A05F008FB044618EE900A0D4651
:10D2880005F002FB06460F4647EC116B45EC104BC8
:10D2980007F062FD36A3D3E9002351EC100BCDE96A
:10D2A800004505F045FB3246CDE902013B463949C8
:10D2B80039480AF0AFF948E019EE900A05F0E4FAA7
:10D2C80004461AEE100A0D4605F0DEFA2246CDE9AC
:10D2D80000012B46304831492AE019EE100A05F0C2
:10D2E800D3FA41EC100B07F0BFFD00222C4B51EC98
:10D2F800100B05F01DFB05F0FDFD05F0C5FA024613
:10D308000B46254827491EE019EE100A05F0BCFA1D
:10D31800064620460F4605F0B7FA17A3D3E90023BF
:10D3280005F006FBCDE900011B481F4932463B4684
:10D338000AF070F909E017EE900A05F0A5FA02461E
:10D348000B46154819490AF065F9134C00230220C9
:10D35800CA212246F9F752F8002323700FB0BDEC1A
:10D36800068BF0BDAFF30080AE47E17A14AEEF3F15
:10D378006666666666A64C40F6285C8FC2A54C4079
:10D388000C3700209C3800208C3A0020A4707D3F88
:10D39800FC2C0020DAB70508A0360020F4B70508F1
:10D3A800000034C004B8050816B8050832B80508E6
:10D3B80000B560EEA07A40EE007A2DED028B17EEF4
:10D3C800900A87B0B0EE408AF0EE608A8DED020ACE
:10D3D800CDED030A05F058FA41EC100B07F0CAFD31
:10D3E80051EC100B05F086FDDFED117A07EE100AFF
:10D3F80078EEA78A38EE078A68EEA87A48EE087AA7
:10D40800C7EE277A17EE900A05F03EFA41EC100BAA
:10D4180007F0B0FD51EC100B05F06CFD00EE900A22
:10D4280020EE880A60EEA80A07B0BDEC028B00BDAA
:10D4380000000000F0B52DED028BDFED3A1A3A4BF3
:10D448008DB030EEA17AF0EE407AB7EE001A8DED8D
:10D45800020A83ED001A30EE010AC3ED011A31EE1B
:10D46800671A71EEE01ACDED030AF0EE470A8DED6A
:10D47800077A8DED081ACDED091A8DED060AFFF72A
:10D488001CFE8DED000ACDED010A9DE8030004ABFA
:10D4980083E803009DED058ADDED048A68EE087ACD
:10D4A80048EEA87A17EE900A05F0EEF941EC100B59
:10D4B80007F060FD18EE100A57EC106B05F0E4F960
:10D4C800044618EE900A0D4605F0DEF945EC104BBF
:10D4D80041EC110B07F040FC3946304655EC104B37
:10D4E80005F008FD05F0D0F941EC100B07F036FC0B
:10D4F800002251EC100B0D4B05F01AFA05F0FAFC5E
:10D5080029460646204605F0F5FC00EE900AF6EEA0
:10D51800007A60EEA70A00EE106A0DB0BDEC028B2F
:10D52800F0BD00BF00000000E43A00200000E03F2A
:10D53800F0EE407A86B020EE200A67EE810A06B047
:10D5480070472DE9F04F2DED028B85B0FCF726F8DA
:10D5580010EE105AFCF728F8284610EE104A05F08D
:10D5680093F980462046894605F08EF941EC100B68
:10D5780041EC180B07F094FA57EC106BB0EE480A20
:10D58800F0EE680A07F08CFB32463B4640464946B7
:10D598005BEC10AB05F0CCF905F0ACFC9FED138A01
:10D5A80007EE100ADFED127A57EE087A114C5B4647
:10D5B800C4ED007A52464046494605F0B9F905F0EF
:10D5C80099FC07EE900A27EE888A04AB84ED018A5D
:10D5D80094E8030003E90300DDED030A9DED020A68
:10D5E80005B0BDEC028BBDE8F08F00BF0000F04233
:10D5F80000008C42743B002030B53F4B2DED088B6A
:10D60800D3ED008AD3ED019A3C4BD3ED00AAD3EDBC
:10D6180001BA3B4B93ED008A93ED019A394B93ED98
:10D6280000AA93ED01BA38EEEA0A79EEEB0A38EE71
:10D638004A1A79EE4B1A93B08DED0A0ACDED0B0A12
:10D648008DED0C1ACDED0D1AFFF72AFD8DED000AB0
:10D65800CDED010A9DE803003AEE6A0A7BEE6B0AFB
:10D6680004AB38EE681A79EE691A83E803008DED89
:10D67800081ACDED091A8DED0E0ACDED0F0AFFF748
:10D688000FFD8DED000ACDED010A9DE8030006AB04
:10D6980083E803009DED040ADDED050A9DED061AF9
:10D6A800DDED071AFFF709FD8DED000ACDED010A42
:10D6B8009DE8030002AD85E80300134B9DED021AB7
:10D6C80093ED000AD3ED010ADDED031AFFF7E8FC3C
:10D6D8008DED000ACDED010A9DE8030012AB03E9C8
:10D6E80003006C46DDED110A85E803009DED100A84
:10D6F80013B0BDEC088B30BD98360020F8360020FA
:10D70800683B0020F83A0020C0380020F7EE007A85
:10D7180077EEC07A20EE022A20EE210A07EEA00A50
:10D72800F0EE420A47EE810A88B008B070472DE94A
:10D73800F0432DED028B924B1B78012B89B081466B
:10D74800884646D14FEAC00901291FFA89F92BD822
:10D7580009F58065A8B2FAF7F1FA8A4C0435A8B23F
:10D7680084ED000AFAF7EAFA09F58645A8B284EDCD
:10D77800010AFAF7E3FA844C043584ED000AA8B2EA
:10D78800FAF7DCFAA9F5FC4084ED010A80B2FAF751
:10D79800D5FA7E4CA9F5FA40FC3884ED000A80B22F
:10D7A800FAF7CCFA84ED010A08F1FF385FFA88F835
:10D7B800B8F1010F00F2DF80A9F57C5080B2FAF7CA
:10D7C800BDFA734CA9F57A5984ED000AA9F17C09D0
:10D7D800CBE0022B40F0CF806E4B6F4A1B680129CB
:10D7E80092ED007A00F2AC8007EE900AF8EE676AD4
:10D7F80007EE903A46EE877ABDEEE77A17EE104AC2
:10D80800A4B207EE104A04F18005ED00B8EE478A8D
:10D81800ADB2284637EEC88AFAF790FA0435A8B2AE
:10D8280004F50665EE008DED020AFAF787FAB6B23E
:10D8380030468DED030AFAF781FA043604F582576B
:10D84800B0B28DED040AFE00FAF778FAB6B23046A7
:10D858008DED050AFAF772FA0436B0B281348DED0F
:10D86800060AE400FAF76AFAA4B220468DED070A20
:10D87800FAF764FA434E0434A0B286ED000AFAF7C8
:10D888005DFA6C1CE400A4B2204686ED010AFAF7A2
:10D8980055FA3D4D0434A0B285ED000AFAF74EFA68
:10D8A8007C1CE400A4B2204685ED010AFAF746FA8A
:10D8B800364F0434A0B287ED000AFAF73FFAD6EDE6
:10D8C800001A96ED012ADDED020AF0EE408A87ED96
:10D8D800010A9DED031AB0EE480AFFF717FF8DED18
:10D8E800000ACDED010A9DE80300D5ED001A95ED7B
:10D8F800012AB0EE480ADDED040A86E803009DED32
:10D90800051AFFF703FF8DED000ACDED010A9DE82A
:10D918000300D7ED001A85E80300B0EE480ADDEDF4
:10D92800060A9DED071AB0EE682AFFF7EFFE8DEDA7
:10D93800000ACDED010A9DE8030087E803006C4664
:10D9480008F1FF385FFA88F8B8F1010F13D809F524
:10D95800C1594FEAC9091FFA89F94846FAF7EEF999
:10D968000B4C84ED000A09F104091FFA89F0FAF753
:10D97800E5F984ED010A09B0BDEC028BBDE8F0833E
:10D98800C9010020683B0020F8360020F83A002042
:10D99800983600206C260020AC2600202DE9F04F98
:10D9A8006E4B2DED048B1C78012CC7B0054605D0B5
:10D9B80006D3022C0CBF3024002402E0002400E02F
:10D9C80010244FF47670FAF775F907464FF475701E
:10D9D800FAF770F980464FF47470FAF793F9032D4B
:10D9E800C0B21D9040F094805D4A5E4924A809F0B9
:10D9F80011FEC1B224A8FDF7FFFB3B4642465A4937
:10DA080024A809F007FEC1B224A8FDF7F5FB574A80
:10DA1800544924A809F0FEFDC1B224A8FDF7ECFB87
:10DA280004F1C800FAF76EF9064604F1CC00FAF7DB
:10DA380069F9054604F1D000FAF764F9074604F1DC
:10DA4800D400FAF75FF9AB1B06EE903AB8EEE67A27
:10DA580006EE907AF8EEE67A2B46C7EE277A32463B
:10DA680001904349009724A8FDEEE77ACDED027AAC
:10DA780009F0D0FDC1B224A8FDF7BEFB3D4A3949E3
:10DA880024A809F0C7FDC1B224A8FDF7B5FBE8201A
:10DA9800FAF738F90546EC20FAF734F90446F0208D
:10DAA800FAF730F90646F420FAF72CF9631B07EE6B
:10DAB800903A06EE906AB8EEE77AF8EEE67A2A46E9
:10DAC800C7EE277A01902A490096234624A8FDEE3E
:10DAD800E77ACDED027A09F09DFDC1B224A8FDF7E1
:10DAE8008BFB1D9A022A06D1234924A809F0BAFD06
:10DAF80024A8142109E01D9B012B40F089821F49AD
:10DB080024A809F0AFFD24A81021FDF775FB7FE2DA
:10DB18001D9A012A40F00E8104F1C800FAF7F2F8C4
:10DB28001B9004F1CC00FAF7EDF8074604F1D00099
:10DB3800FAF7E8F81B9B1C90FF1A06EE907AB8EEED
:10DB4800E67A06EE900AF8EEE67A0024C7EE277A1F
:10DB5800FDEEE77ACDED1F7AE7E000BF1C0E00204E
:10DB680042B805083DB805084CB8050859B8050875
:10DB78005FB80508A9B80508AFB80508C4B805080E
:10DB88001C9B1B9A2046012103FB042AFFF7CFFDAB
:10DB9800914B924A18681768D3ED018A92ED019A61
:10DBA8008F4B904AD3F80090D3ED019A1368012D5A
:10DBB800209392ED018A7ED1F5EEC08AF1EE10FA3B
:10DBC80054BF4FF0000C4FF0010CB5EEC09ABCF1F9
:10DBD800000F0CBF4FF02B084FF02D08F1EE10FA94
:10DBE80054BF4FF0000E4FF0010EF5EEC09ABEF193
:10DBF800000F0CBF2B262D26F1EE10FA54BF002182
:10DC08000121B5EEC08A00290CBF4FF02B0B4FF055
:10DC18002D0BF1EE10FA54BF00220122002A0CBF8E
:10DC28002B232D231E93BCF1000F01D0F1EE688A3F
:10DC3800BEF1000F01D0B1EE499A09B1F1EE699A2F
:10DC48000AB1B1EE488A04F01FFECDE9000118EED2
:10DC5800900ACDF8088004F017FECDE90401384693
:10DC680004F012FECDE9060119EE100A089604F038
:10DC78000BFECDE90A01484604F006FECDE90C0189
:10DC880019EE900ACDF838B004F0FEFDCDE9100188
:10DC9800209804F0F9FD1E9ACDE9120118EE100A39
:10DCA800149204F0F1FD5246CDE9160124A84E491C
:10DCB80009F0B0FC2FE0022D2ED1FFF79DFC8DED71
:10DCC800220ACDED230A22AB93E8030046AB03E911
:10DCD8000300DDED457AF5EEC07AF1EE10FA4498CE
:10DCE80005D5F1EE677A17EE906A2D2702E017EE58
:10DCF800906A2B2704F0C8FD02460B463046CDE952
:10DD08000023029704F0C0FD5246CDE9040124A87F
:10DD1800364909F07FFCC6B224A83146FDF76CFAF3
:10DD28000120FDF787FF0134A4B21F9BA342BFF671
:10DD380027AF6AE11D9A022A40F06781E820F9F7C7
:10DD4800E1FF1B90EC20F9F7DDFF0646F020F9F71C
:10DD5800D9FF1B9B1C9006EE900AF61AB8EEE68ACD
:10DD680006EE906AF8EEE67A04F1C800C7EE887A03
:10DD7800FDEEE77ACDED1E7AF9F7C4FF064604F109
:10DD8800CC00F9F7BFFF074604F1D000F9F7BAFF56
:10DD9800BF1B07EE100A06EE907AF8EEC77AB8EEC7
:10DDA800E67A1B9A1F9087EE277A931B012D06EEC1
:10DDB800903ABDEEC77A88EE278A0D4B8DED207A12
:10DDC800B8EEE67A87EE277A83ED007A094B83ED81
:10DDD800008A40F0D0808FE0683B0020F8360020B1
:10DDE800F83A002098360020D5B8050810B905087B
:10DDF8006C260020AC2600201F9A002102FB04623A
:10DE080020462192FFF793FC95ED018AD8ED018A0F
:10DE1800B5EEC08AF1EE10FA54BF4FF0000C4FF087
:10DE2800010CF5EEC08A9AED019ABCF1000F0CBF07
:10DE38002B272D27F1EE10FA54BF4FF0000E4FF0AC
:10DE4800010EB5EEC09ABEF1000F0CBF4FF02B0BC0
:10DE58004FF02D0BF1EE10FA54BF00210121286874
:10DE6800D8F80090DAF8003000290CBF2B222D22B8
:10DE7800BCF1000F01D0B1EE488ABEF1000F01D00D
:10DE8800F1EE688A09B1B1EE499A19921A9304F031
:10DE9800FBFCCDE9000118EE100A029704F0F4FC2F
:10DEA800CDE90401484604F0EFFCCDE9060118EE7F
:10DEB800900ACDF820B004F0E7FC1A9BCDE90A01DE
:10DEC800184604F0E1FC199ACDE90C0119EE100A84
:10DED8000E9204F0D9FC219ACDE910014F4924A8EB
:10DEE80009F098FBC1B224A8FDF786F90134012096
:10DEF800FDF7A0FEA4B205E0494DDFF83481DFF854
:10DF080034A10024209BA342BFF676AF0024454DE0
:10DF18002DE01C9B1B9A2046022103FB0426FFF7D9
:10DF280006FC95ED018AB5EEC08AF1EE10FA286874
:10DF380003D5B1EE488A2D2700E02B2704F0A4FC76
:10DF4800CDE9000118EE100A029704F09DFC324654
:10DF5800CDE90401344924A809F05CFBC1B224A826
:10DF6800FDF74AF90120FDF765FE0134A4B21E9BB6
:10DF7800A342CEDA49E0022D47D142E01C9B1B9A0E
:10DF88000121204603FB0425FFF7D1FBFFF734FBF3
:10DF98008DED220ACDED230A22AB93E8030046ABB0
:10DFA80003E90300DDED457AF5EEC07AF1EE10FAEB
:10DFB800449806D5F1EE677A17EE908A4FF02D094E
:10DFC80003E017EE908A4FF02B0904F05DFC06463B
:10DFD8000F464046CDE90067CDF8089004F054FCA0
:10DFE8002A46CDE90401104924A809F013FBC1B25F
:10DFF80024A8FDF701F901340120FDF71BFEA4B2A6
:10E0080000E000241E9BA342B8DA084B1D9A1A7040
:10E0180047B0BDEC048BBDE8F08F00BF24B90508FC
:10E02800683B00209836002052B90508C901002035
:10E03800F8360020F83A0020F0B52DED028B0446A2
:10E048008FB0002800F04981AF4B18890419A4B299
:10E0580022B2002A05DB40F23F139A42C8BF1C4691
:10E0680000E00024F7F740FAA0B24EF29C71F7F7EF
:10E078004DFAA54B1C81A54B586804F005FC9AA3E2
:10E08800D3E9002304F054FC04F034FFA04B1860DB
:10E09800A04B1B780A2B05463DD123B206EE903AD9
:10E0A800F8EEE67A17EE900A04F0EEFB9A4B064675
:10E0B80018680F4604F0D6FB02460B468CA1D1E93E
:10E0C800000104F05FFD02460B463046394604F075
:10E0D8002FFC064628460F4604F0D6FB02460B46A0
:10E0E8003046394604F024FC00228C4B04F04AFDEB
:10E0F80004F000FF04F0C8FB02460B4604A8884958
:10E1080009F088FA0020F8F741F90520D72104AA78
:10E118000023F8F773F97F4B1B780D2B814B188878
:10E1280024B200FB04F06FD104F09CFB72A3D3E986
:10E13800002304F027FD04F0DDFE7B4B1B6806EE90
:10E14800903A07EE900AB8EEE67A784B27EE877A8F
:10E15800FCEEE77ABDEEC77A17EE900A17EE104A82
:10E168001B68012180B2E418FFF7E1FA704B714A8D
:10E17800D3ED017A704B93ED018A92ED007A38EE77
:10E18800678A28EE078A92ED017A77EE677A93ED2F
:10E19800007A67EE877A88EE278A18EE100A04F06C
:10E1A80073FB57A3D3E9002304F03EFEDFED637A47
:10E1B800002818BFB0EE678A18EE100A04F064FB56
:10E1C80041EC100B06F050FE002251EC100B5C4B9A
:10E1D80004F0AEFB04F08EFE04F056FB02460B463C
:10E1E80006A8584909F016FA9620DC2106AA002349
:10E1F800F8F704F94FF6FF7300930520DC21224657
:10E208000023FEF76DF968E004F02CFB3AA3D3E98C
:10E21800002304F0B7FC04F06DFE434B1B6806EEC8
:10E22800903A08EE100AF8EEE67ABCEEC87A68EE84
:10E23800277A17EE105AFDEEE77A3C4B17EE906AF4
:10E248001B68ADB228460121F618FFF770FAFFF7F0
:10E25800D3F98DED020ACDED030A02AC94E8030070
:10E268000AAB83E80300681C80B20121FFF75FFA5C
:10E27800FFF7C2F98DED020ACDED030A94E8030019
:10E288000EAB06EE905A03E90300B8EEE60ADDEDA0
:10E298000A0A38EE400A9DED0B1ADDED0C1A9DEDC9
:10E2A8000D2AFFF733FA8DED020ACDED030A94E843
:10E2B800030008AB83E803004FF6FF7300930520C3
:10E2C8000023DC213246FEF70BF91F4B9DED080AAF
:10E2D8001878DDED090AFEF735FF0FB0BDEC028BAB
:10E2E800F0BD00BFAFF300807B14AE47E17A843FF6
:10E2F800000000A0D954BD410000000000F07340A8
:10E30800FCA9F1D24D62503FB80D00201C0300203B
:10E318005C3B002071260020082D00200000F43FFF
:10E3280065B90508DC3A0020E42C0020F02600201E
:10E33800F8360020F83A0020983600206F12833A09
:10E34800000034406EB90508FC2C00202DE9F84384
:10E35800461F8846B6B200250D4F12E008EB0401AF
:10E3680089B23046F7F774F829F814000A20013406
:10E37800FAF7A0FE062CF1D116350136F22DB6B209
:10E3880004D06FF0040407EB0509E7E7BDE8F8835C
:10E39800183B00202DE9F04F85B00B1A0193431E5E
:10E3A8009BB20293431C441F00F1060901F1FF3A96
:10E3B80001F1010B9BB20F461646A4B21FFA89F968
:10E3C8001FFA8AFA1FFA8BFB0393804620465146B0
:10E3D8003246F7F775F8204639463246F7F770F8AF
:10E3E800204659463246F7F76BF8019B0298E51824
:10E3F800ADB229463246F7F763F840462946324619
:10E40800F7F75EF80134039829463246F7F758F8CB
:10E41800A4B20A20FAF74EFE4C45D7D105B0BDE8A4
:10E42800F08F2DE9F843461F8846B6B200250E4FF7
:10E4380012E008EB040139F8142089B23046F7F7E6
:10E448003FF801340A20FAF735FE062CF1D11635CB
:10E458000136F22DB6B204D06FF0040407EB0509BB
:10E46800E7E7BDE8F88300BF183B00202DE9F0433B
:10E478002DED068B70EE007A8DB017EE900AB0EE97
:10E48800408A10EE904A20EE009A04F0FDF9064604
:10E4980020460F4604F0F8F9F7EE008A41EC100B1D
:10E4A80041EC1A0B06F0FCFA79EE287A55EC104B81
:10E4B80017EE900A04F0E8F92246804689462B4672
:10E4C8003046394604F034FA02460B46404649467F
:10E4D80004F07AF804F00EFDB0EE4A0AF0EE6A0A8B
:10E4E80009EE900A38EEC99ADFED377A89EE299A53
:10E4F80029EE279A06F0D4FB304653EC102B394608
:10E5080004F016FA044619EE900A0D4604F0BCF918
:10E5180002460B462046294604F034FB00222B4BCA
:10E5280004F006FA04F0E6FCB4EE688ADFED287A17
:10E53800284BF1EE10FA044619EE100A08BFB0EEA7
:10E54800678A1D6804F0A0F902460B4603A8224911
:10E5580009F060F8204604F097F902460B4606A831
:10E568001E4909F057F878EE287A38EEC88A87EEFF
:10E57800888A18EE100A04F087F902460B4609A8A3
:10E58800174909F047F80520014603AA0023F7F7C1
:10E5980035FF0520142106AA0023F7F72FFFC8200E
:10E5A800052109AA0023F7F729FF4FF6E073009326
:10E5B8000520DC212A460023FDF792FF0DB0BDECB3
:10E5C800068BBDE8F08300BF0000484200004940C8
:10E5D800A4707D3FB838002077B905087FB90508D1
:10E5E80087B905082DE9F04F494B2DED048B1D78AF
:10E5F800022D85B080467BD1464E348A01212046C3
:10E60800FFF795F8FEF7F8FF8DED000ACDED010A4A
:10E618009DE8030004AB03E9030028469DED020AC8
:10E62800DDED030AFEF78EFD3B4B1A683B4B1B687A
:10E6380002FB04343A4B1C603A4BDFED3B7A93ED16
:10E64800008A68EE277A5F6817EE900A04F01CF9D2
:10E65800824638468B4604F017F941EC100B41EC22
:10E66800190B06F01DFA504653EC102B594604F0CE
:10E678005FF923A3D3E9002303F0A8FF04F01AFCF1
:10E68800B0EE490AF0EE690A054684B206F008FBC6
:10E69800504653EC102B594604F04AF90B460246F3
:10E6A80019A1D1E9000103F08FFF04F003FCB37C4A
:10E6B80081461FFA80FA1BB9B08AF18AFFF7B1FECA
:10E6C800002320465146B374FFF740FE20465146CA
:10E6D8001F22FFF75FFEB0EE480A00EE907AFFF7C0
:10E6E800C5FE338AB5829844A6F81080A6F816901D
:10E6F80005B0BDEC048BBDE8F08F00BFAFF3008020
:10E708000000000000E063400000000000C05D4021
:10E71800FC2C0020B80D0020E42C0020F02600205E
:10E72800B83800208C3A00200000C842124B1B78F1
:10E73800022B10B50CD1114B1B78022B08D1104CB1
:10E748002078C0B140B2FFF74DFF0023237010BD01
:10E758000C4C237E23B99F20F6F7A0FE01232376D5
:10E76800064B1B78022B06D1054C94F90000FFF7E5
:10E7780063FC0023237010BDFC2C0020E43800202B
:10E78800251B0020B80D0020034B00201860034B08
:10E798001870FDF78FBB00BFE4360020E438002076
:10E7A800034B00201860034B02221A70FDF782BB4E
:10E7B800E4360020E438002037B500242546A0B20E
:10E7C80028213223024601340095F7F769FCB4F595
:10E7D800A07FF4D13EBD2DE9F04F2DED088B022826
:10E7E80097B080468DED070AB34B05D0032805D0B6
:10E7F800012805D10C2202E0092200E00B221A7040
:10E808001878F2F70BFA042103914FF00009F3EEA0
:10E818000EAA9FEDAABADFEDAABA7DE1A94B1A6844
:10E82800A94B1B6802FB093307EE103A01211FFAB6
:10E8380089F0B8EEC78AFEF77AFFFEF7DDFE8DEDA8
:10E84800080ACDED090A08AD95E803000AAB83E88C
:10E8580003009E4B1A6802EBC9030EAF19689C4B64
:10E8680019600399521812685A60FEF7C5FE8DEDBB
:10E87800080ACDED090A95E803000CAB83E803000C
:10E88800DDED0A9A9DED0BAADDED0C8A9DED0D9A42
:10E89800B0EE690AF0EE4A0AB0EE681AF0EE491ACC
:10E8A800FEF7FEFB8DED080ACDED090A95E8030099
:10E8B800B0EE691AF0EE4A1A87E80300B0EE680A6B
:10E8C800F0EE490AFEF7F9FB8DED080ACDED090ACD
:10E8D80095E8030010AB83E803009DED0E0ADDED1B
:10E8E8000F0AFEF765FD8DED080ACDED090A95E8DA
:10E8F800030016AA02E903009DED100ADDED110AD6
:10E90800149EFEF755FD8DED080ACDED090A95E830
:10E91800030087E80300DDED0F0AF5EEC00AF1EE0B
:10E9280010FA48BFF1EE600A9DED0E0ACDED0F0A10
:10E93800FEF780FD8DED080ACDED090A08AA92E8D8
:10E94800030012AB83E803000798129D03F09CFFB5
:10E958005D4B139FD3F800B05E4BBDEEC87AD3F879
:10E9680000A0CDE9040117EE102A58465146FDF7DC
:10E9780061FC07EE10AAF8EEC77A07EE10BAB4EEFB
:10E98800E78AF8EEC77AF1EE10FAB4EEE78A8CBFA0
:10E9980000220122504B0690F1EE10FAD4BF00225B
:10E9A80002F00102B8F1020FDA6012D0B8F1030FD9
:10E9B8003ED0B8F1010F68D1304603F065FF36A3A9
:10E9C800D3E9002303F0B4FF0022444B03F0FEFD1B
:10E9D8002AE0284603F058FFDDE9042304460D46E3
:10E9E8002FA1D1E9000104F0CDF802460B462046DC
:10E9F800294603F09DFF2CA3D3E9002303F098FFD9
:10EA080004F078FA07EE900AC7EEAA7A17EE900A91
:10EA180003F03AFF41EC100B06F026FA002251EC05
:10EA2800100B2F4B03F084FF04F01CFA04462CE073
:10EA380018EE100A03F028FF044638460D4603F086
:10EA480023FF17A3D3E9002303F072FFDDE90423B2
:10EA580004F098F804F04EFA03F016FF14A3D3E973
:10EA6800002303F065FF02460B462046294604F0C2
:10EA780089F804F03FFA07EE900AB0EE6B7A07EED9
:10EA88008B7AFDEEC77A17EE904A002C2ADBC72C4A
:10EA9800A8BFC72427E000BF8716D9CEF753F5BF14
:10EAA8008FC2F5285CAF4340000000000090704022
:10EAB80000000080DBC48641FC2C00200000C8C395
:10EAC8000000C843E42C0020F0260020D0360020A7
:10EAD80098360020082D0020B80D0020000069405D
:10EAE800000049C00024114BDB685BB1104B18884B
:10EAF800104B1988069B4FF6FF759AB2A3B2009582
:10EB0800F7F7CEFA0B4B039A1C600699084B0832AC
:10EB1800196009F101090392074B1B884B45BFF6A1
:10EB28007DAE17B0BDEC088BBDE8F08FB80D0020A6
:10EB3800D83800207C3B0020DC3A00202DE9F04347
:10EB48002E4B85B01878F2F769F82D4B0B221A7006
:10EB58002C4B1C78012C05D006D3022C0CBF30247A
:10EB6800002402E0002400E01024274B1B78012B2E
:10EB780007D104F1C800F9F7C5F8064604F1D0003A
:10EB880004E0E820F9F7BEF80646F020F9F7BAF8ED
:10EB980000240746DFF880901C4DDFF8808020E0D5
:10EBA80007FB0463204601216B61A8F82040FEF7AB
:10EBB800BEFDFEF721FD8DED000ACDED010A9DE8B1
:10EBC800030004AB03E903000C4B9DED020A18781F
:10EBD800DDED030AFEF7B6FA6869FDF72BFD01348F
:10EBE800A4B2B9F80030A342DADA094B02221A704B
:10EBF800084B00221A7605B0BDE8F083FC2C0020F3
:10EC0800712600201C0E0020C90100209C3800201D
:10EC1800E4380020B80D0020DC3A00208C3A0020AF
:10EC28001FB5044600214FF0804002F0DCFE2E4B59
:10EC380018682E4B1B6800FB04302D4B1B6898424C
:10EC480009DB2C4B1B68984205DCFAF733FE2A4B8C
:10EC58001868FCF7EFFFFCF71FFF284A284B1168DC
:10EC6800526819605A60214B1A68214B1B68D31AE5
:10EC780006EE903A1C4B1B68B8EEE67A06EE903A20
:10EC8800F8EEE67A0021C7EE277AFCEEE77A17EE6F
:10EC9800904AA0B2FEF74BFDFEF7AEFC8DED000AE0
:10ECA800CDED010A9DE8030004AB03E90300154B11
:10ECB8009DED020A1878DDED030AFEF743FA124BC0
:10ECC8001868124B1B6824B200FB0430FDF7B2FC35
:10ECD8000F4B00224FF0804001211A7004B0BDE8AC
:10ECE800104002F080BE00BF68260020D836002001
:10ECF800E4260020D42600209C2600209C380020F2
:10ED080098360020FC2C0020E42C0020F02600205F
:10ED18009526002008B5FFF783FF0A4B1A680A4BAF
:10ED28001B689A420CDD4FF08040002102F05BFE28
:10ED3800064B02221A70064A00231370054A1376FE
:10ED480008BD00BFD8360020D4260020E4380020B3
:10ED580095260020B80D002010B500214FF0804006
:10ED680002F041FE0A4B00241C700A4B20461C701E
:10ED7800F7F736FA084B1868FAF79CFD074B08486E
:10ED880001221A70074B1C70BDE81040F2F7D5BF7E
:10ED980095260020E8360020E4260020FC2C0020E0
:10EDA800A01800207126002007EE100A034BF8EE89
:10EDB800477A0022C3ED007A5A6070470C3700206A
:10EDC80007EE100A034BF8EE477A0022C3ED007AEB
:10EDD8005A607047C03800200F4B10491A68104B12
:10EDE8001B68D31A06EE903A0E4B1B68B8EEE67A0B
:10EDF80006EE903AF8EEE67AC7EE277AFCEEE77A66
:10EE080017EE903A9AB20B80074B188890422CBFA5
:10EE180000200120704700BF082D0020DC3A0020A8
:10EE2800F0260020E42C0020E826002013B502ABD1
:10EE3800011D23ED010A054A89B213F8014B145448
:10EE4800013080B28842F8D11CBD00BF1A380020BA
:10EE58002DE9F8431F4F0740002F04460D4603DAFB
:10EE6800013F67F00F070137BFB2DFF874804FEA40
:10EE7800C7091FFA89F9484698ED000A09F10409FB
:10EE8800FFF7D4FF1FFA89F098ED010AFFF7CEFFCC
:10EE9800114B10261B8894FBF6F6F6019C42B6B27D
:10EEA8000CD1701980B20D498022FAF7A3F900B18C
:10EEB800FEE721B24FF47F70F8F7EEFE0F2F07D16F
:10EEC8007519A8B205498022FAF794F900B1FEE74E
:10EED800BDE8F8830F000080DC3A00201A380020D3
:10EEE8009C3800202DE9F043744B2DED028B1888D7
:10EEF800FF2898BF4FF4807093B0C00008F018F84E
:10EF08006F4B0546186028B90520B4216D4A2B4679
:10EF1800F7F774FA0024694F6B4E4FF000086AE067
:10EF2800FCF7BAFD20464FF44141FFF791FF674BCC
:10EF38001A685B683260002173602046FEF7F7FBB1
:10EF4800FEF75AFB8DED020ACDED030A0DF1080913
:10EF580099E803000AAB83E803005D4B9DED0A1AAC
:10EF680093ED007AD3ED017ADDED0B1A31EE470A05
:10EF780071EEE70A31EE071A71EEA71A8DED0E0A47
:10EF8800CDED0F0A8DED101ACDED111AFEF795F89B
:10EF98008DED020ACDED030A99E803000CAB83E876
:10EFA8000300FF2C4FEAC4032B4404D9C3F80080A4
:10EFB800C3F8048003E00C9A1A600D9A5A603B88E3
:10EFC80040F23F10604390FBF3F080B24FF4FC63D3
:10EFD8000246282100933223F7F762F83D4B186860
:10EFE8003D4B1B68C018FAF765FC3C4B1868FCF7EA
:10EFF80021FE0134A4B23B88A34291DA01221346D0
:10F008004FF4807105A805F03DF8354EDFF8F8801B
:10F01800294605A805F018FB08233370314B012455
:10F028001C700020F6F7AAFB2F48F2F786FE30780E
:10F03800F1F7F4FD2D4B9FED2E8ADFED2E8A1C7023
:10F048000024D5ED007AB0EE687A07EEC87A20463B
:10F05800FCEEC77A17EE906A03F004FC264B0022F8
:10F0680003F066FC03F026FFB6B2A3B2C72E28BF92
:10F07800C72687B253B1214BB8F8000019884FF65C
:10F08800FF7300933A463346F7F70AF81B4BC8F864
:10F09800007001340835B4F5807F1E60D1D1184B5B
:10F0A8001868FAF707FC114B02221A70154B002258
:10F0B8001A7613B0BDEC028BBDE8F083DC3A002071
:10F0C800D036002031B10508983600209C38002041
:10F0D8000C370020D8360020682600209C26002007
:10F0E800FC2C00207B0D0020FC170020E4380020B9
:10F0F800000016430000C8420000F43F7C3B00209B
:10F10800E4260020B80D0020D8380020F0B5294B9F
:10F11800294F2A4D2A4E012285B01A7000243AE060
:10F12800284B1A68336802FB04336B61264B1C8436
:10F13800FCF7B2FC20464FF44141FFF789FE234B10
:10F148002A681A606A6820465A600021FEF7EFFABA
:10F15800FEF752FA8DED000ACDED010A9DE8030095
:10F1680004AB03E903001A4B9DED020A1878DDEDA4
:10F17800030AFDF7E7FF6869FDF75CFA154B1868A5
:10F18800154B1B68C018FAF795FB144B1868FCF769
:10F1980051FD0134A4B23B88A342C1DA104B186870
:10F1A800FAF788FB034B02221A700E4B00221A76DC
:10F1B80005B0F0BDE4380020DC3A00209C3800207F
:10F1C800F0260020E42C00208C3A002098360020FD
:10F1D800FC2C0020D8360020682600209C26002021
:10F1E800E4260020B80D002038B5FDF7DBF80F4BFA
:10F1F8000F4C9F221A810F4B012518782570F1F7C3
:10F208000DFD0D4B00221A600C4B1B78072B04D008
:10F218000B2B07D0062B08D102E0BDE8384075E774
:10F22800257038BDBDE8384088E438BDB80D0020E9
:10F23800E4380020FC2C0020E43600207126002051
:10F248002DE9F743002581462C46154E154FDFF86A
:10F258005C801FE0FCF720FC49462046FFF7F8FDDC
:10F26800D8F800303868C018FAF724FB0E4B186835
:10F27800FCF7E0FC308895FBF0F080B24FF4FC63BB
:10F288000093282102463223F6F70AFF05F59E75FA
:10F29800013403353388A342DCDABDE8FE8300BFBE
:10F2A800DC3A0020D83600209C2600206826002062
:10F2B80010B5104C4FF47570B4F90010F8F7ECFC69
:10F2C8000D4B4FF47670B3F90010F8F7E5FC40F2F7
:10F2D800D230F8F7EFFCB02804D040F2D230B02199
:10F2E800F8F7DAFC2088FFF75FFD034B1888BDE8C4
:10F2F800104065E5C4010020C001002000210A2259
:10F3080008B509F0D7FAD0F1010038BF002008BDD0
:10F3180073B5041D0E46A4B20C2200234FF6E07507
:10F32800204601360095F6F75FFF00230C22B1B2A4
:10F3380020460095F6F758FF0D4B1B78012B16D188
:10F348000C4E0D4D308829880024043080B20C22E0
:10F3580023460094F6F748FF308829880094043043
:10F36800013180B289B20C222346F6F73DFF7CBDFD
:10F37800BC3600200A370020BC38002008B54FF6FC
:10F38800FF70F6F701FF0020F7F700F8E1202321CE
:10F398002C4A0023F7F732F8E1204621294A0023B6
:10F3A800F7F72CF8E1206921264A0023F7F726F819
:10F3B800E1208C21244A0023F7F720F82348FFF79F
:10F3C8009DFF20B121482249012208F023F94B2052
:10F3D80023211E4A0023F7F711F81E48FFF78EFF76
:10F3E80020B11C481A49012208F014F94B20462183
:10F3F800184A0023F7F702F81748FFF77FFF20B1F4
:10F4080015481349012208F005F94B206921124AD1
:10F418000023F6F7F3FF1148FFF770FF20B10F48FC
:10F428000B49012208F0F6F84B208C2100230B4AE7
:10F43800F6F7E4FF0A4B18880A4B1988BDE808401C
:10F4480066E700BF41AF050893B90508B426002058
:10F45800B7AC0508D8260020EE2C0020A0260020F6
:10F46800F43A0020BC3A002070B5044600200D464E
:10F478001646F6F78BFF0020F6F79CFE4FF4FC606B
:10F48800F6F782FE2046294656BB1E4A3346F6F753
:10F49800B5FF1D48FFF732FF20B11B481B49012269
:10F4A80008F0B8F804F17006B6B230462946164A94
:10F4B8000023F6F7A3FF1648FFF720FF20B11448F2
:10F4C8001249012208F0A6F83235ADB22046294685
:10F4D800104A0023F6F792FF304629460C4A07E007
:10F4E8000D4A0023F6F78AFF32350B4AA9B22046A7
:10F4F8000023F6F783FF094B1888094B1988BDE8E4
:10F50800704005E798B90508603B0020DCB00508A5
:10F51800D03A0020A0B905087CB10508F43A0020CB
:10F52800BC3A002030B5144D9DF80C402C70134D9A
:10F538002880134D02FB04002980124D80B22880D8
:10F54800114D2980114D2A80114A1380114B1880C2
:10F55800114B1980114B1249E2B21A7000230B703B
:10F5680010490A709DF810200134013254430E4AA4
:10F5780014700E4A137030BD783C0020583B0020B0
:10F588009A380020F43A0020BC3A002018380020AD
:10F59800843B00200A370020BC380020BE3A0020F7
:10F5A800E9360020F63A0020C4360020BC36002098
:10F5B80038B5054600200C46F6F7E8FE0020F6F7B9
:10F5C800F9FD4FF4FC60F6F7DFFD0B48FFF796FEF8
:10F5D80028B1094809490A4B002208F01BF82846B7
:10F5E80021460023044AF6F709FF064B1888064B04
:10F5F8001988BDE838408BE600370020ADB505080E
:10F608000000F03FF43A0020BC3A0020114B1B6880
:10F61800002B70B505460C4604DA5B420E480F49CC
:10F628002D2202E00C480D49202207F0F3FF0020AC
:10F63800F6F7ACFE0020F6F7BDFD4FF4FC60F6F7D8
:10F64800A3FD054A284621460023BDE87040F6F789
:10F65800D5BE00BFF03A0020C8380020A8B9050878
:10F668000F4B10B519684FF4E170F8F732FB40F210
:10F678003D114FF4E070F8F70FFB0020F6F786FE17
:10F688000020F6F797FD4FF4FC60F6F77DFD054A7C
:10F69800192064210023BDE81040F6F7AFBE00BF73
:10F6A800F03A0020B0B9050808B54FF4E070F8F753
:10F6B80001FB40F23D13984205D14FF4E170BDE8DB
:10F6C8000840F8F71FBB002008BD38B505460020E4
:10F6D8000C46F6F75BFE0020F6F76CFD4FF4FC6075
:10F6E800F6F752FD0B48FFF709FE28B109480A4909
:10F6F8000A4B002207F08EFF284621460023054AC0
:10F70800F6F77CFE064B1888064B1988BDE838408A
:10F71800FEE500BFDC360020ADB505080000F03F6F
:10F72800F43A0020BC3A002038B5C501ADB2002437
:10F73800601980B2F9F706FB0134C0B2FBF74CFD43
:10F74800A4B24FF47A70F9F7B5FC802CF0D138BD2B
:10F7580073B5104D00240E20FBF73EFD002609E08E
:10F768000DF10700FBF749FD20B19DF80730AB55B7
:10F778000136F6B23306F3D5E00180B2054980229E
:10F78800F9F738FD00B1FEE70134A4B2B4F5007F03
:10F79800E1D17CBD1A38002007EE100AF8EE477A4E
:10F7A8007FB517EE900A03F06FF802460B4601A8E2
:10F7B800054907F02FFF0A20962101AA0023F6F732
:10F7C8001DFE07B000BD00BFB7B905082DE9F34716
:10F7D80000240746B0F5024F14BF4FF0910A4FF0CE
:10F7E800690A25462E4EA0460DE094FBF0F080B243
:10F7F800462102465023CDF80080F6F751FC04F567
:10F808009E74013503343088A842EEDA0020F6F7FA
:10F81800D1FC4FF4FC60F6F7B7FC00258C2051466C
:10F828003F220023F6F7CCFD2C461D4EDFF87C80E6
:10F83800DFF87C9027E0F9F7C9FE88ED000AF9F7B0
:10F84800CBFE394688ED010A2046FFF701FB154B30
:10F858001868D9F8003000FB0430FAF72BF8124B7F
:10F868001868FCF7E7F9308895FBF0F080B24FF4A0
:10F87800FC630093462102465023F6F711FC05F578
:10F888009E75013403353388A342D4DA8C2051465F
:10F898003C22002302B0BDE8F047F6F791BD00BF57
:10F8A800DC3A0020682600209C2600209C38002096
:10F8B800E426002070B53E4B3E4E3F4D01222DED13
:10F8C800048B1A703D4B00241C609FED3D9A5BE051
:10F8D800F9F77CFEF0EE408AF9F77EFE20464FF4F9
:10F8E8004141B0EE408A85ED010AC5ED008AFFF777
:10F8F800AFFAA0B20021FDF71AFF324BD3ED017A1F
:10F90800314B38EE678A93ED007A28EE078A93ED3B
:10F91800017A77EE677A67EEA88A88EE288A18EE69
:10F92800100A02F0B1FF20A3D3E9002303F07CFA08
:10F93800002818BFB0EE498A18EE100A02F0A4FF9A
:10F9480041EC100B05F090FA002251EC100B1F4B04
:10F9580002F0EEFF03F0CEFA1D4B18601D4B18683D
:10F968001D4B1B6800FB04306861FCF763FE1B4BF2
:10F9780018681B4B1B6800FB0430F9F79BFF194BF9
:10F988001868FCF757F901343388A342A0DA164BFC
:10F998009F221A8100221A76054B02221A70BDECAA
:10F9A800048B70BDAFF30080FCA9F1D24D62503FCB
:10F9B800E4380020DC3A00209C380020E43600209F
:10F9C8006F12833AF8360020F83A002000003440DD
:10F9D800C0360020E42C0020F026002068260020F5
:10F9E800E42600209C260020B80D0020AFF30080FC
:10F9F8000EB403B070470A2810B5044602D10D2092
:10FA0800FFF7F9FF064A13681BB103F8014B1360AF
:10FA180010BD044B1B680BB12046984710BD00BFB2
:10FA2800D80D00207C3C002010B5044601E0FFF70B
:10FA3800E2FF14F8010B0028F9D110BD2DE9F04FB1
:10FA4800044685B00D464FF00A0A00E03546207896
:10FA5800002800F0C480252801D0013467E06078D0
:10FA6800302803D1A0780123033407E02D2802D0E1
:10FA78000234002302E0A078022303344FF0000888
:10FA880005E00AFB080814F8010BA8F13008A0F1FA
:10FA98003002D2B2092AF4D96C2801D04C2803D1FB
:10FAA80014F8010B43F00403002800F09880602844
:10FAB80086BFA0F12002D2B202464F2A3DD006D816
:10FAC800432A2DD0442A09D0422A30D133E0552A7E
:10FAD80004D0582A29D0532A29D101E00A272DE039
:10FAE8002E1D2F68002500E001357A5D002AFBD124
:10FAF80004E02020FFF77FFF4D4601E0980704D47B
:10FB0800454505F10109F4D34D463846FFF78CFF0A
:10FB180003E02020FFF76FFF01354545F9D395E74E
:10FB280028782E1DFFF767FF90E7102706E0FFF7FC
:10FB380062FF2E468AE7022700E008272E1D442A86
:10FB4800296804D1002902DA494243F00803002257
:10FB580000E02A46B1FBF7FE07FB1E11CDB2092DC6
:10FB6800714607D9782814BF4FF0070C4FF0270CBF
:10FB78006544EDB230350DF80250551CBEF1000F4A
:10FB880002D0102DE5D10F22190705D504A94D196A
:10FB98002D2105F8101C951C13F0010F0CBF4FF018
:10FBA800200B4FF0300B9B072F4604D508E0584632
:10FBB800FFF721FF4F46474507F10109F7D34F46A5
:10FBC800013D1DF80500FFF716FF002DF8D103E0F1
:10FBD8002020FFF710FF01374745F9D336E705B076
:10FBE800BDE8F08F70B5064D0C462E68286001E020
:10FBF800FFF701FF14F8010B0028F9D12E6070BD42
:10FC08007C3C00200FB407B504A951F8040B0191FE
:10FC1800FFF714FFBDE80E4004B070470EB417B5E7
:10FC280005A9084C51F8043B206018460191FFF7DC
:10FC380005FF2268002313702360BDE81E4003B04F
:10FC4800704700BFD80D00200EB433B505A9074C86
:10FC580051F8043B2568206018460191FFF7EEFE35
:10FC68002560BDE83C4003B0704700BF7C3C0020E5
:10FC780070B51E4604461C481546FFF7C3FF022E02
:10FC88001FD0042E25D0012E2AD105E0A15D1748EA
:10FC9800FFF7B8FF013600E00026AE42F6DB202071
:10FCA800FFF7A9FE002609E0A05DA0F12003DBB262
:10FCB8005E2B88BF2E20FFF79EFE0136AE42F3DB97
:10FCC8000EE034F8021B0A48FFF79CFF013DF8D10B
:10FCD80006E054F8041B0748FFF794FF013DF8D1EC
:10FCE8000A20BDE8704086E6BEB90508C5B9050812
:10FCF800CBB90508D1B9050808B501214FF48070C2
:10FD080001F07CFA4FF480700021BDE8084001F052
:10FD180075BA43680A6823F0407323F48073134369
:10FD28000A7943EA02234360CA680B6930B51A436B
:10FD380084688D68084B2A43234013434A7943EA71
:10FD4800420383600B7DC26A013B22F47002DBB27E
:10FD580042EA0353C36230BDFDF7FFC000230360CE
:10FD6800037143718360C3600361012303757047A6
:10FD7800074A084B516810B50B4090E81200214320
:10FD88008468C068214301430B43536010BD00BF22
:10FD980000230140E030FCFF0023036043608360E0
:10FDA800C3607047836811B143F0010301E023F099
:10FDB800010383607047436823F4400323F400730E
:10FDC8000B4343607047416282627047436823F087
:10FDD8001F030B4343607047044B5A6810B142F449
:10FDE800000201E022F400025A607047002301403B
:10FDF800044B5A6810B142F4800201E022F48002F8
:10FE08005A60704700230140092970B50CB20CD91B
:10FE180004EB44041E3CC6680725A54026EA0505F0
:10FE2800A34045EA0304C4600AE0066904EB4404FD
:10FE38000725A54026EA050513FA04F42C430461B6
:10FE4800062A0CD80523013A5A43446B1F239340D2
:10FE580024EA0303914043EA0102426370BD0C2A7D
:10FE680012B20CD802EB8202233A046B1F23934090
:10FE780024EA0303914043EA0102026370BD02EBE6
:10FE88008202413AC46A1F23934024EA0303914043
:10FE980043EA0102C26270BD836843F08043836015
:10FEA80070478068C0F380507047836811B143F48D
:10FEB800806301E023F4806383607047836811B135
:10FEC80043F0020301E023F00203836070474368B4
:10FED800013923F4604343EA413343607047436880
:10FEE80011B143F4006301E023F4006343607047F9
:10FEF800C06C80B27047014B1868704708230140F6
:10FF0800836811B143F4807301E023F48073836044
:10FF18007047836811B143F4007301E023F4007360
:10FF280083607047044B5A6810B142F4005201E0F4
:10FF380022F400525A60704700230140092970B525
:10FF48000CB20CD904EB44041E3CC6680725A54036
:10FF580026EA0505A34045EA0304C4600AE00669E9
:10FF680004EB44040725A54026EA050513FA04F422
:10FF78002C430461836BC3F30154121B0232D2B2C7
:10FF880002EB82021F24944023EA040391400B43AE
:10FF9800836370BD836B013923F4401343EA015333
:10FFA8008363704782B0002301930190019BCB18B3
:10FFB8000193019B1A6002B07047836823F4702391
:10FFC8000B4383607047836823F440130B438360BB
:10FFD8007047836843F48003836070478068C0F388
:10FFE80080507047436811B143F4806301E023F403
:08FFF800806343607047436819
:020000040801F1
:1000000011B143F4805301E023F4805343607047FF
:1000100082B0002301930190019B28335B18019368
:10002000019B186880B202B070470123C9B213FA6D
:1000300001F143680AB1194301E023EA010141607B
:100040007047036819420CBF002001207047C94364
:10005000016070474368006810EA112007D0012250
:10006000C9B212FA01F119420CBF002001207047F9
:100070006FEA112101607047036823F001030360F8
:100080000023036043608360C360036121234361F5
:100090002C4B98421CD02C4B984220D02B4B984292
:1000A00025D02B4B98422AD02A4B98422FD02A4B4E
:1000B000984233D0294B984237D0294B984204D1EB
:1000C0004FF03D5243F8AC2C7047264B984203D179
:1000D0003D2243F8082C7047234B984204D14FF43B
:1000E000746243F8202C7047204B984204D14FF49F
:1000F000741243F8382C70471D4B984204D14FF0CE
:10010000746243F8502C70471A4B984203D11A4A34
:1001100043F8642C7047194B984203D1184A43F8AE
:100120007C2C7047174B984203D1174A43F8942C04
:100130007047164B984204BF4FF03D5243F8AC2C29
:10014000704700BF106002402860024040600240DB
:10015000586002407060024088600240A060024027
:10016000B8600240106402402864024040640240CB
:1001700058640240706402403D00002088640240E0
:10018000400F0020A064024000003D20B8640240FF
:100190000268134B10B51340CC680A6822434C69BF
:1001A00022438C692243CC6922430C6A22434C6A65
:1001B00022438C6A22434C6B22438C6B22431343B1
:1001C000036042690C6BCB6A22F00702234313439E
:1001D00043610B6943604B6883608B68C36010BDEB
:1001E0003F801CF00023036043608360C3600361B1
:1001F00043618361C361036243628362C3620363D9
:10020000436383637047036811B143F0010301E066
:1002100023F0010303607047036811B143F4004306
:1002200001E023F4004303607047036811B143F019
:10023000200301E023F02003036070474160704712
:10024000406880B27047036812B143F4002301E0B4
:1002500023F40023036001617047036811B143F484
:10026000802301E023F48023036070470AB1016119
:100270007047C16070470068C0F3C04070470068B5
:1002800000F001007047406900F0380070470A4AEA
:100290000A4B10B50A4CA04288BF13468A004CBFD7
:1002A0005B681B6821F0F02121F0821119420CBF1C
:1002B0000020012010BD00BF006402400060024029
:1002C0000F64024010B5084B084A094CA04288BF91
:1002D000134611F0005F21F0F02121F0821114BFCC
:1002E000D960996010BD00BF006002400064024008
:1002F0000F6402400B0607D5436912B143F0800337
:1003000001E023F080034361802909D001F01E0140
:10031000036812B119430160704723EA01010160CB
:100320007047124B124A10B5124CA0428CBF1446B3
:100330001C4621F0F02323F0C3132BB1026802F016
:100340001E0202EAD12202E0426902F08002880025
:100350004CBF6368236821F0F02121F0821018401F
:1003600002D0101C18BF012010BD00BF0060024069
:10037000006402400F64024010B5084B084A094C63
:10038000A04288BF134611F0005F21F0F02121F058
:10039000821114BFD960996010BD00BF0060024097
:1003A000006402400F640240044B00221A605A604D
:1003B0009A60DA60024A5A61704700BF003C01400F
:1003C000FFFF7F00837910B5002B29D01A4B0168FD
:1003D0001C68CA4314401C605C6822405A60027961
:1003E00002F1804202F59E321468214311600268D6
:1003F0009C68D1430C409C60DC682140D960417905
:10040000102906D1996811439960D9680A43DA60C6
:1004100010BD01F1804303F59E3319680A4308E0DB
:100420000379016803F1804303F59E331A6822EAD9
:1004300001021A6010BD00BF003C014000230C22E5
:1004400003600371427183717047024B1A69024362
:100450001A617047003C0140034B5B6918420CBFB6
:1004600000200120704700BF003C0140014B586153
:10047000704700BF003C0140054B1A685B690340B0
:1004800004D010420CBF002001207047184670476E
:10049000003C0140014B5861704700BF003C0140E7
:1004A0004FF0204318B943F2DB021A6003E043F235
:1004B000D20243F820204FF02042411C6FF07043DD
:1004C00042F8213002F5827242F82030704770B550
:1004D00084684568C368C16A026825431D4303698F
:1004E0001D4343691D4383691D43C3691D43036A5B
:1004F0001D43436A1D43836A1D43036B0D431D4324
:100500004FF02043082C43F8225005D153F82240E5
:1005100044F0400443F82240436B9E691D68354314
:100520005E6845EA06159E6845EA0625DE6845EAE6
:1005300006451E695B6945EA0655541C45EA036594
:100540004FF02043B1F5804F43F8245010D1836B16
:10055000986919680143586841EA0011986841EAAE
:10056000002118695B6941EA005141EA036101E039
:100570006FF07041014B43F8221070BD040100A0E0
:10058000022242604FF480524262416B4FF40052AB
:1005900010B5826200230F22FF2403608360C360D2
:1005A000036143618361C3610362C36203630A60E1
:1005B0004A608C60CA600A614A618B61816B0A6023
:1005C0004A608C60CA600A614A618B6110BD4FF05D
:1005D000204321B153F8202042F0010203E053F8F8
:1005E0002010024A0A4043F820207047FEFF0F0007
:1005F00010280CBF064B074B4FF040024FF018017C
:1006000019605A604FF0FC329A60DA60704700BFA0
:10061000600000A0800000A030B5836844681C43DF
:10062000C36844F008041C4303691C43436944EA5B
:100630004324836944EA4334C36999685A680904C6
:1006400041EA02211A68DB68114341EA0361036A47
:100650009A685D68120442EA05221D68DB682A4335
:1006600042EA03620368102B0CBF034B034B1C6070
:100670009960DA6030BD00BF600000A0800000A07B
:1006800010230360C269002343608360C360036179
:1006900043618361FC23136053609360D360026AFB
:1006A000136053609360D360704741B110280CBF52
:1006B000074B084B1A6842F004021A607047102872
:1006C0000CBF034A034A044B11680B401360704788
:1006D000600000A0800000A0FBFF0F0041B11028C7
:1006E0000CBF084B084B1A6842F040021A60704772
:1006F00010280CBF034A044A044B11680B401360D6
:10070000704700BF600000A0800000A0BFFF0F0086
:10071000102802D1024B58697047024B5869704744
:10072000600000A0800000A0054B18221A60002283
:100730005A604FF0FC329A60DA601A61704700BF6D
:10074000A00000A00268436842F0100242EA43227F
:10075000836842EA4332144B10B51A60C26891684C
:100760005468090441EA04211468D268214341EA2B
:1007700002629A60026991685468090441EA04219E
:100780001468D268214341EA0262DA6042699168E2
:100790005068090441EA00211068D268014341EA27
:1007A00002621A6110BD00BFA00000A0C268002351
:1007B000036043608360FC23136053609360D360E5
:1007C0000269136053609360D360426913605360A1
:1007D0009360D3607047054B18B11A6842F0040269
:1007E00002E01968024A0A401A607047A00000A09F
:1007F000FBFF0F0062B1102801D10E4B03E0B0F5F2
:10080000807F03D10C4B5A68114311E00B4BFAE780
:10081000102804D1074B5A6822EA010108E0B0F51C
:10082000807F0CBF044B054B5A686FEA01011140F1
:1008300059607047600000A0800000A0A00000A0E8
:10084000102801D1064B04E0B0F5807F0CBF054BAA
:10085000054B5B680B420CBF00200120704700BFB6
:10086000600000A0800000A0A00000A0102804D11B
:10087000074B5A6822EA010108E0B0F5807F0CBFFF
:10088000044B054B5A686FEA0101114059607047EB
:10089000600000A0800000A0A00000A0102801D1EE
:1008A000084B04E0B0F5807F0CBF074B074B5B683B
:1008B00013EA010004D013EAD1010CBF002001208B
:1008C000704700BF600000A0800000A0A00000A052
:1008D000102804D1084B5A6822EAD10109E0B0F58A
:1008E000807F0CBF054B064B5A684FEAD10122EAC4
:1008F00001015960704700BF600000A0800000A0A7
:10090000A00000A008B52C4B984205D1012001465B
:1009100000F048FC012048E0284B984205D1022015
:10092000012100F03FFC02203FE0254B984205D119
:100930000420012100F036FC042036E0214B9842CF
:1009400005D10820012100F02DFC08202DE01E4BD0
:10095000984205D11020012100F024FC102024E051
:100960001A4B984205D12020012100F01BFC2020C9
:100970001BE0174B984205D14020012100F012FCEA
:10098000402012E0134B984205D18020012100F055
:1009900009FC802009E0104B98420BD14FF4807085
:1009A000012100F0FFFB4FF480700021BDE80840FA
:1009B00000F0F8BB08BD00BF000002400004024088
:1009C00000080240000C02400010024000140240E7
:1009D00000180240001C0240002002402DE9F047B0
:1009E0000023D1F800801A464FF0010C03270CFABF
:1009F00002F404EA0805A5422ED1066817FA03F4AA
:100A0000E443264006600E79D0F8009006FA03FA17
:100A1000013E4AEA0909012EC0F8009014D8866800
:100A200091F8059026408660866809FA03F949EA3C
:100A300006068660466826EA050545608D794668A3
:100A40009540ADB235434560C5682C40C460CC7953
:100A5000C5689C402C43C46001320233102AC6D1C1
:100A6000BDE8F0874FF6FF73036000230371437105
:100A70008371C371704782B04FF480330193019B3F
:100A80000B430193019BC361C161019BC361C369B6
:100A90000193C369019302B07047036919420CBF07
:100AA000002001207047006980B2704743691942F5
:100AB0000CBF002001207047406980B2704701835D
:100AC0007047418370470AB1018370474183704783
:100AD0004161704743694B404361704701F0070330
:100AE000C908083130B59B0050F821500F249C40B4
:100AF00025EA040440F8214050F8214012FA03F39B
:100B00001C4340F8214030BD08B5134B984207D133
:100B10004FF40010012100F069FB4FF4001014E0C5
:100B20000E4B984207D14FF48000012100F05EFB8C
:100B30004FF4800009E00A4B98420BD14FF40000BB
:100B4000012100F053FB4FF400000021BDE80840F4
:100B500000F04CBB08BD00BF0054004000580040EE
:100B6000005C00407FB50446868868460D4600F06C
:100B70006DFA02992C482B6826F03F063604B1FB2B
:100B8000F0F0360C80B20643A680228822F00102E3
:100B90001204120C2280254A93420AD85B00B1FB52
:100BA000F3F301309BB280B22084032B98BF04235F
:100BB00021E0EE884BF6FF72964205D103225343A3
:100BC000B1FBF3F39BB206E019225343B1FBF3F3FD
:100BD0009BB243F480431A054FF4967208BF43F06A
:100BE000010350434FF47A7290FBF2F0013080B26F
:100BF00043F400432084A38323886989AA889BB295
:100C000043F001032380238823F4816323F002034C
:100C10001B040A431B0C13439BB223802A89AB8914
:100C200013439BB223817FBD40420F00A086010089
:100C300041F288330360002383804BF6FF72038107
:100C400043814FF48043C28083817047038819B188
:100C50009BB243F0010303E023F001031B041B0CD0
:100C600003807047038819B19BB243F4807303E09B
:100C700023F480731B041B0C03807047038819B195
:100C80009BB243F4007303E023F400731B041B0CBA
:100C90000380704712B141F0010101E001F0FE0153
:100CA00001827047038819B19BB243F4806303E06B
:100CB00023F480631B041B0C0380704783899BB261
:100CC00001F0FE0123F0FE030B438381704783890B
:100CD00019B19BB243F0010303E023F001031B04AD
:100CE0001B0C83817047038819B19BB243F040030A
:100CF00003E023F040031B041B0C038070470388B0
:100D000029B16FEA43436FEA53439BB201E05B04AE
:100D10005B0C03807047038819B99BB243F08003D2
:100D200003E023F080031B041B0C03807047B1F524
:100D3000804F838B04D023F480431B041B0C02E000
:100D40009BB243F4804383837047B1F5006F0388FF
:100D500003D19BB243F4006303E023F400631B045C
:100D60001B0C03807047B1F5005F038803D19BB271
:100D700043F4005303E023F400531B041B0C0380D3
:100D80007047038819B19BB243F0100303E023F0CE
:100D900010031B041B0C0380704701827047008AFC
:100DA000C0B27047038819B19BB243F4805303E08B
:100DB00023F480531B041B0C03807047B1F5006FB4
:100DC000038803D19BB243F4006303E023F4006380
:100DD0001B041B0C03807047038819B19BB243F0BE
:100DE000200303E023F020031B041B0C0380704747
:100DF000008BC0F307207047838819B19BB243F47E
:100E0000006303E023F400631B041B0C8380704722
:100E1000838819B19BB243F4805303E023F48053D9
:100E20001B041B0C8380704782B000230193019048
:100E3000019BCB180193019B188880B202B07047C8
:100E400083889BB20AB1194301E023EA0101818042
:100E50007047838A008B9BB243EA0040084020F031
:100E60007F40431A584240EB03007047838A008B4F
:100E70009BB243EA004020F07F40704782B00023DD
:100E8000009301930B0F01900093009B21F07F4191
:100E900013B1019B143302E0019B090C1833019339
:100EA000019B1B6819420CBF0020012002B0704753
:100EB000C94389B2818270478388808A80B20840A2
:100EC0009BB206D001F0E06113EA11410CBF002093
:100ED00001207047C94389B2818270470A4B1A6862
:100EE00042F001021A6000229A60196821F08471B0
:100EF00021F48031196005495960196821F4802175
:100F00001960DA60704700BF0038024010300024DA
:100F1000024B00221A701870704700BF023802405E
:100F2000034B1A6822F0F80242EAC0021A607047C6
:100F300000380240014B1860704700BF0000474274
:100F4000064B002201281A701A7002D0042804D11E
:100F500001E01870704705221A707047703802401F
:100F6000014B1860704700BF800E4742014341EAC1
:100F7000821200995B08013B42EA016141EA0341A8
:100F8000014B5960704700BF00380240014B1860A8
:100F9000704700BF600047428001034B40EA017187
:100FA000C3F88410704700BF00380240014B18603E
:100FB000704700BF68004742014B1860704700BF90
:100FC0004C004742034B9A6822F0EC6202430A430A
:100FD0009A60704700380240034B9A6822F07842CA
:100FE00002430A439A60704700380240034B9A68F4
:100FF00022F0030202439A60704700BF00380240AB
:10100000024B986800F00C00704700BF00380240A7
:10101000034B9A6822F0F00202439A60704700BFC7
:1010200000380240034B9A6822F4E05202439A606F
:10103000704700BF00380240034B9A6822F46042B8
:1010400042EAC0029A607047003802401E4B9A681C
:1010500002F00C02042A10B503D0082A03D01B4B5F
:1010600018E01B4B16E059685A6811F4800F596854
:1010700014BF174B154B02F03F02B3FBF2F3124AB9
:101080005268C2F30142C1F3881101324B4352004E
:10109000B3FBF2F30C4903608B680E4A0468C3F398
:1010A0000313D35C34FA03F343608C68C4F38224E3
:1010B000145D33FA04F484608968C1F34231525CF0
:1010C000D340C36010BD00BF003802400024F400CC
:1010D00000127A003403002000F44073B3F5407F1F
:1010E000084B08D1996820F0704221F4F81122F4DD
:1010F00040720A439A601A6F000542EA105018675E
:10110000704700BF00380240014B1860704700BFB5
:101110003C0E4742014B1860704700BF400E4742EB
:10112000014B1860704700BF5C014742044B1A6BCB
:1011300009B1104301E022EA00001863704700BFC4
:1011400000380240044B5A6B09B1104301E022EA17
:1011500000005863704700BF00380240044B9A6B90
:1011600009B1104301E022EA00009863704700BF14
:1011700000380240044B1A6C09B1104301E022EA26
:1011800000001864704700BF00380240044B5A6CDE
:1011900009B1104301E022EA00005864704700BF23
:1011A00000380240044B1A6909B1104301E022EAF9
:1011B00000001861704700BF00380240044B5A69B4
:1011C00009B1104301E022EA00005861704700BFF6
:1011D00000380240044B9A6909B1104301E022EA49
:1011E00000009861704700BF00380240044B1A6A43
:1011F00009B1104301E022EA00001862704700BF05
:1012000000380240044B5A6A09B1104301E022EA57
:1012100000005862704700BF00380240044B1A6D4E
:1012200009B1104301E022EA00001865704700BFD1
:1012300000380240044B5A6D09B1104301E022EA24
:1012400000005865704700BF00380240044B9A6D9B
:1012500009B1104301E022EA00009865704700BF21
:1012600000380240044B1A6E09B1104301E022EA33
:1012700000001866704700BF00380240044B5A6EE9
:1012800009B1104301E022EA00005866704700BF30
:1012900000380240044B1A7809B1104301E022EAF9
:1012A00000001870704700BF0D3802404309012B41
:1012B000074A01D1136803E0022B0CBF136F536F71
:1012C00000F01F0033FA00F000F00100704700BF8B
:1012D0000038024007B5002301933120FFF7E6FFF5
:1012E000019B01330193019BB3F5A06F01D000284E
:1012F000F3D03120FFF7DAFF003018BF01200EBD18
:10130000024B5A6F42F080725A67704700380240B1
:10131000034BDB6818420CBF00200120704700BF60
:1013200000380240014B1870704700BF0E38024071
:1013300008B5154B98420BD101214FF48050FFF7AF
:1013400061FF4FF480500021BDE80840FFF75ABF0D
:101350000E4B984207D14FF480400121FFF746FF22
:101360004FF4804009E00A4B98420BD14FF4004003
:101370000121FFF73BFF4FF400400021BDE808408A
:10138000FFF734BF08BD00BF003001400038004007
:10139000003C00400B88028810B54C8823438C88A1
:1013A0002343CC8823430C8923434C8923438C89D2
:1013B0002343CC8902F44152234313439BB203805D
:1013C000838B23F400631B041B0C83830B8A03822F
:1013D00010BD838B23F47B6323F00F031B041B0CD2
:1013E0008383022303848B68F0B5858B022BADB217
:1013F00038D0294A8E889468002E14BF0226012610
:10140000240203D5946824F400049460D2F8844044
:10141000D2F884705268DFF884C002F03F02BCFB4F
:10142000F2F2C4F388145443C7F30272B4FBF2F42B
:10143000CA88B2F5007F4FF00A0201D1240A02E007
:101440007601B4FBF6F46243B2FBF3F305330A22F0
:101450009BB2B3FBF2F303F001021202C3F34F039A
:1014600092B200E000229C1EA4B2FE2C28BF0022F3
:10147000CC8828BF0223134323439BB203840B88E9
:101480004A882B4343F4006313438A8813438A89B1
:1014900013439BB28383F0BD0038024000127A00F0
:1014A0000023038043808380C38003814381838141
:1014B000C3810723038270470023022203804380F5
:1014C0008380C380826083817047038819B19BB297
:1014D00043F0400303E023F040031B041B0C038094
:1014E0007047838B19B19BB243F4806303E023F40C
:1014F00080631B041B0C83837047038823F4006301
:101500001B041B0C038003889BB20B4303807047B2
:10151000B1F5804F038803D19BB243F4804303E0CD
:1015200023F480431B041B0C038070474FF6FF63BA
:101530009942038803D09BB243F4807303E023F401
:1015400080731B041B0C03807047838819B19BB206
:1015500043F0040303E023F004031B041B0C83800B
:101560007047838819B19BB243F0100303E023F066
:1015700010031B041B0C83807047838B23F47B6355
:1015800023F00F031B041B0C8383022303840B88AB
:10159000828BB3F5007F10B592B205D0002B0CBF43
:1015A0004FF48073002301E04FF480734C88224392
:1015B0008C88898942F4006222430A4392B2134321
:1015C000838310BD808980B2704781817047038812
:1015D00019B19BB243F4005303E023F400531B04FE
:1015E0001B0C0380704703889BB243F48053038035
:1015F0007047012902D0008B80B27047808A80B288
:101600007047008A80B2704783889BB20AB1194341
:1016100001E023EA010181807047090901238B4021
:101620009BB21AB1828892B2134303E0828892B2CD
:1016300022EA030383807047038919420CBF00200C
:1016400001207047C94389B20181704710B5848871
:101650000089012301F00F0280B213FA02F2104058
:10166000A4B205D009098B401C420CBF0020012008
:1016700010BD01F00F0101238B40DB439BB20381BE
:10168000704700BF08B501214FF48040FFF7BAFD55
:101690004FF480400021BDE80840FFF7B3BD014B87
:1016A000186070470038014001F0030289080A4BB6
:1016B000023130B5920053F821500F24944025EAAE
:1016C000040443F8214053F8214010FA02F2144375
:1016D00043F8214030BD00BF00380140014B186085
:1016E000704700BFDC002742014B1860704700BF05
:1016F00000042742024B186AC0F30020704700BF65
:101700000038014030B5048C24F001042404240C7A
:101710000484058B048CADB2A4B225F0F305154307
:1017200024F00A0445EA031544F00104ADB20C4369
:101730000583048430BD30B5048C24F010042404E7
:10174000240C0484048B058C24F44074ADB224056D
:10175000240D25F0A00544EA022445F0100544EAD2
:10176000033445EA0115A4B2ADB20483058430BD4B
:1017700008B5474B984205D101200146FFF742FDCD
:1017800001203DE0B0F1804F05D101200146FFF777
:101790002DFD012076E03F4B984205D1022001212A
:1017A000FFF724FD02206DE03B4B984205D1042059
:1017B0000121FFF71BFD042064E0384B984205D15E
:1017C00008200121FFF712FD08205BE0344B98420E
:1017D00005D110200121FFF709FD102052E0314B07
:1017E000984205D120200121FFF700FD202049E08B
:1017F0002D4B984209D102200121FFF703FD022061
:101800000021BDE80840FFF7FDBC284B984207D1F6
:101810004FF480300121FFF7F5FC4FF48030EFE703
:10182000234B984207D14FF400300121FFF7EAFC27
:101830004FF40030E4E71F4B984207D14FF480206B
:101840000121FFF7DFFC4FF48020D9E71A4B9842C3
:1018500005D140200121FFF7C9FC402012E0174BC1
:10186000984205D180200121FFF7C0FC802009E0CB
:10187000134B98420BD14FF480700121FFF7B6FC57
:101880004FF480700021BDE80840FFF7AFBC08BDF1
:10189000000001400004004000080040000C00402F
:1018A00000100040001400400004014000400140CE
:1018B000004401400048014000180040001C004066
:1018C000002000401C4A038890429BB212D002F5CF
:1018D000806290420ED0B0F1804F0BD0A2F58032E2
:1018E000904207D002F58062904203D002F58062F8
:1018F000904203D14A8823F0700313430F4A904269
:1019000008D002F58062904204D023F440730A8923
:101910009BB2134303804B68C3620B880385064B5D
:10192000984203D003F58063984201D18B7A0386F5
:1019300001238382704700BF000001400010004077
:101940004FF0FF33436000230380038143808372A1
:101950007047018582827047038823F070031B045F
:101960001B0C0B430380704741627047C162704794
:10197000406A7047008D80B27047038819B19BB2EE
:1019800043F0020303E023F002031B041B0C03805B
:101990007047038819B19BB243F0040303E023F0BE
:1019A00004031B041B0C03807047038819B19BB20E
:1019B00043F0800303E023F080031B041B0C03802F
:1019C0007047038823F008031B041B0C0380038863
:1019D0009BB20B4303807047038823F440731B04BE
:1019E0001B0C038003889BB20B4303807047038862
:1019F00019B19BB243F0010303E023F001031B0480
:101A00001B0C03807047038C23F001031B041B0C89
:101A1000038470B5038C8488028B0D884E8822F075
:101A200073021204120C2A438D8923F002031B0453
:101A300035431B0CADB22B430E4DA842A4B203D0CC
:101A400005F58065A8420ED1CD894E8A23F00803A2
:101A50002B438D8823F004032B430D8A354324F454
:101A60004074ADB22C43848002838A68426303844D
:101A700070BD00BF00000140038C23F010031B0465
:101A80001B0C0384038C828830B5048B0D8824F4EE
:101A9000E6442404240C23F0200344EA05241B0418
:101AA0008D891B0C43EA05134D8843EA0513134D3A
:101AB000A84292B2A4B29BB203D005F58065A842B9
:101AC00015D1CD8923F080039BB243EA05134FF66D
:101AD000BF751D408B8845EA03130D8A22F44062CE
:101AE00042EA85024D8A42EA85029BB292B2828026
:101AF0008A6804838263038430BD00BF0000014014
:101B0000038C23F480731B041B0C0384038C8288D6
:101B100030B5848B0D8824F073042404240C23F442
:101B200000731B042C438D891B0C43EA05234D884D
:101B300043EA0523124DA84292B29BB203D005F5A9
:101B40008065A84215D1CD8923F400639BB243EA96
:101B500005234FF6FF351D408B8845EA03230D8A88
:101B600022F4405242EA05124D8A42EA05129BB223
:101B700092B282808A688483C263038430BD00BFCE
:101B800000000140038C23F480531B041B0C0384CE
:101B9000038C30B58488828B0D8822F4E6421204CF
:101BA000120C23F4005342EA05221B048D891B0CFE
:101BB00043EA05334D8843EA05330B4DA842A4B2EE
:101BC00092B29BB203D005F58065A84205D10D8A7B
:101BD00024F4804444EA8514A4B2848082838A6811
:101BE0000264038430BD00BF000001400023038075
:101BF0004380838083608381C381038243827047F3
